:10000000F01F001059B200008B2900008B2900005E
:100010008B2900008B2900008B29000000000000C4
:100020000000000000000000000000008B2900001C
:100030008B290000000000008B29000091230000A4
:1000400045AA000045AA000045AA000045AA0000F4
:1000500045AA000045AA000045AA000045AA0000E4
:1000600045AA000045AA000045AA000045AA0000D4
:1000700045AA000089290000892900003D280000C8
:10008000DD230000F52300000D24000025240000DE
:10009000892900005D2400008929000089290000C9
:1000A0008929000089290000892900008929000088
:1000B0008929000089290000892900008929000078
:1000C0000B4900238868C96810B500220BF0FAFDBF
:1000D000084C03000120002B09D0B8340023A0688D
:1000E000E16800220BF0EEFD43425841400010BD94
:1000F000180C0010700B0010F7B503270092019345
:100100000A4E013FB268F36834687568B261F36102
:1001100034617561103E002FF3D1054B18605960B2
:100120000099019A034B19605A60F7BD380C001012
:10013000180C0010200C0010F8B51F00064B04002E
:100140001B780D001600002B05D02000290032007E
:100150003B00FFF7D1FFF8BD140C0010F0B5B82438
:10016000A44685B002920393154B164A9C440600A0
:10017000146855680F009068D1680090019161463D
:100180000C604D60009801991C00C03420606160D3
:100190001900D8318C68CD680868496810605160D2
:1001A0001A00D032146055601A00B033A8321660BD
:1001B00057600299039A19605A6005B0F0BDC046B5
:1001C000700B0010380C00100022044B1A70044A07
:1001D000137859424B4113707047C046F20B001020
:1001E000F10B00100022044B1A70044A1378594294
:1001F0004B4113707047C046F10B0010F20B00101A
:1002000070470023034AD356591E0B43DB0F13706C
:100210007047C046F40B00100122014B1A70704762
:10022000140C00100122014B1A707047140C0010BE
:10023000164BD0B5DA6F164B1100164C19401A4206
:100240000CD1154BA5341A68002A02DD2270196002
:10025000D0BD22781A6004232370F9E72300863387
:100260001B78002BF4D00C4B58680C4BE358A4348B
:10027000C01A0EF0EBFD0022094B0DF019FA002315
:100280000022FFF759FF0123E6E7C046780B001074
:1002900000FFFF00700B00105801001074070000F1
:1002A00000408F400022014B1A707047F00B001085
:1002B00070470022014B1A807047C046EE0B0010B9
:1002C0000122014B1A807047EE0B00108022024B76
:1002D00052001A807047C046EE0B0010034A137894
:1002E000DB431B06DB1713707047C046F40B00108E
:1002F00070B5FFF7E5FE03000020012B12D00A4B7A
:1003000000221C685D68094B200029000BF0EAFC04
:10031000002807D0064B0022200029000BF0F6FC35
:10032000431E984170BDC046180C00100000F03FFD
:100330000000F0BF0021054B054A11801A008632EB
:1003400011700122A4331A707047C046700B001060
:10035000EC0B00100122014B1A707047F00B0010DB
:10036000704783280ED80F290CD88422CB085B4213
:10037000134018180723194079330B41024A115CC6
:100380000B4313547047C0469402001030B5FA2452
:1003900001000023084AE4001578180001332B2DD2
:1003A00004D155788D4201D1023030BD0132A342D3
:1003B000F2D10020F9E7C0469C03001010B5682870
:1003C00002D8FFF7E3FF10BD0A4BFE280CD1E9224B
:1003D000D2009B18186859680EF0CEFC030040420A
:1003E000002BF0DBD8B2ECE70322873300201A7031
:1003F000E9E7C046700B0010502818D842280BD8E7
:1004000007280DD8052383428041404270470B489E
:10041000D84001231840F9E74338C3B20848F7E74A
:100420000D38C3B200201E2BF0D80648F0E76B3819
:10043000C3B2152BEBD90020E8E7C04611F93F0005
:100440003333000011000040F8B505000400074FE9
:10045000002C03DC0123281B1840F8BD661EB85D84
:10046000FFF7CAFF0028F5D03400F1E79C03001025
:100470007C221A491A4B8A5A9B5C502B24D8422B57
:100480000FD8072B26D90D3BDBB21E2B03D81548FE
:10049000D840C0070BD4144B9A4210D87C230132A9
:1004A0000AE0433B1148DBB2D840C007F3D5104BFC
:1004B0009A4204D87C2302320020CA527047872314
:1004C00003220120CA54F9E76B3BDBB2152BE2D8BB
:1004D0000848E9E7052BDED9E9E7C046700B0010B4
:1004E0009C03001011000040CE07000033330000D1
:1004F000CD07000011F93F007C23F0B5124A83B00C
:100500000092D75A012F17D9104EBB1E0025019318
:10051000F41804E0631E0135A64205D01C002078C3
:10052000FFF76AFF0028F5D1ED0707D57C23009A75
:100530000199D15203B0F0BD002FFBD07C23009A6B
:10054000013FD752F6E7C046700B00109C03001025
:1005500070B50A4D04B223B2002B01DC084809E053
:100560002B5D66192B2B06D12000FFF76DFF0028AD
:1005700001D1707870BD013CEDE7C0469C030010CE
:10058000FFFFFF7F70B5FA250124084EED00305DB6
:10059000002809D0FFF730FF431E98410019441C82
:1005A000AC42F4DBFA24E400200070BD9C03001090
:1005B00010B5054C2388002B02D0FFF79DFF10BD1E
:1005C000FFF7E0FF2080FAE7EC0B0010F8B504001D
:1005D0000D00FFF7D7FF144B1B1AAB4203DA0322BF
:1005E000124B1A70F8BDFA22D2009442FADA2E1990
:1005F000F8D40F4B012D09D100221B18A042F1DBCA
:100600001978013859701A70013BF7E7002108008A
:10061000121B1B191F781D1B0131AF5518700133B8
:100620009142F7D1DEE7C046CF070000F70B00107C
:100630009C030010F7B5114B01911B88104C07006B
:10064000E25C104D002A01D1002B01D1FFF710FF11
:100650007C3528880121FFF7B9FF2E883800A7557F
:10066000FFF7CAFE002807D00121701CFFF7AEFF7C
:100670002B88E418019B6370F7BDC046EC0B00109B
:100680009C030010700B001010B5064B064C1B7835
:10069000002B03D00B217620FFF7CCFF0123A434DD
:1006A000237010BDF50B0010700B001010B5064B39
:1006B000064C1B78002B03D00C217620FFF7BAFFE5
:1006C0000123A434237010BDF50B0010700B001033
:1006D00010B50A4A0A4B1278002A0BD17F331B78D7
:1006E0000022002B07D0074B0DF024FC064A074BD5
:1006F0000CF0DEFF10BD064BF6E7C046EE0B001017
:10070000700B001000007940182D4454FB21194053
:1007100000807640F0B53F4A4B005B0D85B09A18DB
:1007200006000F000C00050003900192132A32DC32
:10073000002A14DA384A394B0CF0A0FB00220023BF
:100740000BF0DAFA002807D0002F5CDA7C0064088E
:1007500025435BD18024240627002E0028E0304B5F
:10076000019A134102930B40034321D02A4A2B4B99
:100770000CF084FB002200230BF0BEFA0028EBD023
:10078000002F04DA8024019B64031C41E419029BBE
:1007900000259C43E0E7019A332A0DDD8023DB002E
:1007A0009A4205D102000B000CF068FB06000F0016
:1007B0003000390005B0F0BD1A4A9B1801225242A0
:1007C000DA4002920242F3D0134A144B0CF056FB6B
:1007D000002200230BF090FA0028BDD0002F03DA8E
:1007E000019B142B03D10134029B9D43B4E73422B7
:1007F000019BD21A01239340F518039B9D429B4114
:100800005B42FC18F0E700252C00A5E70025064C0C
:10081000A2E7C04601FCFFFF9C7500883CE4377EE0
:10082000FFFF0F00EDFBFFFF0000F0BF70B50022DF
:10083000002304000D000BF04BFA002807D080269F
:1008400036062000A919FFF765FF891970BD200041
:100850002900FFF75FFFF9E74B0070B55B0D14004F
:100860000D00002B0DD14B005B08034310D0234B30
:1008700000220DF05FFB224B9C420ADA214A224BF8
:1008800018E0224A934208D102000B000CF0F6FA5D
:1008900070BD0D004B005B0D363B1D4A94420CDDD4
:1008A0001C48C90FC907084303001B4A1900100060
:1008B000184B194A0DF03EFBEAE7E218174B9A4233
:1008C000EEDC002A05DD164B12052B401343190000
:1008D000DEE71300353308DA0B48C90FC9070843B0
:1008E0000300084A19001000C8E70D4B36321D40BE
:1008F00012052A4311000B4B0022DBE70000504396
:10090000B03CFFFF59F3F8C21F6EA501FF070000BE
:1009100050C300003CE4377E9C750088FE07000051
:10092000FFFF0F800000903CF0B587B00492059364
:100930004B005B080193F923019A04000D009B050D
:100940009A4204D20EF018FA002800D184E0220066
:100950002B00200029000DF0EDFA0022404B06008C
:100960000F000DF0E7FA3F4A029003913E4B300032
:1009700039000DF0DFFA3D4A3D4B0CF07FFA3200B2
:100980003B000DF0D7FA3B4A3B4B0DF09BFD32008C
:100990003B000DF0CFFA394A394B0CF06FFA3200B8
:1009A0003B000DF0C7FA374A374B0DF08BFD320094
:1009B0003B000DF0BFFA354A354B0CF05FFA3200C0
:1009C0003B000DF0B7FA32003B000DF0B3FA049A89
:1009D000059B06000F00200029000DF0ABFA020075
:1009E0000B00300039000DF06DFD2A4B019A049088
:1009F00005919A420DD802000B00029803990DF060
:100A000061FD020000200B0023490DF05BFD07B0E3
:100A1000F0BD224B019A00269A421BD81300204AAF
:100A2000944663441F0032003B0000201A490DF039
:100A300049FD320004000D00029803993B000DF0BF
:100A400041FD049A059B0DF03DFD02000B002000C6
:100A50002900DAE7134FE6E700200F49D7E7C04641
:100A60000000E03FD43888BEE9FAA8BDC4B1B4BDE7
:100A70009EEE213EAD529C804F7E923E9015CB194A
:100A8000A001FA3E7751C1166CC1563F4C555555E1
:100A90005555A53F3233D33F0000F03F0000E93FFA
:100AA0000000E0FF0000D23FF8B50022324B0DF00D
:100AB00041FA0022002306000F000BF003F9002882
:100AC00054D10022300039002C4B0BF0FBF80028E9
:100AD0004FD132003B00300039000DF02BFA0400FA
:100AE0000D00274A274B0DF025FA274A274B0DF01A
:100AF000E9FC22002B000DF01DFA254A254B0CF0D5
:100B0000BDF922002B000DF015FA234A234B0DF0FE
:100B1000D9FC22002B000DF00DFA214A214B0CF0DC
:100B2000ADF922002B000DF005FA1F4A1F4B0DF006
:100B3000C9FC22002B000DF0FDF91D4A1D4B0CF0E5
:100B40009DF922002B000DF0F5F91B4A1B4B0DF00F
:100B5000B9FC22002B000DF0EDF9194A194B0CF0ED
:100B60008DF932003B000DF0E5F9F8BD00200021C1
:100B7000FBE700201449F8E70000E03F0000D03F09
:100B800098456D69B8D1B93F722CC67097F7E63FAA
:100B9000A79ED5E9358F0E400CD7D1DD74302E409D
:100BA000CB90514883074540437562CE2C2D53406E
:100BB0006EAA7567BC66544052BE25E6BCAB444085
:100BC000182D4454FB2119400000F03FF0B589B0C6
:100BD00002920393F9224B0006000F005B08920576
:100BE000934203D20EF0C8F800284CD032003B00EC
:100BF000300039000DF09EF904000D0002000B00DA
:100C0000300039000DF096F9394A00900191394BC6
:100C1000200029000DF08EF9374A384B0DF052FCB8
:100C200022002B000DF086F9354A364B0CF026F9E0
:100C300022002B000DF07EF9334A344B0DF042FCBC
:100C400022002B000DF076F9314B324A0CF016F9E8
:100C50000E9B04900591002B19D102000B0020007F
:100C600029000DF067F92C4A2C4B0DF02BFC009A53
:100C7000019B0DF05FF902000B00300039000CF011
:100C8000FDF806000F003000390009B0F0BD002269
:100C900002980399224B0DF04DF9049A059B06909A
:100CA0000791009801990DF045F902000B00069894
:100CB00007990DF007FC22002B000DF03BF9029A7A
:100CC000039B0DF0FFFB144A04000D0000980199EE
:100CD000124B0DF02FF902000B00200029000CF040
:100CE000CDF802000B00300039000DF0EBFBC8E737
:100CF0007CD5CF5A3AD9E53DEB9C2B8AE6E55A3EA6
:100D00007DFEB157E31DC73ED561C119A0012A3F41
:100D10001111813FA6F81011495555555555C53F3C
:100D20000000E03FF0B50A000D0055490400030043
:100D3000080085B02840884211D122002B002000F5
:100D400029000DF0F7F802000B00200029000CF03C
:100D500095F804000D002000290005B0F0BD002D1D
:100D600011DC690049082143F5D00020854210D0EC
:100D700022002B00200029000DF0A4FB02000B0034
:100D80000CF096FCE5E7281515D1802400216403BA
:100D900007E0DA0A15385B05002AFAD0F5E75200B9
:100DA00001312242FBD04C1E001B20241D00641A7E
:100DB000E5408B402A433349120344188021120B2B
:100DC00049031143C00703D4DA0F490051185B00EF
:100DD0006210002449000392DA0F52188021162570
:100DE00020005B0089034618964202DC7018921BB3
:100DF0006418DE0F5200013DB2185B004908002D57
:100E0000F1D120268027290001963F067E19B4469D
:100E1000824202DC14D19E4212D865466646ED1924
:100E20000290002E03DAEE43F60F86190296121A8C
:100E3000634580414042121A60461B1A0298C91944
:100E4000DE0F5200B218019E5B00013E7F08019642
:100E5000002EDBD11A4303D04B1C0CD131000134DE
:100E6000094B6010C018039BE4071D052B184908A7
:100E70001D000C436FE7012301319943F0E7C046A1
:100E80000000F07F01FCFFFF0000E03F434203430E
:100E900001204A005208DB0F13430449044A9A1800
:100EA000CB1A1343DB0F58407047C0460000F07F59
:100EB00000001080F7B514001D0000900191002281
:100EC000200029001A4B0AF003FF002801D000245B
:100ED000174D260000242F00154D3000009A019B6D
:100EE00039000AF0FFFE002803D12000290003B0DA
:100EF000F0BD32003B00200029000DF01BF804007B
:100F00000D00FFF7C3FF634223436A005208DB0F63
:100F10001343084AD31ADB0F0343E6D130003900EC
:100F20000022034B0BF0AAFF06000F00D5E7C046D6
:100F30000000F03F0000F07FF0B504000D00354EDA
:100F400085B0634223436A005208DB0F1343F31A50
:100F5000DA0F0392002B59DB20002900FFF796FFE0
:100F60000290002854D100220023200029000AF01A
:100F7000A9FE00283CD100220023200029000AF00D
:100F8000A7FE002807D080231B06EB1800940193CE
:100F9000009C019DD5E70022200029001E4B0AF08D
:100FA000B5FE002815D000261C4F22002B00300073
:100FB00039000AF0A1FE00281AD130003900174B81
:100FC00000220CF0B7FF029B060001330F000293D2
:100FD000EBE70123124E134F029322002B00300047
:100FE00039000AF07FFE002805D0029B5B42029385
:100FF000029805B0F0BD30003900084B00220CF01B
:1010000057FB029B06000F000133E5E70023EEE7E4
:10101000039BECE70000F07F0000F03F000024405D
:101020009A9999999999B93FF8B504000D00FFF77D
:101030002DFF002800D005E1002200232000290018
:101040000AF046FE00280BD0802636062000A9199B
:10105000FFF7EAFF8919002200230BF00FFFF8BD0C
:1010600000220023200029000AF02CFE002802D0D4
:1010700000200021EFE7002220002900744B0AF035
:1010800021FE002800D0E0E0002220002900714B62
:101090000AF018FE0028EBD16F4B69002F004908B9
:1010A000994219D922002B00200029000BF0E6FEFE
:1010B00002000B000CF0FCFA04000D0000222000DE
:1010C0002900634B0AF00EFE002800D188E02000C2
:1010D0002900FFF7E9FCBEE78023E80F2600220085
:1010E000C007DB05994208D8E8D1002C05D15B4B3D
:1010F000000F1B181C685D68E0E7594B1F4217D1B1
:10110000584BCD021C00002D0FDCA34213D0E41A73
:101110001F2C32DC35000A005349A2405918CD403B
:10112000290011433200A2400AE0013B6D00EAE7CA
:101130004E4B0915CB1880213F033F0B4903394320
:101140005C1E4B4BCB18002C1DD180256D03A94292
:1011500000DA0B001C0001211443C8D0AB421EDB97
:10116000404CA14221DB424C1B1903434148091862
:1011700009050B431D001400A0E731003E4AD21AB6
:1011800091400022DCE74900002B03DB19001143EA
:10119000ADD05900D30FC9185200013CD1E7D40F8C
:1011A0005B001B1952000139D8E7641A142C09DCC2
:1011B0002D4DE24049191D008D4023412A4318431B
:1011C0000500D8E71F2C06DCE240274C09198B40AC
:1011D0001A430300F3E7284A521A13411A00F8E7AA
:1011E0000022200029001B4B0AF07CFD002806D0BD
:1011F00022002B00002017490DF064F969E7002256
:10120000200029001D4B0AF06DFD002200280AD0A5
:10121000200029000F4B0DF055F9FFF745FC802306
:101220001B06C91817E7802320002900DB050AF0F8
:1012300059FD002800D11BE7802122002B0000204F
:10124000C905E8E700200E4905E70020014902E74B
:101250000000E03F0000F03FFFFFEF7F80F2000062
:101260000000F07F02FCFFFF1E04000001FCFFFFF6
:101270000000F0FFFF030000E2FBFFFF0000F83F6B
:101280000000F87F8023F0B55B030E008DB099421B
:1012900023DA4B005B08034307D100220023002020
:1012A000B4490CF005FA0DB0F0BD002906DA0200D1
:1012B0000B000DF007F900220023F2E7AE4B0022ED
:1012C0000CF038FE36230E005B42AC4A964206DD37
:1012D00002000B000BF0D2FDE5E70023F5E7A84C78
:1012E000321512193603A74CD218330B02931B196F
:1012F000802464032340A44C029D5C401B159B1872
:1013000025430022009329009F4B0DF0DBF8029B40
:10131000060002331B030F0000221B0B022B64DCB0
:1013200000230AF0CFFC002819D0009B002B00D12D
:101330001CE118000DF05CFD944A954B04000D0073
:101340000CF0F8FD934A06000F00934B2000290093
:101350000CF0F0FD02000B0030003900BAE78F4AB4
:101360008F4B300039000CF0E5FD02000B0000202F
:101370008C490DF0A7F8320004000D003B0030004E
:1013800039000CF0D7FD0B000200290020000CF002
:10139000D1FD009B02900391002B06D102000B00AF
:1013A000300039000DF08EF87DE700980DF020FD3B
:1013B000764A774B04000D000CF0BCFD754A009096
:1013C0000191754B200029000CF0B4FD02000B00C8
:1013D000029803990DF076F832003B000DF072F898
:1013E00002000B0000980199DCE78023DB050BF07D
:1013F00045FD02000B00300039000CF059F9049053
:10140000059100980DF0F4FC049A059B0690079155
:10141000100019000CF08EFD634A029B9446634451
:1014200002000B930B00089009910CF083FD04005F
:101430000D005E4A5E4B0CF07DFD5E4A5E4B0BF08C
:101440001DFD22002B000CF075FD5C4A5C4B0BF07F
:1014500015FD22002B000CF06DFD5A4A5A4B0BF083
:101460000DFD089A099B0CF065FD584A08900991FA
:10147000574B200029000CF05DFD564A564B0BF0EF
:10148000FDFC22002B000CF055FD544A544B0BF090
:10149000F5FC22002B000CF04DFD02000B0008981B
:1014A00009990BF0EBFC029A4E4B04009B1A0B9A25
:1014B0000D001343002B34DD00223A4B300039007D
:1014C0000CF038FD32003B000CF034FD02000B0044
:1014D00002900391200029000BF0D0FC049A059B98
:1014E0000CF028FD009B04000D00002B06D102002B
:1014F0000B00029803990CF0E5FF4FE7234A244BB9
:10150000069807990CF016FD224A00900191069862
:101510000799214B0CF00EFD22002B000BF0AEFCC6
:1015200054E702000B00300039000CF0CBFF049AA6
:10153000059B0CF0FFFC009B04000D00002B02D16A
:1015400002000B002CE7114A114B069807990CF08A
:10155000F1FC104A00900191069807990E4B0CF08F
:10156000E9FC02000B002000290033E700200021E5
:1015700099E6C046000050C300005043FFFFEF7FD4
:1015800001FCFFFF645F09000000F03F0000E0FE87
:10159000422EE63F763C7935EF39EA3D55555555B3
:1015A0005555D53F0000E03F86EBF9FF44523EDF42
:1015B00012F1C23FDE03CB966446C73F5993229493
:1015C0002449D23F935555555555E53F9FC678D090
:1015D000099AC33FAF788E1DC571CC3F04FA979925
:1015E0009999D93F51B8060007B5002200280CD1BF
:1015F000E023DB050092019300980199E02300228B
:10160000DB050CF097FC03B000BDF0231B06F1E7EF
:1016100007B5002200280CD180235B0500920193BE
:1016200000980199802300225B050CF083FC03B035
:1016300000BD90231B06F1E7F0B5904A4B00060071
:101640000F0089B0CC0F5B0893422CD98C4A93428F
:1016500011D90B031B0B034306D002000B00300013
:1016600039000BF00BFC0FE0002C00D003E1300040
:10167000390009B0F0BD834A834B0AF03DFB051EDB
:1016800005D00020FFF7B0FF06000F00EFE73000A5
:1016900039007E4A7E4B0AF01BFB00287AD02800D6
:1016A000FFF7B6FFF0E77B4A934200D89BE07A4A07
:1016B00093426FD8794DE300ED182A696B690CF0FD
:1016C00001FF2A6A6B6A0492059301230290039139
:1016D00063401B1B0193049A059B029803990CF02D
:1016E000F1FE06000F0032003B00300039000CF024
:1016F00021FC04000D006A4A6A4B0CF01BFC6A4A8C
:101700006A4B0CF0DFFE22002B000CF013FC684A41
:10171000684B0BF0B3FB22002B000CF00BFC664A6D
:10172000664B0CF0CFFE22002B000CF003FC644A49
:10173000644B0BF0A3FB22002B000CF0FBFB020020
:101740000B00300039000CF0BDFE0B00020004005D
:101750000D00300039000CF0EDFB019B0690079165
:10176000002B55D18023002220002900DB050CF03E
:10177000A9FE02000B00069807990BF099FF3200B2
:101780003B000CF09FFE02000B0000204E490CF0C5
:1017900099FE79E7414BE4001C194C4A4C4B300050
:1017A00039000CF0C7FB226B636B0BF067FB0DF08D
:1017B000E3FA01900DF01CFB464A474B04000D0074
:1017C0000CF0B8FB02000B00300039000CF07AFE80
:1017D000424A02900391424B200029000CF0AAFBE0
:1017E0000490059177E73F4A93420CD83E4A3F4B1D
:1017F0000BF044FB0022344B0AF07EFA002805D09F
:101800000022314B2BE7002301936CE701906AE73C
:1018100080212B0022000020C9050CF053FE02009D
:101820000B00069807990BF043FF02000B00049889
:1018300005990CF047FE029A039B0CF043FE020050
:101840000B00002020490CF03DFE294B019A0D00B1
:101850009A4203DB110506004F1908E7FA229200AD
:101860009446019B002263441B055918B8235B046E
:101870000CF060FB08E700260027F8E6412E8640C2
:10188000FFFFEF7FEF39FAFE422E864051302DD513
:10189000104987C0422ED63FB1A2F03F80F200002F
:1018A000D0A4BE726937663EF16BD2C541BDBB3E66
:1018B0002CDE25AF6A56113F93BDBE166CC1663F44
:1018C0003E5555555555C53F0000F03FFE822B65EE
:1018D0004715F73F0000E0FE422EE63F763C7935A3
:1018E000EF39EA3DFFFFEF3D9C7500883CE4377E11
:1018F00003FCFFFF70B51E4A4D006D0DAA180B00CA
:10190000132A18DC002A0ADAC90FC9070B000132B2
:1019100001D1184B0B4300221900100015E0164CA2
:10192000144123000B4003430FD080231B031341BA
:101930005B18A343EFE7332A08DD8023DB009A42DC
:1019400003D102000B000BF099FA70BD0B4EAE19DB
:1019500001256D42F5402842F7D03321891A012232
:101960008A4012188242A44164421B19AA43D3E759
:1019700001FCFFFF0000F03FFFFF0F00EDFBFFFF4A
:10198000F8B50D0017001E0004000DF0F5F93860E1
:101990000DF02EFA02000B00200029000CF092FD41
:1019A0000022104B0CF0C6FA04000D00FFF7A2FF56
:1019B0000DF0E2F930600DF01BFA02000B00200080
:1019C00029000CF07FFD0022074B0CF0B3FAFFF763
:1019D00091FF0DF0D1F9002800D10130069B18606D
:1019E000F8BDC04600408F4000005940F0B54F00A0
:1019F0007C088BB0260000945C006408A446270095
:101A0000A64207DBB44637000094260014001900F4
:101A1000020020000290039100996346039102980E
:101A2000039900900191F02014001D00B91B80045F
:101A3000814208DD009A019B200029000BF01EFA6C
:101A400004000D0018E07D498F4200DC9BE07C49DA
:101A50008F4215DD3B031B0B134307D0009A019BFC
:101A6000200029000BF00AFA04000D00754B009AC3
:101A70007340134300D1DEE0200029000BB0F0BD1D
:101A80007149029A039B761833007F1800920193E4
:101A900096233D009B0002936C4B9E421BDC8023EF
:101AA0005B039E4271DA009B3343E5D000980199B5
:101AB0000022674B0CF03EFA002200900191644B2B
:101AC000200029000CF036FA624A040094460D000A
:101AD000029B63440293009A019B200029000CF0B2
:101AE000F1FC02000B0004900591009801990AF0A6
:101AF000EFF80022002858D03B00100039001600F3
:101B00000CF018FA8022009B049005911800019BAC
:101B100012069918009A019B0CF00CFA3200009002
:101B200001913B00200029000BF0A8F9320006903B
:101B300007913B00200029000CF0C4FC02000B00C0
:101B4000069807990CF0F6F902000B00009801992D
:101B50000CF0B8FC02000B00049805990CF0B2FCE4
:101B6000FFF7E0F8029B04000D00002B00D183E793
:101B70000020394A1B0599180B000200290020009B
:101B80000CF0D8F95CE7002385E79623334A9B05E0
:101B90009446FF18F618029B3D0063440293009A96
:101BA000019B33000092019395E733008021069258
:101BB0000793002249037B180698079916001F0017
:101BC0000CF0B8F98022049B089009911800059B3D
:101BD00012069918049A059B0CF0ACF922002B0010
:101BE00004900591200029000BF048F932003B00D9
:101BF0000CF068FC009A019B0CF09CF9069A079B7C
:101C000004000D00009801990CF05CFC32003B00D0
:101C10000CF090F902000B00200029000BF02EF9C7
:101C200002000B00049805990CF04CFC02000B001C
:101C30000898099992E7009C019D1DE70000305F1C
:101C4000FFFFEF7F0000F07F000080DAFFFFAF2092
:101C50000000D07F02FCFFFF0000F03FA8FDFFFF67
:101C6000F0B5CC4ACC0F4B0006000F0089B0E4075A
:101C70005B0893423CD9C84A93421FD9C74A934252
:101C80000DD90B031B0B034304D002000B000BF018
:101C9000F5F80DE0002C0DD00026C14F0AE0C14A36
:101CA000C14B0AF029F8002808D00020FFF79CFC5F
:101CB00006000F003000390009B0F0BD002C00D143
:101CC000BDE0BA4ABA4B300039000BF0D7F8002219
:101CD000002309F0FDFF0028DED1B64AB64B3000E4
:101CE00039000CF027F902000B000020B349B0E0E6
:101CF000B34A934200D8D4E0B24A934200D9C6E036
:101D0000B14AB24B002C00D08FE00CF0DBFB01237A
:101D100004000D000093AE4AAE4B02920393029A68
:101D2000039B200029000CF0CDFB02000B000600F5
:101D30000F00200029000CF0C5FB029A039B0CF059
:101D4000C1FB029003910022A34B300039000CF03C
:101D5000F1F802000B0004900591300039000CF0FE
:101D6000E9F804000D009D4A9D4B0CF0E3F89D4AF4
:101D70009D4B0BF083F822002B000CF0DBF89B4A04
:101D80009B4B0CF09FFB22002B000CF0D3F8994AE0
:101D9000994B0BF073F822002B000CF0CBF8974A0C
:101DA000974B0CF08FFB22002B000CF0C3F80022A5
:101DB000944B0BF063F802000B0006900791049817
:101DC00005990CF0B7F802000B0000208E490CF0CA
:101DD00079FB02000B0004900591069807990CF01E
:101DE00071FB049A059B06900791300039000CF0B6
:101DF000A1F802000B00002084490CF063FB0200F4
:101E00000B00069807990BF053FC2B0022000CF0F6
:101E100091F8009B002B5AD102000B0030003900D2
:101E20000CF088F822002B0048E00BF027F8012383
:101E30005B42009304000D00654A754B6DE75D4AF7
:101E40005D4B300039000CF075F802000B000020EB
:101E500061490BF013F80CF08FFF00900CF0C8FFF5
:101E6000594A5A4B029003910CF064F802000B009F
:101E7000300039000CF026FB554A04000D00029892
:101E80000399544B0CF056F80290039147E7494AE6
:101E9000494B0CF04FF802000B00002C00D024E757
:101EA000D5E700215B4A0091934200D94BE75A4A9B
:101EB0005A4B39000AF0E2FF02000B000CF002FB63
:101EC00002000B00300039000CF0FCFAF0E6029A38
:101ED000039B0CF0F7FA32003B000CF02BF8029A4F
:101EE000039B0CF0EFFA2B0022000CF0EBFA009BA6
:101EF00004000D0001330CD102000B00300039004A
:101F00000CF0E0FA0022344B0CF014F80022324BB3
:101F1000DAE7009B012B26D1002230003900404B2C
:101F200009F0D6FE002811D00022300039002A4BDB
:101F30000AF0A4FF02000B00200029000CF0C2FAF6
:101F4000C02300221B060BF0F5FFB1E622002B0098
:101F5000300039000CF0B6FA02000B000AF08EFFD8
:101F60000022284B93E6009B1B050293009B013344
:101F7000392B57D932003B000CF0A4FA02000B00B9
:101F8000002020490CF09EFA029C002263181900E0
:101F90001C4B99E779684340412E8640FFFFEF7F55
:101FA0000000F0BFEF39FAFE422E864059F3F8C226
:101FB0001F6EA501FE822B654715F73F0000E0BFAD
:101FC000422ED63FB1A2F03F0000E0FE422EE63F97
:101FD000763C7935EF39EA3D0000E03F2DC3096ECC
:101FE000B7FD8ABE3952E686CACFD03EB7DBAA9E7D
:101FF00019CE143F8555FE19A0015A3FF410111156
:102000001111A13F0000F03F0000084000001840FF
:10201000EF39EABDFFFF8F3C9C7500883CE4377EBA
:102020000000D0BF009B132B18DC8023009A9B0379
:1020300013410020134AD11A0090019132003B0055
:10204000200029000CF03EFA02000B0000980199D4
:102050000CF038FA029B06005F182BE600980A493C
:102060000022091A0B05200029000AF007FF0200D0
:102070000B00300039000CF025FA0022014B0AF069
:10208000FDFEE7E70000F03FFF0300004023044AA5
:1020900011680B4313600122024B1A727047C0464D
:1020A00080800440580100100E4B70B51B7A04006C
:1020B0000E001500002B01D1FFF7E8FF631E022B75
:1020C0000AD8094B2004C01801230268B340012D2F
:1020D00004D11343036070BD0348F5E79A430260DF
:1020E000F9E7C04658010010008000500E4B70B553
:1020F0001B7A04000E001500002B01D1FFF7C6FF6C
:10210000631E022B0AD8094B2004C0180123026861
:10211000B340012D04D11343036070BD0348F5E7BC
:102120009A430260F9E7C04658010010FC3F005096
:10213000012270B5082106001000FFF7D7FF072421
:10214000002208210120FFF7D1FF320001252241A2
:10215000022100202A40FFF7C9FF2A000821280099
:10216000FFF7C4FF013CEBD270BD002210B50400A4
:1021700011000220FFF7BAFF2000FFF7D9FF10BDC2
:1021800070B50D0004000122FFF78EFF2900012227
:102190002000FFF7ABFF70BD012210B510000B212E
:1021A000FFF782FF00220B210120FFF79FFF012292
:1021B00002210320FFF778FF002202210320FFF70E
:1021C00095FF10BD084B70B51B7A04000D00002B65
:1021D00001D1FFF75BFF1822236893432360236834
:1021E0001D43256070BDC0465801001070B5050044
:1021F0000024054EA05D054B2900C0180134FFF7EF
:10220000E1FF0A2CF6D170BDC0F20000004004408E
:10221000F8B500251020FFF7E9FF0A4C267867780B
:10222000002239003000FFF73FFF0135012239005D
:102230003000FFF75BFF02340A2DEFD10122024B81
:10224000DA60F8BDCAF2000058010010F8B51A4E65
:102250000400F368002B01D1FFF7DAFF002C09D04E
:10226000012207210220FFF71FFF00220721022081
:10227000FFF73CFF337A002B01D1FFF707FF0F4F29
:1022800001253B681B0509D5337A002B01D1FFF7E7
:10229000FDFE01253B681B05DB0F5D40002C09D0CE
:1022A000002207210220FFF7FFFE01220721022062
:1022B000FFF71CFF2800F8BD58010010FC3F00503C
:1022C000F0B5012087B0FFF7C1FF01230493002878
:1022D00044D10124274B049003932700039B012240
:1022E0001B780193039B01985B7819000293FFF719
:1022F000DBFE002202990198FFF7F8FE1E4DAB7934
:10230000EE7905931D4B1B7A002B01D1FFF7BEFE22
:10231000059B032B2BD8180009F0D0FB022325279F
:10232000174B0122B2401B6813405A1E9341002BE9
:102330001DD00137231D023D9F42E0D100220299AA
:102340000198FFF7B1FE012202990198FFF7CEFE36
:10235000039B3C0002330393292FBED1049807B09E
:10236000F0BD084BDDE7084BDBE7084BD9E7FBB2D4
:102370000493DEE7CAF20000DEF20000580100100C
:10238000FC3F0050FC3F0150FC3F0250FC3F03501B
:10239000064B5A68013202D11A6901321A615A6831
:1023A00001325A605A6901325A617047580100106F
:1023B000C143094A5368994209D2591C0918506807
:1023C000984200D2704750688142FCD8F7E75168C4
:1023D000C91A8142FBD3F5E7580100100122034BD3
:1023E0001A60034A936901339361704700C000404B
:1023F000580100100122034B1A60034AD3690133CC
:10240000D361704700000140580100100122034BC6
:102410001A60034A136A0133136270470040014097
:10242000580100100122034B1A60034A536A01331A
:10243000536270470080014058010010064A537BE8
:10244000D318D873537B0133DBB253735BB2002BC9
:1024500001DA00235373704704020010194B10B5C2
:1024600018680E23184002380A2811D809F026FBF4
:102470002010131006101010101019009E22124B7D
:102480001B68134205D0114ADBB25360104B1B6826
:1024900010BDDB07FCD50E4B1868C0B2FFF7CEFFAE
:1024A000F6E78023094A5B0051680B435360EFE76E
:1024B000054B1A68054B920602D500229A60E7E7A1
:1024C0000122FBE708800040148000400402001055
:1024D00000800040F8B5551E0C001E0011000700DA
:1024E0002B000200092E16D90A21300009F022FA29
:1024F000210003002A003800FFF7ECFF04003F181A
:1025000030000A2109F09CFA30313970601CF8BDA6
:102510001470013B0132002BFADC0C1E00DC01249C
:10252000CA17521AD2171540013C7F19E8E7F0B5D7
:1025300085B00B9B05000C000A9E0393571E002BD1
:1025400001D1092E28D90A2200230399300009F06D
:10255000E7FB3A000090019121002800FFF7E7FF18
:1025600004002F18300003990A22002309F0D8FB39
:10257000601C30323A7005B0F0BD0C70013B013187
:10258000002BFADC141E00DC0124D3179A1AD21790
:102590001740013CEF19E5E73B000100F0E7F7B514
:1025A0001D00DB170F00E918594004000B000191D2
:1025B000561E092916DD18000A2109F0BBF903008F
:1025C000002D00DA4342320020003900FFF7E7FF18
:1025D0000600241801980A2109F032FA3031701CE3
:1025E0002170FEBD002D00DA961E2300A119CA1A23
:1025F000002A0ADCF043C0170640A419002DE9DACE
:102600002D23013623700134E4E71F700133EEE718
:10261000F7B51E00089B1700013A1D0904001300BE
:10262000002D12D033000095FFF7F2FF24180F237E
:10263000089D1D40EAB21300092D12D83033013035
:102640002370FEBD0170013B0130002BFADC381E07
:1026500000DC0120FB17DB1BDB1713400138E418FB
:10266000E5E75733002EEAD0203BE8E703000020DF
:102670001A5C002A00D170470130F9E7F8B51D4C0B
:1026800000252000FFF7F2FFC3B2A3755A1E934145
:1026900023762378C0B22D3B5A4253418446A37619
:1026A00029002A002B000120134EE5756576E5769A
:1026B0009C450ADC002902D0330028335D76002ACD
:1026C00002D001232836F375F8BD277801332E2F69
:1026D0000ED0452F05D162782D2A04D001210A00A1
:1026E000DDB20134E4E7320001212832D176F5E78A
:1026F0000200F6E780010010580100107FB51A4B68
:102700001A4A1B7E12780600194D1A4C134318D131
:10271000194B996EDA6E009101921A6F5B6F0098F7
:10272000019902920393029A039BFDF705FD210094
:1027300000220023A8310A604B602100B0310A60FA
:102740004B602B0078342833997DDA7D20788A1A03
:10275000824204DB5B7E002B01D1452E01D128355E
:102760006E54FFF78BFF7FBD800100100C0C001032
:1027700058010010700B001080F2000010B53020DE
:10278000FFF7BCFF10BD10B53120FFF7B7FF10BD3C
:1027900010B53220FFF7B2FF10BD10B53320FFF7A0
:1027A000ADFF10BD10B53420FFF7A8FF10BD10B568
:1027B0003520FFF7A3FF10BD10B53620FFF79EFFB1
:1027C00010BD10B53720FFF799FF10BD10B53820A8
:1027D000FFF794FF10BD10B53920FFF78FFF10BD34
:1027E00010B5074BDA7D002A08D11B78002B02D1E7
:1027F0003020FFF783FF2E20FFF780FF10BDC0467B
:102800008001001010B50A4B0A4C1B7E002B05D12D
:102810003120FFF773FF0122074B1A702834637EC3
:10282000002B04D14520FFF769FFA37D637610BD1F
:102830008001001058010010140C00104E4B10B510
:102840005A6C4E4901325A644D4A1268D2B2302A4B
:1028500064D019D8182A0ED005D8082A35D0102AE5
:1028600043D008234CE0202A67D0282AF9D1986C5D
:102870005A6E904246D29A6C501C98644C339B5CC2
:10288000404ADBB21360ECE7482A56D009D8382A10
:102890004CD0402AE5D19A6E0423012A4AD10B601C
:1028A000DFE7502A52D0582ADBD1364A1268186E18
:1028B000D2B2441C1C661C006C3422540222FF322B
:1028C000DA658023F13ADB0551E000229A649A6CC4
:1028D000501C986418004C30825C2A48D2B20260C6
:1028E00028220A60273ADA6510BD00221A669A6C1F
:1028F000501C98644C339B5C224ADBB21360282343
:102900000B60F1E78022986ED205002801D02023C9
:10291000B8E70220FF30D8651023B3E780221020EB
:10292000D205106008220A60FA32DCE782225200E7
:10293000DA6596E78022D205A4E780221020D2052E
:10294000106008220A600422FF32CCE70D4A1268A8
:10295000186ED2B2441C1C661C006C3422549A6E51
:10296000186E531E0422834203D98023DB051A60AC
:1029700077E70A6075E7C04658010010180000406C
:102980000400004008000040FEE7FEE7F0B5D84C28
:102990005E1EA54408900A91D01E182114000793CA
:1029A00009F096F81823421C5B4253431B1900930D
:1029B000079B841B04330693CE4FE31802900493C5
:1029C00020AD002C00DAB3E0A300F8580CF010FAA8
:1029D000049B013403C59C42F3D13400079B089A41
:1029E000DB00D318099370AF20ABE5000022ED188F
:1029F000002304920593089E2A686B6803CE0BF0AF
:102A000099FA0B000200049805990AF037FA099B1D
:102A100004900591083D9E42EED10B0002000CC7C8
:102A2000069B0134A342DFD10427029BB14A9B00DD
:102A30009B180B933C00FB0070AAD3181D685E68BE
:102A40000CAB06930293002C75DC28003100009A31
:102A5000FDF702FFFF2300229B0504000D000BF091
:102A600069FAFDF757FE0022A34B0BF063FA020050
:102A70000B00200029000BF025FD0D0004000CF0D8
:102A80007BF904900CF0B4F90B000200290020003F
:102A90000BF018FD009B05000E00002B73DD1824C1
:102AA0007B1E9B000CA81A5800999C46641A1100C2
:102AB0002141049B5B18A14004936346521A1A50AB
:102AC000172300995B1A1A410292029B002B6BDDBF
:102AD0000022049B140001330493884B01209C4680
:102AE0000699974200DD9CE0009B002B05DD012B41
:102AF00000D1A6E0022B00D1ABE0029B022B53D108
:102B00002A00330000207E490BF0DCFC05000E009B
:102B1000002C49D0009A00207949FDF79DFE020063
:102B20000B00280031000BF0CDFC05000E003BE04F
:102B3000002000214CE70022724B280031000BF0EE
:102B4000F9F90CF019F90CF053F900226E4B0490CE
:102B500005910BF0EFF902000B00280031000BF09B
:102B6000B1FC0CF009F9029B013C01C3029370AA6D
:102B7000E300D3181A685B68049805990AF07EF997
:102B800005000E005FE7009B002B06D17B1E9B001B
:102B90000CAA9B58DB15029397E700225B4B09F0C8
:102BA000B5F800283AD10290002200232800310015
:102BB00009F088F8002800D1ACE000227B1E0CA9A7
:102BC000032B4DDC002A64D0009B013F183B00938F
:102BD0000CAABB009B58002B00D184E00020009A77
:102BE0004749FDF739FE3E0004000D00002E00DBD2
:102BF000C8E03D00464B0893002D00DA32E1089B07
:102C000070AA78331C00EB009B1807930022002366
:102C1000009201937B1B00260693DEE002230293C1
:102C200056E70B68002C0AD1002B04D080246404E2
:102C3000E31A0B6003001C000132043151E76446C3
:102C4000F6E77B1E0CA99B005A585202520A5A50B2
:102C500053E77B1E0CA99B005A589202920AF6E792
:102C600098004058013B0243AAE70133069A043A10
:102C700006921269002AF8D0079AFB18BC18E400E3
:102C800020AA7D1CA4180493049B9D4203DD1F0011
:102C9000D0E60123EAE70B9AAB00D0580CF0A8F875
:102CA0000022002327002060616002920393089EA7
:102CB0003A687B6803CE0BF03DF90B0002000298E6
:102CC00003990AF0DBF8099B02900391083F9E42AA
:102CD000EED1EB0070AAD3180A000100013519608B
:102CE0005A600834D0E7009B013F183B009370E71F
:102CF0009CFDFFFF1CF7000000002040FFFFFF00CD
:102D00000000F03F0000703E000070410000E03F16
:102D100080F20000009B28005A423100FDF79CFD24
:102D20000022584B04000D0008F0F0FF002821D0CD
:102D30000022554B200029000BF0FCF80CF01CF889
:102D400006900CF055F800224E4B0BF0F3F8020001
:102D50000B00200029000BF0B5FB0CF00DF80CAEB9
:102D6000BB00F050009B069A183301370093BB005C
:102D70009A5133E7200029000BF0FEFFBE000CAB98
:102D800098512BE7F30070AAD31800930CAAB30054
:102D900098580CF02DF822002B000BF0CBF8009B7C
:102DA00000221860596020002900374B0BF0C2F850
:102DB000013E04000D0019E7079901360CC907917F
:102DC00003CC0BF0B7F802000B00009801990AF051
:102DD00055F800900191052E02D0069BB342EBDA24
:102DE000069B013DDC0048AB1C19009A019B226048
:102DF000636001E7EB00E3181A685B680AF03EF8CD
:102E0000013D002DF6DA029D02000B00002D02D0DC
:102E100080252D064B190A9D2A606B6002000B006D
:102E2000489849990BF04EFB012500900191083418
:102E3000AF421CDA029B002B07D0009880210200D1
:102E4000019809064318009201930099019A0720FE
:102E50000A9B9960DA60049B0340180099239B0049
:102E60009D44F0BD3D000020002148ACC9E700981A
:102E70000199226863680AF001F801350090019118
:102E8000D5E7C046000070410000703E064A137846
:102E900001788B4201D0581A704701320130002B63
:102EA000F5D11800F8E7C04680010010F0B5050024
:102EB0001C0085B0002801D00023037000263300D9
:102EC0001178002900D19CE0632E04D90023013D34
:102ED0002B70013E99E0252904D00132297001367A
:102EE0000135EDE751780391252902D1297002328D
:102EF000F5E70399971C302902D0571C2022039232
:102F00003A782D3A50424241BF18002230214942BE
:102F10008C4638788444614609290ED99119642970
:102F200002DD6422921BD2B26C2817D862280BD81B
:102F3000582857D00126764267E00A214A43821872
:102F4000303AD2B20137E1E763380928F2D808F005
:102F5000ABFD541FF1F1F1F11FF1F12F752821D0D4
:102F6000782837D07328E5D108CC00209C466346EA
:102F70001B5C002B3AD1121A2B18D1188C466146D3
:102F8000C91A002935DCD343DB1713401B1805E0B1
:102F9000280008CC0399FFF702FB03007A1CED1808
:102FA000F6188DE7280008CC0399FFF793FAF4E7A9
:102FB00078786C28F2D1B8787528EFD107230734D8
:102FC0009C4303CC00900191280003990237FFF73E
:102FD000AEFAE2E708CC0093002328000399FFF73C
:102FE00017FBDAE708CC00930123F6E72B540130F6
:102FF000BDE7039919700133C1E708CC2B70012399
:10300000CCE7632E00D961E72970300005B0F0BD30
:10301000F0B589B0059305230391049202937A28B1
:103020001BD800213E4B10381A78884218DC991CB6
:103030005B78019102938B1806930E9B002B04D0B2
:10304000039B029A9B1A01330393059B002B27D104
:1030500000252F00029BBB4225DC029809B0F0BD81
:1030600002329B180131DFE76B461C7C049B102267
:103070001B07DB0FBB4200D00822D3B20793039B90
:103080005E19F6B221003000FDF76BF90134079BA1
:10309000E4B29C42F6D10135029BAB42E4DCD7E7B7
:1030A00000250127F8E76B461C7C049B10221B07B8
:1030B000DB0F012B00D008220826D3B20793082E7D
:1030C00008D1069B019A9342C7D013000026013312
:1030D0001578019301231D4215D0039BF818059B19
:1030E000C0B2002B18D083280DD884228121E30898
:1030F0005B4213407D3A2240494211411818094B66
:103100001A5C0A401A540134079BE4B26D10013670
:103110009C42D4D101379DE72100FDF722F9F2E767
:1031200078F4000094020010F0B587B00C0017008E
:1031300003900493FFF79AFA451E002D01DB002C43
:1031400001DC07B0F0BD039B2100585D01233A006C
:103150000093049BFFF75CFF049B241A002B13D001
:10316000002D11D03B071022FEB2DB0F012B00D047
:103170000822D3B205933100E0B2FDF7F2F8013630
:10318000059BF6B29E42F6D1013C013DD5E7F7B56D
:10319000012300246D4600930194502300262868E3
:1031A0005B421843C0B2FEF7E0FF0020FEF7DDFFF0
:1031B0001020FEF7DAFFE020FEF7D7FF094FE719EE
:1031C000012200210220FEF791FFB85D0136FEF7D3
:1031D000AFFF842EF4D10435842C00D1F7BD340028
:1031E000DBE7C046940200100223174A10B51168AD
:1031F00016480B4313602023154A11680B431360D4
:10320000144B1A6802401A600122196811431960B0
:10321000114B19680140196019680A431A606C2241
:103220000E4B0F491A600F4BD86F08F051FC8022EB
:103230000D4B120218600D4B18600D4B1A60802365
:103240004022DB051A6010BD04800440F8FCFFFF3B
:103250008080044030400440344004401800004066
:10326000400D030058010010140000401000004001
:1032700000E100E08022114B10B5DA679218DA679E
:103280008022D200DA6780225201DA67802212019E
:10329000DA6780229200DA6700230121084A494256
:1032A0001360084A1160084A1360084A136001223B
:1032B000074B1A60FFF798FF10BDC04604E100E01D
:1032C000048204400882044004C000403CC0004026
:1032D00000C00040802210210820064BD20511605A
:1032E000186080235B011068084202D0013B002B6C
:1032F000F9D1704718000040802100222020134B94
:10330000C90510B5DA651A669A6408601049D86D67
:10331000012807D08A4203D1FFF7DCFF002010BD4F
:103320000132F4E78A42F7D00022596C0139D86D96
:10333000FF2801D9D86DF2E7586C884202D0596C49
:103340005A680A3258688242F1D1E5E75801001004
:10335000FF0F0000F8B50500032402260127A22272
:10336000084B5E669F664C331A7001325D709A702E
:10337000FFF7C2FF0223FF33984202D0013C002C2A
:10338000EDD1F8BD5801001010B5814208D20139C5
:103390000138002A00D110BD8B5C8354013AF8E754
:1033A0008142F8D9002302E0CC5CC45401339A4234
:1033B000FAD1F0E7F7B52E4B2E4A01931378002B84
:1033C00006D00C2B02D10B3B1370F7BD0133FBE78A
:1033D000294D2B7E002B17D06E7EA97EAA7D7442CC
:1033E00074410C40E97E701C2818AB190C4304D0C2
:1033F00001001800FFF7C8FFE7E71900FFF7C4FF57
:103400002D236C75AB55E0E70122019BA4331A70A4
:10341000019B0022A8331C685D689E68DF6820005D
:103420000023290008F04EFC002803D18021090662
:103430006B181D00002200233000390008F042FC08
:10344000002803D1802109067B181F0000220023D9
:10345000300039000AF06EFD22002B0009F00EFD4D
:10346000019C064BB0341860596026606760ACE779
:10347000700B0010F30B001080010010180C0010EE
:1034800010B50B4C2068002806D00220FFF762FF21
:103490000238FF3843425841064BE0721A780A233B
:1034A0005106490F4B430F210A409B18637110BD11
:1034B000D8010010C4010010F8B505000E00032467
:1034C000A227094BB21C5A6600224C33DA611F70E6
:1034D0005D70FFF711FF0223FF33984202D0013CD9
:1034E000002CEED1F8BDC04658010010012010B5E7
:1034F000FFF730FF0223FF33984210D10120094A21
:10350000094B14781860094B220706D003224C336C
:10351000224001009A70FFF7CFFF200010BD012468
:103520006442FAE7C4010010D801001058010010ED
:10353000074B10B51B68002B09D0064B140A1A70F4
:103540005C70140C120E9C70DA70FFF7B5FF10BDA2
:10355000D8010010A601001010B5FFF7C7FF022028
:10356000FFF7F8FE0223FF33984220D1104A114B97
:1035700012787F2A16D9104A1268002A12D01A002F
:103580000021082001244E329070D47051701170C7
:10359000142252330638D970073118705C709A7053
:1035A000FFF78AFF04210920044AFFF7C1FF10BD7D
:1035B000C401001058010010D801001080808080E4
:1035C00030B50A4B652803DD032287331A7030BDFE
:1035D00000011B180933FF331C685D689A68DB68BB
:1035E0000C604D608A60CB60F1E7C046700B001044
:1035F00010B5802805D8034B8000C358002B00D09D
:10360000984710BDA4F8000070B5114B11491A88F5
:10361000114C885C002803D1002A01D0188070BDAD
:10362000230085331B78002B02D0FCF721FFF6E73F
:103630002500012386352B70FFF7DAFF2B78002B4E
:1036400001D0FCF715FF002386342370E7E7C0465E
:10365000EC0B00109C030010700B0010030010B561
:1036600063280CD96420FE2B09D00130FD2B06D035
:10367000094CFF2B04D0032300208734237010BD96
:10368000E923DB00E318186859680BF075FB08F0B4
:10369000FDF86328EFDCF2E7700B001010B5682826
:1036A00002D8FCF773FE10BD094BFE280AD1E922AF
:1036B000D2009B18186859680BF05EFB08F0E6F81A
:1036C000C0B2EEE70322873300201A70EBE7C04652
:1036D000700B0010030010B50E2809D90F20FE2B27
:1036E00006D1044B186859680BF046FB08F0CEF879
:1036F00010BDC046B812001010B509280BD9094BEF
:10370000FE2809D1E922D2009B18186859680BF0ED
:1037100033FB08F0BBF810BD0322873300201A707A
:10372000F9E7C046700B00100FB430B59BB01EAB6C
:1037300004CB642101A80093FFF7B8FB63280DDDDB
:10374000FEE7013315680D42FCD020601878002890
:10375000F7D11BB030BC08BC04B018472021024A86
:10376000024C01ABF2E7C0461480004000800040EC
:103770000EB403B503AB04CB64210193FFF796FBB2
:1037800002B008BC03B01847F0B5374B89B00493BA
:103790000023364D0E006C5C02A903900B739A4215
:1037A00004D01522324904A8FFF7E2FF2000FCF7FD
:1037B00023FE07003000FCF747FE002F1AD0002838
:1037C0001AD1AD196D7806AF00210522380003F03B
:1037D00095F82849FE2D02D0FF2D1ED1264938002C
:1037E000FFF7C6FF762C2CD1244BAD005B19244982
:1037F0009B6B0AE0002804D0731EEC5CAD5D1E00DC
:10380000E1E7204BA4002049E358009332000398DD
:1038100004ABFFF7ADFF09B0F0BD1C49FD2DDED0B4
:10382000632D1AD923004F3B012B04D92B2C02D036
:10383000A31F012B11D82A0038000D49233AFFF7A6
:1038400097FF104BA400E3583200009310490398EF
:10385000019704ABFFF78CFFDDE72A0038000D4924
:10386000FFF786FFBEE7C046202000009C03001043
:10387000F3EF000083EF0000F0EE000000F3000023
:10388000FDEE0000A8FA0000E8EE0000F4EE0000F3
:1038900006EF0000FAEE0000F0B585B00600002447
:1038A0000391FEF7E3FE25000700AF4201DD832C04
:1038B00001DD05B0F0BD0023705D2100039A009387
:1038C000FFF7A6FB241801340135EEE782B070B58E
:1038D00005930492124B652806DD032287331A7084
:1038E00070BC08BC02B0184702019A18F832049C58
:1038F000059D14615561069C079D9461D5616528FD
:10390000EED1EB22D200991808684968054A064BA7
:103910000AF010FB09F094F907F0BCFFE0E7C0469D
:10392000700B00100000C0FFFFFFDF41F8B5FEF78D
:10393000C7FC594F0400031E3E69584D42D1032E67
:103940000AD12B002A0085337A321B781278134370
:10395000002B05D1340003E0532E2CD0002E20D0B4
:103960002B0081331A78002A03D0052E01D00022C3
:103970001A702B0082331A78002A03D0092E01D046
:1039800000221A702B00002284339A56002A05D098
:103990002F2E05D0572E03D000221A703A2E0ED0AB
:1039A00026002A0000237A32793513703B612B7090
:1039B0007B613000F8BD2B0085331B78C8E7FCF72E
:1039C00037FCEDE72A0081321278002A21D0283412
:1039D000FB22053B134204D12000282108F05EF9A8
:1039E0000C00B44243D1032C2BD12B0085331B7820
:1039F000002B15D000257B69022B31DD642DD8DC2E
:103A00000120FEF7D5FCFEF75BFC002810D0013545
:103A1000F1E72A0082321278002AD9D05034D7E751
:103A20001F4C0120FEF7C4FCFEF74AFC002801D120
:103A30000026BEE7013C002CF3D17A3501232B7020
:103A4000F6E7532CD6D0174C0120FEF7B1FCFEF759
:103A500037FC0028ECD0013C002CF5D1A036A8E7BB
:103A6000114A9542CCD101337B612600A1E72B009E
:103A70000833DA6F0D4B3C611A42F6D1032C01D0AA
:103A8000532CF2D1C820FEF793FCFEF719FC002856
:103A9000CED07935D2E7C046D8010010700B0010A7
:103AA000D1070000E90300005902000000FFFF00F9
:103AB00049004B0819007047F0B54B0091B05B0806
:103AC00000931700B14B009A08919A4207D8002240
:103AD000002338607960BA60FB60002626E0AC4BBA
:103AE000009A9A4200D973E0089BAA4CAA4A002B7C
:103AF00037DDA84B0AF0E6FC009B02900391A3423D
:103B000017D0A64AA64B0AF0DDFC02000B00040009
:103B10000D00029803990AF0D5FCA04AA04B0AF0C8
:103B2000D1FC01263C607D60B860F960300011B0C6
:103B3000F0BDD32202980399994B52050AF0C2FCBA
:103B4000984A994B009001910AF0BCFC02000B00CE
:103B500004000D00009801990AF0B4FC914A924BC0
:103B6000DDE78C4B09F08AF9009B02900391A34298
:103B700016D08A4A8A4B09F081F902000B00040032
:103B80000D00029803990AF09DFC844A844B09F0C9
:103B900075F901263C607D60B860F9607642C5E742
:103BA000D322029803997E4B520509F067F97D4AAA
:103BB0007D4B0090019109F061F902000B000400B7
:103BC0000D00009801990AF07DFC764A764BDEE7FD
:103BD000764B009A9A4200D9CBE0FFF769FF744A0E
:103BE000744B04000D000AF0A5F90022724B09F095
:103BF00045F90BF0C1F806000BF0FAF8664A654B80
:103C0000069007910AF096F902000B0020002900A7
:103C10000AF058FC614A0290039106980799604B9C
:103C20000AF088F902000B000490059102980399AC
:103C30000AF048FC04000D001F2E06DC5F4B721ECC
:103C40009200D358009A934208D1009B1B15099308
:103C5000099A6B005B0DD31A102B02DC3C607D606F
:103C60003CE0D322069807994D4B52050AF062F9C1
:103C700004000D0002000B00029803990AF022FCD8
:103C800002000B0000900191029803990AF01AFCBF
:103C900022002B000AF016FC04000D00069807997C
:103CA000404A414B0AF046F922002B000AF00AFC78
:103CB00002000B0004900591009801990AF002FCA3
:103CC000099A4B005B0D04000D00D31A312B1EDC4A
:103CD000009A019B3C607D600292039302980399D5
:103CE00022002B000AF0EEFB049A059B0AF0EAFB87
:103CF000089BB860F960002B00DB17E780221206F2
:103D0000AB187B608B183C60B860FB6046E7B8225C
:103D100006980799244B92050AF00CF904000D004F
:103D200002000B00009801990AF0CCFB02000B0086
:103D300002900391009801990AF0C4FB22002B0025
:103D40000AF0C0FB04000D00069807991C4A1D4BA1
:103D50000AF0F0F822002B000AF0B4FB02000B007E
:103D600004900591029803990AF0ACFB04000D0041
:103D700074E7154B009A9A4228D902000B000AF00A
:103D8000A1FBB860F96038607960A6E6FB21E93FE5
:103D90007BD90240FB21F93F000040543163621A95
:103DA00061B4D03D7370032E8A19A33BFB213941C6
:103DB00083C8C96D305FE43F0000E03F24F8000095
:103DC000C14920259A837B39FFFFEF7F009A29495B
:103DD0001215521813050292009A0400D51A2900F0
:103DE0000AF0CAFF0BF004F802000B0020002900C3
:103DF0000A920B930AF066FB00221F4B0AF09AF816
:103E00000D0004000AF0B8FF0AF0F2FF02000B00F8
:103E100020000C920D9329000AF054FB0022164B4F
:103E20000AF088F80AAE3400032530617161206918
:103E30006169002200230095083C013D07F042FF24
:103E40000028F4D13000009B3900029AFEF79EFD55
:103E5000089B0600002B00DB68E6802079683A6842
:103E600000060B18F9683A607B60BA680B18BA60F4
:103E7000FB6093E6EAFBFFFF0000704130B5214A8A
:103E80004B0087B05B08934204D800220023FCF764
:103E90004BFD06E01C4A934205D902000B000AF0D4
:103EA00011FB07B030BD0023002202AC0292039345
:103EB000049205932200FFF7FFFD049C059D03007B
:103EC0000298039903221340012B06D0022B0DD038
:103ED000002B10D122002B00D9E7009322002B00E9
:103EE000FCF774FE80231B06C918DAE722002B00BA
:103EF000FCF71AFDF6E70123220000932B00FCF7E4
:103F000065FECEE7FB21E93FFFFFEF7F30B5234A97
:103F10004B0087B05B08934206D800230022009331
:103F20000023FCF753FE06E01D4A934205D9020028
:103F30000B000AF0C7FA07B030BD0023002202AC24
:103F400002920393049205932200FFF7B5FD049CAF
:103F5000059D03000298039903221340012B08D00A
:103F6000022B0BD0002B13D10133009322002B0026
:103F7000D7E722002B00FCF7D7FCDCE70123220067
:103F800000932B00FCF722FE80231B06C918D2E702
:103F900022002B00FCF7C8FCF6E7C046FB21E93FF6
:103FA000FFFFEF7F82B0D3B5069207930400069817
:103FB0000799FDF741FB06000F0008980999FFF7E4
:103FC000A5FF32003B0009F0B5FF00900191089871
:103FD0000999FFF753FF32003B0009F0ABFF0022C5
:103FE00006000F0000980199002309F0A3FF0200CA
:103FF0000B003000390008F041FF009A019B20605F
:104000006160A260E3602000D6BC08BC02B0184723
:10401000F0B58DB0009201934B005B080493049AB5
:10402000C94B04000D0009919A425DD80AF0A4FE24
:104030000290002800D084E0129B049A01332343AD
:1040400013430FD120002900FFF732FD02000B00BF
:104050000020BE4909F02CFB04000D0020002900BF
:104060000DB0F0BD129B012BF8D0009A019B2000EF
:10407000290008F003FF020002980B00049005914C
:104080000020B34909F014FB220006900791049820
:104090000599069E079F2B000AF014FA029E020063
:1040A0000B00009801990AF00DFA32003B0009F06C
:1040B00041FF320004000D00049805993B0009F00F
:1040C00039FF0022A14B08F0D9FE02000B002000AE
:1040D000290008F0D3FE069A079B09F02BFF320057
:1040E0003B0008F0CBFEB7E79A4B049A9A4228D9D6
:1040F000099B002B0DDA80208021000684460906EA
:104100006B1800991D000A00019961440B00009290
:10411000019322002B00904890490AF0D3F9009AAD
:10412000019B04000D008E488E490AF0CBF9220055
:104130002B0008F0A3FE0022002304000D000092D3
:10414000019322002B002000290009F0F3FE020059
:104150000B000290039109F0EDFE029A039B06000A
:104160000F002000290009F0E5FE7F4A0690079124
:104170007E4B3000390009F0DDFE7D4A7D4B08F0B2
:104180007DFE32003B0009F0D5FE7B4A7B4B08F0F8
:1041900075FE32003B0009F0CDFE794A794B08F0FC
:1041A0006DFE32003B0009F0C5FE774A774B08F000
:1041B00065FE32003B0009F0BDFE754A754B08F004
:1041C0005DFE029A039B09F0B5FE734A0A900B91BB
:1041D000724B3000390009F0ADFE714A714B08F0A6
:1041E0004DFE32003B0009F0A5FE6F4A6F4B08F010
:1041F00045FE32003B0009F09DFE6D4A6D4B08F014
:104200003DFE32003B0009F095FE6B4A6B4B08F017
:1042100035FE32003B0009F08DFE694A694B08F01B
:104220002DFE02000B000A980B9908F027FE069A53
:10423000079B09F07FFE009A019B08F01FFE029A7F
:10424000039B09F077FE009A019B08F017FE060019
:104250000F00069807995C4A5C4B09F06BFE320030
:104260003B0008F00BFE02000B00029003912000BF
:10427000290008F003FE374B049A06000F009A420B
:104280003DD912980AF0B4FD3200009001913B0034
:104290003000390009F04EFE009A019B0490059110
:1042A0003000390008F0EAFD02000B00049805997F
:1042B00009F0FEF9029A039B0AF004F902000B00D0
:1042C000200029000AF0FEF802000B0008F0D6FDDD
:1042D00002000B00009801990AF0F4F80222040091
:1042E0000120099B0D009B171340C01A0AF080FDA6
:1042F00002000B002000290009F01CFEACE6129B16
:10430000012B1DD00023009601970093009A019B7A
:104310000492059302000B0000200D4909F0C8F932
:1043200022000690079104980599069E079F2B008E
:104330000AF0C8F8002602000B0002980399B2E6C2
:1043400004000D008AE6C046FFFF2F3E0000F03F4C
:104350000000F0BF2794E53F182D4454FB21E93FAE
:10436000075C143326A6813CD47ABF74702AFB3EC6
:10437000E9A7F0320FB8123F68108D1AF726303FC8
:104380001583E0FEC8DB573F93846EE9E326823F46
:10439000FE41B31BBAA1AB3F735360DBCB75F3BED9
:1043A000A69237A0887E143F0165F2F2D844433FBD
:1043B000280356C9226D6D3F37D60684F464963FB4
:1043C0007AFE10111111C13F635555555555D53F12
:1043D000F0B5984B85B04E0004000D0003917608AF
:1043E0009E4218D9944B9E4202D80AD1002808D088
:1043F00022002B002000290008F040FD04000D00E1
:1044000005E0039B8D4C002B00DC11E18C4D20005E
:10441000290005B0F0BD8B4B9E420FD88A4B9E42BF
:1044200009D88A4A8A4B08F029FD0022894B07F0F7
:1044300063FC0028EBD101235B4225E0FFF738FB4A
:10444000854B04000D009E4200D9AAE0834B9E429A
:1044500000D990E002000B0008F010FD00227D4B17
:104460000AF030F8802306000F0000222000290007
:10447000DB0508F003FD0B0002003900300009F0F5
:1044800017F9002304000D002200029320002B00E6
:10449000290009F04FFD02000B000090019109F086
:1044A00049FD06000F006E4A6E4B09F043FD6E4A4F
:1044B0006E4B08F0E3FC32003B0009F03BFD6C4A18
:1044C0006C4B08F0DBFC32003B0009F033FD6A4A1C
:1044D0006A4B08F0D3FC32003B0009F02BFD684A20
:1044E000684B08F0CBFC32003B0009F023FD664A24
:1044F000664B08F0C3FC009A019B09F01BFD644A5F
:1045000000900191634B3000390009F013FD624ABD
:10451000624B09F0D7FF32003B0009F00BFD604A07
:10452000604B09F0CFFF32003B0009F003FD5E4A0B
:104530005E4B09F0C7FF32003B0009F0FBFC5C4A10
:104540005C4B09F0BFFF32003B0009F0F3FC0200B6
:104550000B000098019908F091FC2B00220009F053
:10456000E9FC029B013343D102000B00200029002B
:1045700009F0A8FF42E70022364B09F0A3FF002212
:1045800006000F0020002900324B08F077FC0B00DA
:1045900002003900300009F08BF8012304000D00FF
:1045A00072E7454B9E4219D80022444B09F08AFF1E
:1045B000002206000F0020002900404B09F0BAFC41
:1045C0000022244B08F05AFC0B0002003900300096
:1045D00009F06EF8022304000D0055E70B000200FD
:1045E0003749002009F064F8032304000D004BE76D
:1045F000029B344FDE00344BBF199E193269736938
:1046000009F060FF22002B0009F05CFF0B000200A4
:10461000386F796F09F056FF039B04000D00002BE3
:1046200000DBF4E6802109066B1804001D00EEE6AD
:10463000264DECE6FFFF0F440000F07F182D445498
:10464000FB21F93FFFFFDB3FFFFF1F3E9C7500880A
:104650003CE4377E0000F03FFFFFF23FFFFFE53F05
:1046600011DA22E33AAD903FEB0D76244B7BA93F64
:10467000513DD0A0660DB13F6E204CC5CD45B73F32
:10468000FF8300922449C23F0D5555555555D53FDE
:104690002F6C6A2C44B4A2BF9AFDDE522DDEAD3FD2
:1046A0006D9A74AFF2B0B33F711623FEC671BC3F72
:1046B000C4EB98999999C93FFF7F03400000F83FE8
:1046C0000000F0BF00F3000080F30000FB21F9BF01
:1046D000F7B554425E001443454F7608E40F01934A
:1046E0003443BC4208D844424D0004436D08E40FF3
:1046F00000912C43BC4203D908F0C0FB03B0F0BDCD
:104700003C4C1C19144302D1FFF762FEF6E79C17DC
:10471000A446022467463C40CF0F3C432F0007438A
:1047200006D1022C58D0032CE8D133483349E5E7B1
:104730003700174305D1009B2F48002B55DB30492C
:10474000DCE72B4FBE4212D1013CB54207D1022C0F
:1047500045D82C4BE4001B19186B596BCEE7022C83
:1047600040D8284BE4001B19986CD96CC6E7204F41
:10477000BD42E0D0AD1B2D153C2D17DC019E002E57
:1047800001DA3C3515DB08F093FFFFF791F9FFF7ED
:104790001FFE012C10D0022C13D0002CAED01A4AD0
:1047A0001A4B09F08FFE144A194B12E012481449B3
:1047B000EFE700200021ECE7802424060B19190004
:1047C0009CE7114A114B09F07DFE02000B000A48DC
:1047D0000F4909F077FE91E707480D498EE7064833
:1047E0000C498BE70020002188E70B4986E7C0468B
:1047F0000000F07F000010C0182D4454FB2109C0B8
:10480000FB21F93F80F30000075C143326A6A13C8E
:10481000FB210940FB21E93FFB21F9BF82B0D3B561
:10482000069207930400089A099B06980799FDF7DA
:10483000DDF8FCF727FD069A079B00900191089888
:104840000999FFF745FF0022002306000F0009F039
:1048500071FB009A019B08F011FBA660E7602060E5
:1048600061602000D6BC08BC02B0184782B0F0B529
:1048700089B00E920F930E9E0F9F0390002200238B
:104880003000390007F01EFA002808D0109811995E
:104890000022714B07F030FA002800D0CDE0320042
:1048A0003B003000390009F045FB02000B0000908E
:1048B00001910020684909F005FE109A119B04003F
:1048C0000D001000190009F035FB02000B0020005C
:1048D000290009F0F7FD04000D0032003B00300014
:1048E000390008F0CBFA22002B00FFF7F1FE00227E
:1048F0005A4B09F01FFB5A4A5A4B0490059108F095
:10490000D7FE0022002304000D0007F0FFF900226B
:10491000524B002800D18BE02000290008F0AEFAAD
:1049200000224D4B04000D001098119909F0CAFDAA
:1049300002000B0009F0FEFA009A019B08F09EFAB3
:10494000002200230690079107F0BCF9002800D050
:1049500073E0290020000AF00FFA0AF049FA002259
:1049600006000F00109811993B4B08F087FA0200DF
:104970000B0009F0DFFA009A019B08F07FFA069A13
:10498000079B08F095FEFCF77DFC0022364B09F0F2
:10499000D1FA364A00900191354B3000390009F0C8
:1049A000C9FAA822069007912E4B30003900D20593
:1049B00009F0C0FA02000B000498059909F082FD85
:1049C000802204000D00300039002A4B520509F006
:1049D000B1FA02000B002000290009F073FD00224B
:1049E00006000F0000980199002309F0A3FA069A27
:1049F000079B04000D003000390009F063FD020040
:104A00000B002000290008F039FA002204000D00F4
:104A100000980199002308F031FA039B9860D9604F
:104A200018001C605D6009B0F0BC08BC02B01847FB
:104A30002000290009F046FD72E700220E4B0020FD
:104A4000002109F077FA00220B4B08F017FA040056
:104A50000D0000200849E0E70000F03F0000E03FC3
:104A6000182D4454FB2109400000D03F6EC0453151
:104A700063626A3C460B213E0000F07F82B0F0B5D5
:104A80008BB010921193129C139D0022109E119FC7
:104A900000230790290020000094019507F012F9E7
:104AA0000022002300283AD03000390007F00AF92C
:104AB000002831D130003900FEF7FAFFFCF732F957
:104AC0000022002304000D003000390007F000F937
:104AD00000220023002816D02000290009F02AFA1D
:104AE0000022002308F0CAF900940195009E019F5E
:104AF000079B1860596018009E60DF600BB0F0BC27
:104B000008BC02B018470098019909F013FA220076
:104B10002B0008F0B3F9E9E700200021E6E73000B8
:104B2000390007F0CFF8002829D020002900FEF72F
:104B3000BFFF0022734B09F0FDF9FCF7F3F80022E8
:104B4000002306000F0009F0F5F900220090019102
:104B500000232000290007F0CFF8009A019B0028CD
:104B600004D03000390008F089F9C1E7300039007D
:104B70008024240609F0A6FC3B191F00B8E730008A
:104B80003900FEF795FF00225F4B07F0B5F80028CB
:104B900009D120002900FEF78BFF00225A4B07F0B5
:104BA000ABF8002875D0002230003900574B09F0CF
:104BB000C1F9564B06000F0020000022290009F021
:104BC000B9F98024002300900191E4050293039435
:104BD000009801990022002309F0ACF932003B0053
:104BE00008F04CF9009A019BFCF700FF0022454BAE
:104BF00009F0A0F9002204900591424B30003900E1
:104C000009F098F9002204000D00009801993D4B2D
:104C100009F090F900220890099100233000390032
:104C200007F06AF822002B00002846D00498059966
:104C300008F024F9FCF776F802000B0004000D00E0
:104C40000898099908F034FDFEF732FF029A039B99
:104C500009F070F9220006000F00029803992B005A
:104C600009F068F904900591002200233000390012
:104C700009F060F9002204000D000098019900235A
:104C800007F026F8002837D00498059922002B0059
:104C90006EE70022300039001D4B09F04BF91C4B28
:104CA00006000F0020000022290009F043F9F92432
:104CB000002300900191A40588E70498059909F064
:104CC00001FCFCF72FF802000B0004000D0008980F
:104CD000099908F0EDFCFEF7EBFE029A039B09F040
:104CE00029F9220004900591029803992B0009F0FC
:104CF00021F906000F00B7E72000049A059B290060
:104D000031E7C0460000E03F000010400000D03F07
:104D10000000504382B0F0B593B0079018921993F9
:104D20001A981B990022002309F004F9189A199B7C
:104D300008F0A4F800240200002500200B004749D9
:104D400002940395049005911A981B990090019183
:104D50000EA807F005F80E9A0F9B0A920B93109A73
:104D6000119B0C920D93189A199B1000190008F0D2
:104D700085F81A9A1B9B09F0DDF822002B0006002B
:104D80000F0009F0D7F81A9A1B9B04000D00189821
:104D9000199909F097FB1A9A1B9B0890099118988A
:104DA000199908F06BF802000B000898099909F0AE
:104DB000C1F822002B0008F061F802000B0000206F
:104DC000264909F07FFB22002B0009F07BFB002223
:104DD00000230892099380231B06FB18020001930D
:104DE00000960B000EA80896FFF748FE0E9A0F9B40
:104DF0000A980B99109E119F08F040F804000D00CE
:104E00000C980D9932003B0008F038F8220000247D
:104E10002B00134D019100900EA8FFF7FFFC109896
:104E200011990E9A0F9B04940595802500242D0658
:104E300000900191029403950EA806F091FF0E9840
:104E40000F99109A119B079C206061602000A2605E
:104E5000E36013B0F0BC08BC02B018470000F03F9C
:104E60000000F0BFF0B5494A4E0004000D000B00F1
:104E700085B07608964208D9020007F0FFFF0400CB
:104E80000D002000290005B0F0BD0022002942DB02
:104E90003F4B009201933F4B9E4249D83E4B9E426E
:104EA0000BD83E4A3E4B2000290007F0E7FF0022C6
:104EB0003C4B06F021FF0028E3D120002900FEF73B
:104EC000F7FDFCF7CDFE374B002204000D0007F084
:104ED000D5FF354B029003919E421ED822002B0035
:104EE0002000290007F0CAFF220006000F002B0057
:104EF0002000290009F01EF8029A039B08F0D8FB55
:104F000002000B003000390009F0DCFA009A019B26
:104F100009F010F8B3E7254BBBE7029A039B20008A
:104F2000290008F0C5FB22002B0007F0A7FFEDE7E2
:104F30001F4B9E4206D820002900FEF7B9FDFCF762
:104F40007BFBE3E71B4B9E4205D91B4B9E4217D1CF
:104F50001A4A944214D820002900FEF7A9FD002225
:104F60000B4B08F0E7FFFCF767FB04000D000200A5
:104F70000B000098019908F0DDFF22002B00C7E725
:104F800020002900054A064BC2E7C046FFFFEF7F1D
:104F90000000E03FFFFF3540FFFF2F3E3374AC3C85
:104FA0001F7BAC7F0000F03FFFFFEF3F0000E0BF42
:104FB000412E8640CD338640CE3386407DF8B98F72
:104FC0003E4BF7B54E0076089E4204D902000B0016
:104FD00008F0B0FF2AE03A4B9E422DD8FEF768FD5C
:104FE000FCF73EFE374B00220090019107F046FF90
:104FF000F22304000D009B059E4219D3009A019BE9
:105000001000190008F096FF220006000F002B0088
:105010002000290007F032FF02000B0030003900A9
:1050200008F046FB0022274B07F028FF04000D0084
:105030002000290003B0F0BD234B9E4216D8FEF796
:1050400037FDFCF7F9FA0022204B04000D0008F0B0
:1050500071FF220006000F002B0000201B4908F002
:1050600027FB02000B0030003900DDE7184B9E42A1
:1050700006D8FEF71DFDFCF7DFFA0022134BA7E769
:10508000144B9E4205D9144B9E4213D1134A9042B1
:1050900010D8FEF70DFD00220C4B08F04BFFFCF77B
:1050A000CBFA04000D000022084B08F043FF220059
:1050B0002B008DE70020FCF797FAB7E7FFFFEF7FA3
:1050C000422ED63F0000F03FFFFF35400000E03F9A
:1050D000412E8640CD338640CE3386407DF8B98F51
:1050E000F7B517001E0004000D00FEF7E1FC0022DA
:1050F0001B4B06F0F7FD00280CD020002900FFF71D
:105100005FFF3860796020002900FFF7ABFE306058
:105110007160F7BD20002900FCF78EFA04000D0035
:1051200002000B0000200E4908F0C2FA0022009095
:1051300001910B4B2000290008F0FCFE009A019B16
:1051400004000D0009F0BEF9220030607160009883
:1051500001992B0007F092FE38607960D9E7C046CC
:105160000000E03F82B0D0B586B004000C980D99E5
:105170000A920B9304AA02ABFFF7B2FF0A980B99AD
:10518000FEF77CFE029A039B08F0D4FE06000F0097
:105190000A980B99FEF7BAFE049A059B08F0CAFE1E
:1051A00000220090019100233000390008F0C2FE77
:1051B00002000B000098019907F060FE206061601A
:1051C0002000A660E76006B0D0BC08BC02B018475B
:1051D000F0B597B004920593049B059F1A007D00DB
:1051E0006D08029003912A431AD18021029A0398F4
:1051F00009034840030092185B4196498B4206D848
:1052000001D000F0CCFC002A01D100F0C8FC049AC7
:10521000059B0298039907F031FE009001918EE002
:10522000039A0692029A0A92039A54008A4A6408E0
:1052300094420ED805D10A9A002AE8D1A542E6D8B0
:1052400002E0854A954204D8834A95420CD1002B4E
:105250000AD0824A039B9B18029A1343D7D180211C
:10526000049A05980903C4E70026069A0894B242F6
:1052700042DA7B4A95423ED87A4A954210D97A4919
:105280002A155218142A18DD3421891A049ACA40A2
:1052900010008840984203D1012102360A40B61A14
:1052A000002B5BD18023DB059F424CD1029A039BEC
:1052B0001000190008F03EFEAFE7002B4ED114336A
:1052C0009A1A2B00134119009140A94203D10122DF
:1052D00002261340F61A654B9D42E3D1029B039CC4
:1052E00000930194002F2ADA1A00002023005F495E
:1052F00008F0DEF991E70226002B2FD1564B9D4294
:10530000E9D1564B029AE318134301D100F047FC50
:10531000544B9C4209D9049B059C00930194002F97
:105320000DDA0023002400F03CFC002FF9DA802283
:1053300012069446049B0093059B634401930098D6
:10534000019917B0F0BD4A4B9F4207D1069B002B35
:1053500004DB02980399FBF7E5FC5EE702980399EA
:10536000FEF7A6FB0A9B00900191002B2CD1039B1A
:105370003E4A9B009B08934201D0002C24D1002F71
:1053800007DA009A019B0020384908F091F9009053
:105390000191069B002BD2DA304BE418344308D13C
:1053A000009A019B1000190009F08CF802000B0014
:1053B0009EE7012EC3D100988021020001980906C2
:1053C000431800920193BAE7039BDB0F013B1A00DD
:1053D000324302D1029A039BE4E7013E00221E43BE
:1053E00013D0224B069207938423DB059D4200D8FD
:1053F000FAE0204B9D4210D91A4B9C4207D8002F4F
:1054000007DA0020FCF7F0F807E71B4BEAE7002F6C
:10541000F7DC0020FCF7FCF8FFE6184B9C420AD8AA
:10542000069807990023002206F052FC431E98417B
:10543000002FEFDAE6E70D4B00229C4220D90698B8
:105440000799002306F044FC431E9841002FD9DC45
:10545000E0E7C0460000F0FF0000F07F000010C051
:10546000FFFF3F43FFFFEF3F01FCFFFF0000F03F66
:105470000000E03F0000F0430000F0BFFEFFEF3F00
:10548000009801994D4B09F01DF8C0224C4BD205F4
:1054900006000F0008F04EFD4A4A029003914A4B65
:1054A0003000390008F046FD002200900191474B82
:1054B0003000390008F03EFD02000B004448454929
:1054C00009F000F832003B0008F034FD02000B0048
:1054D0000020414908F0F6FF320004000D003B00B7
:1054E0003000390008F026FD02000B0020002900E2
:1054F00008F020FD394A324B08F01CFD02000B0079
:105500000098019908F0DEFF02000B0004000D0076
:105510000298039907F0B2FC029A039B00200090C6
:10552000019108F0CFFF02000B002000290008F0D5
:10553000C9FF049C059D002406000F0004980599EE
:1055400022002B000294039508F0BCFF009A019BF7
:1055500008F0F0FC049A059B08900991300039008E
:1055600008F0E8FC02000B000898099907F086FC97
:1055700022002B00049005910098019908F0DAFCB4
:105580000B000200009001910498059907F076FC49
:10559000134B06000F000891994200DCBFE1114B4C
:1055A000CB180343A34200D1A0E10698079900233A
:1055B000002206F08DFB431E984123E70000F03FD8
:1055C0004715F73F44DF5DF80BAE543E0000D03F77
:1055D000555555555555D53F0000E03FFE822B658A
:1055E000FFFF8F40000070BFDC4B039900220B428D
:1055F0000BD1009801990022D94B08F09BFC352271
:1056000000900191019B52420893089BD5491B15BC
:105610005B189B180D93089BD34D1B03D34A1B0BA0
:1056200000261D43934209DDD14A0136934205DD30
:105630000D9B9B1900260D93CE4BED1800980199F8
:105640002900CD4BF2009B18159214935C6E1B6ED3
:105650001A000A930B9423000E900F9108F032FF6A
:105660000E9A0F9B109011910A980B9907F006FC67
:1056700002000B000020BC4908F01AF802000B00E1
:10568000129013911098119908F054FC0890099108
:10569000089B099C80210293039480200023002210
:1056A0006D108905029329430003029B039C09188E
:1056B00000930194B6048B190098019914001D0001
:1056C00008F038FC02000B001098119908F0FAFE5F
:1056D0000A9A0B9B06000F002000290008F0F2FE3A
:1056E00002000B000E980F9908F0ECFE009A019B47
:1056F00008F020FC02000B003000390008F0E2FE48
:10570000129A139B08F016FC089A099B0A900B91B9
:105710001000190008F00EFC06000F00974A984B85
:1057200008F008FC974A984B07F0A8FB32003B00B2
:1057300008F000FC954A964B07F0A0FB32003B00B6
:1057400008F0F8FB934A944B07F098FB32003B00BB
:1057500008F0F0FB914A924B07F090FB32003B00BF
:1057600008F0E8FB8F4A904B07F088FB32000400FA
:105770000D003B003000390008F0DCFB02000B009C
:105780002000290008F0D6FB009A019B04000D00C0
:105790000898099907F072FB0A9A0B9B08F0CAFB5C
:1057A00022002B0007F06AFB009A019B0E900F91DC
:1057B0001000190008F0BEFB00227C4B04000D0015
:1057C00007F05CFB0E9A0F9B07F058FB00200F00C0
:1057D000060002000B000098019908F0ABFB0022C4
:1057E00000900191714B3000390008F06BFE2200EF
:1057F0002B0008F067FE02000B000E980F9908F0CE
:1058000061FE089A099B08F095FB320004000D0028
:105810000A980B993B0008F08DFB02000B0020005A
:10582000290007F02BFB04000D0002000B0000987C
:10583000019907F023FBE02200205D4B12060600D1
:105840000F0008F077FB08900991009A019B300047
:10585000390008F037FE02000B002000290008F094
:1058600031FE544A524B08F065FB534A04000D00C8
:1058700030003900514B08F05DFB02000B002000A6
:10588000290007F0FBFA149B1A6F5B6F07F0F6FA1A
:105890000A900B910D9809F0ABFA04000D000898DE
:1058A0000999159A464B9B181E685F680A9A0B9BCC
:1058B00007F0E4FA32003B0007F0E0FA22002B0088
:1058C00007F0DCFA002022002B000090019108F084
:1058D000F9FD32003B0008F0F5FD089A099B08F03D
:1058E000F1FD02000B000A980B9920E6354A364B71
:1058F0000498059907F0C2FA009A019B04000D0074
:105900003000390008F0DEFD02000B002000290005
:1059100006F0F2F9002800D047E62C4B62E02C4A52
:105920004B005B08934259D92A4BCB18034308D04C
:10593000069807990023002206F0CAF9431E9841F1
:1059400068E5009A019B08F0BDFD049A059B06F0EE
:10595000DDF90028ECD1204B44E0C0460000F07F88
:105960000000404301FCFFFF0000F03F8E98030061
:1059700079B60B000000F0FF80F30000EF4E454ABF
:10598000287ECA3F65DBC9934A86CD3F01411DA9E8
:105990006074D13F4D268F515555D53FFFAB6FDB1E
:1059A000B66DDB3F033333333333E33F000008404E
:1059B00009C7EE3FFD033ADCF5015B14E02F3EBE64
:1059C00000F40000FE822B654715973C00009040D4
:1059D000FFCB904000346F3F00CC9040734A02945C
:1059E000934225D9724A1B159B188022520311003D
:1059F0001941CB195C006F496F4D640D6418254146
:105A00001D401B031B0B13431422121B1341029353
:105A1000089B00202900002B02DA029B5B420293C4
:105A200002000B000098019908F04CFD00900191D4
:105A3000049A059B0098019907F020FA00200022A3
:105A40005E4B06000F0008F075FA009A019B089063
:105A500009913000390008F035FD02000B00049870
:105A6000059908F02FFD564A564B08F063FA564A3E
:105A700004000D0030003900544B08F05BFA0200BE
:105A80000B002000290007F0F9F904000D000200C6
:105A90000B000898099907F0F1F9089A099B06008C
:105AA0000F0008F00FFD02000B002000290008F095
:105AB00009FD3200009001913B003000390008F0F0
:105AC00039FA04000D00424A424B08F033FA424AC8
:105AD000424B08F0F7FC22002B0008F02BFA404A5A
:105AE000404B07F0CBF922002B0008F023FA3E4A86
:105AF0003E4B08F0E7FC22002B0008F01BFA3C4A62
:105B00003C4B07F0BBF922002B0008F013FA02000F
:105B10000B003000390008F0D5FC04000D00020035
:105B20000B003000390008F005FA8023049005913D
:105B3000002220002900DB0508F0C4FC02000B0055
:105B40000498059907F0B4FD009A019B04000D002C
:105B50003000390008F0EEF9009A019B07F08EF949
:105B600002000B002000290008F0ACFC32003B00D2
:105B700008F0A8FC02000B0000201F4908F0A2FC5E
:105B8000029B1B055B181A15002A06DC029AFAF71D
:105B900063FE069A079BFFF78DFB1900F9E70023C8
:105BA000154C00930194FFF7CAFBC0460000E03F8C
:105BB00002FCFFFF01FCFFFF0000F0FF432EE63F69
:105BC000EF39FAFE422EE63F396CA80C615C20BE2C
:105BD000D0A4BE726937663EF16BD2C541BDBB3EF3
:105BE0002CDE25AF6A56113F93BDBE166CC1663FD1
:105BF0003E5555555555C53F0000F03FF0B50C00DA
:105C000085B0050017000268436810001900009273
:105C10000193FBF791F9634A206006001078624B0C
:105C20000138032800D97DE005F048FF02103595C2
:105C3000A6331B78BB4200DB7B1E0F2F00DD0F2736
:105C4000BE4203DA5B429E4200DB96E0300009F080
:105C5000CFF802000B0000205449FFF7B9FA020008
:105C60000B000098019907F023FD01272860696067
:105C7000FBF762F9B84255DB4A4B1B78032B00D087
:105C80007EE0032F00D07BE00022494B2A606B604E
:105C90002368033372E0002200980199454B06F017
:105CA00035F8002807D1009801990022404B06F0F2
:105CB00019F8002861D0300009F09AF802000B00B2
:105CC00000203A49FFF784FA02000B00009801997E
:105CD00007F0EEFC28606960300005F0D7FD032175
:105CE00005F0DCFF0E1E1DD0236800932A686B6848
:105CF00002920393009B002B16DD080009F078F850
:105D000002000B0000202949FFF762FA029A039B68
:105D100008F010F9009B286069609B1B2360771CCA
:105D20000136A5D105B0F0BD03277F1A380009F070
:105D30005FF802000B0000201C49FFF749FA029AA5
:105D4000039B08F0F7F8009B28606960DF1B276061
:105D50000427BF1B8CE70E20801B09F049F80200C6
:105D60000B0000201149FFF733FA02000B000098E6
:105D7000019908F0DFF82860696000232360D1E70B
:105D8000781E09F035F80B00020008490020FFF7E3
:105D90001FFA06F073FF06F08FFF23682860696022
:105DA0000133EBE7150C0010700B001000002440CD
:105DB0000000F03F00408F407FB504000E00151E2C
:105DC00005DD8A4206DD00220023026043600020D8
:105DD00004B070BD0268436828000092019309F086
:105DE00007F802000B0000201649FFF7F1F90290B6
:105DF00003910098019906F05FFF009001910298CD
:105E0000039906F03BFF06F057FF02000B000098D5
:105E1000019907F04DFCFBF76DFD06F02FFF03C461
:105E2000B54203D10843431E9841D1E706F044FF31
:105E3000FBF782F80200751BC017E90FAA42484120
:105E4000C6E7C04600002440F0B5140097B00892A1
:105E500009931D005A0063422343CB495208DB0FCC
:105E60001343CB1A0290C9490DD4C94BDA420ED460
:105E7000290000220023200005F03EFFC54900282C
:105E800000D1C5490298FDF773FC17B0F0BD0022A0
:105E900000232000290005F01BFF002800D129E184
:105EA000BE4B1B780894043B1A00531E9A41802372
:105EB0001B06EB1809931C9B0792013B1C931C9A31
:105EC0000BA908A8FFF79AFE089E099F3000390029
:105ED00006F0D4FE04900591049B059C1800210057
:105EE0000E930F9406F0E8FE0D000400FBF724F873
:105EF00003000133220039000690019330002B008B
:105F000008F0E0FA049B059A06000F00134300D145
:105F1000F2E00F23019A9B1A0393039808F068FF9D
:105F200002000B0000209E49FFF752F902000B000F
:105F300004000D003000390007F0FCFFFBF7DAFC2D
:105F400006F09CFE0C900D9106F0B6FE22002B0090
:105F500005F0DCFE002827D00022002301200021CC
:105F60000C920D93049A059B12184B4119001000D6
:105F70000E900F9106F0A0FEFAF7DEFF019B0B9C3E
:105F8000984211DB002C00D1B8E0069808F030FFF1
:105F900002000B0000208249FFF71AF906F06EFE9E
:105FA0000E900F9101340B9400230B9F9F4207D05A
:105FB000380008F01DFFFAF7BFFFFB0F1B18023374
:105FC000784A1678754A1278032A00D09AE0019A26
:105FD0000199B21AB14200DC0F260399002900D1C1
:105FE00092E00D00914200DD15001C9AD31A019A2F
:105FF00004939C1AAC4200DD2C00E343DB171C40E9
:10600000039B9C421ADA19001A1B0CA8FFF7D4FE56
:10601000002812D00E980F99002200230C920D93A5
:1060200000230122801859410E900F9106F044FE82
:10603000FAF782FF019B984269DA2500049C002C44
:1060400000DC0124019BA34277DD1C1B2200190008
:106050000EA8FFF7B1FE002809D00E980F990B2368
:1060600064220B93002305F05BFE0E900F910B9BB7
:106070001B190B931422002111A800F03FFC2A00E9
:10608000494911A8FDF774FB079B012B08D1029821
:10609000FCF7ECFA029B2D2244491818FDF768FB27
:1060A0000298FCF7E3FA0E9A0F9B029C40492018D5
:1060B000FDF75EFB002D00DC89E00298FCF7D6FAC4
:1060C0000C9A0D9B0299081811A9FDF751FB0B9C26
:1060D000002C00D1D9E6314B02981B78042B00D05C
:1060E00082E0FCF7C3FA2E22029B30491818FDF714
:1060F0003FFBCAE60790E2E610230BE7069B02335C
:10610000019351E7320067E701256D426DE7019B7E
:10611000002F0FD0581E08F06BFE02000B0000206D
:106120001F49FFF755F806F0A9FD01370E900F91B2
:106130000B9782E7013301937FE7019BB34299DD1F
:106140000B9B0393019B9C1B200008F051FE020057
:106150000B0000201249FFF73BF8019B06000F00DF
:106160002200022B26DC19000EA8FFF725FE0E9850
:106170000F9906F0A1FD32003B0007F0DBFE06F0B0
:106180007DFD0E900F9175E70000F07F11EF00008C
:106190000000108016EF000015EF0000150C001035
:1061A00000002440160C00101AEF0000F3EF00006E
:1061B00024EF000001990EA8FFF7FEFD0028D6D0BD
:1061C000002301220E920F93039B033351E7002D0E
:1061D00000D07CE70298FCF749FA029B2E22064980
:1061E0001818FDF7C5FA72E7FCF740FA029B220087
:1061F000024918187BE7C046F3EF000029EF0000C2
:1062000082B0F0B593B019931C9B1892023BDA0F41
:10621000D3185B101622002103900CA8029300F003
:106220006DFB1622002106A800F068FB1899199A48
:106230001A9C1B9D394B69261B78394F0491059296
:10624000002B21D01898199922002B00FBF7CEFBC8
:10625000189A199B0490059120002900FEF738FA3E
:106260003B007E377F331A783B7804000D001343E0
:1062700038D100222B4B07F05DFE2B4A2B4B07F049
:1062800017FA04000D004B3E029B0CA80093049AE1
:10629000059BFFF7D9FD0CA8FCF7E8F9029B984293
:1062A00002D25B001B1A0293029B06AF22000093EE
:1062B00038002B00FFF7C8FD1D4A194B12781D4905
:1062C000042A04D080331B78002B19D01A493300DC
:1062D000009703980CAAFDF74BFA13B0F0BC08BC6A
:1062E00002B018471E26002ACED00022134B07F01A
:1062F00021FE0D4A0D4B07F0DBF904000D00C3E74A
:10630000290000220023200005F0F6FC0C4900289B
:1063100000D10C493B000096DBE7C046F00B0010B3
:10632000700B001000807640182D4454FB2119405A
:10633000150C00102EEF000035EF00000000794032
:106340003EEF000048EF0000F0B50400012685B0E4
:106350002000FCF78BF9237807002D2B06D00025B1
:106360002800BD4205DB704305B0F0BD0134764224
:10637000EEE708F03DFD00900191605D303808F0D7
:1063800037FD02900391781E401B08F031FD02009A
:106390000B0000200849FEF71BFF02000B000298CB
:1063A000039907F0C7FD009A019B06F067FD08F00E
:1063B000E3FC0135D5E7C0460000244070B50E4D22
:1063C000FE232C78492C0FD00C48FCF75FFDFF23EF
:1063D000002809D00A48FCF759FDFD23002803D006
:1063E000402C03D923002333180070BD2800FFF789
:1063F000ABFF0300F8E7C04680010010F0EE00009C
:1064000051EF0000F0B5040087B0FCF72FF92378B6
:1064100003902D2B25D1601CFFF7F4FF80231B0672
:10642000C91807B0F0BDE25C2E2A16D0452A16D056
:106430000133039A9342F6DB8D4202D1AE4215D06E
:1064400035006B4200220293002300270092019343
:10645000039B9F420CDB002010E01D00E8E71E00BC
:10646000E6E72B4D00232E002900E2E7039DE8E735
:10647000BE4210D10136A019FFF766FF08F0B8FC44
:1064800002000B0000202349FEF7A2FE009A019BA8
:1064900007F050FDC5E7BD4222DDE05D303808F071
:1064A000A7FC029B04900591D84308F0A1FC0200D0
:1064B0000B0000201749FEF78BFE02000B0004982A
:1064C000059907F037FD02000B000098019906F0CE
:1064D000D5FC00900191029B013701330293B7E78D
:1064E000BD42F8DAE05D303808F082FC0490059196
:1064F000029808F07DFC02000B0000200549FEF721
:1065000067FE02000B000498059907F0D1F8DAE75E
:10651000E70300000000244082B0F0B587B00C9281
:106520000D9303900E9A0F9B0C980D99FBF75EFA52
:106530000022002304000D0005F0C4FB002800D059
:106540007CE00C9A0D9B0E980F99FEF7C1F8109AFB
:10655000119B0490059120002900FEF739FE3A4A6C
:106560000090019104980599384B07F0A1F8109A12
:10657000119B07F0DFFC002206000F001298139910
:10658000002305F09FFB002827D18022129B1206D2
:106590001800139B9918049A059B07F0CBFCFBF796
:1065A0004BF802000B000098019907F0C3FC009023
:1065B000019120002900FAF765FE129A139B07F05B
:1065C000B9FC214A214B07F073F802000B003000A0
:1065D000390006F053FC06000F0030003900FAF7CE
:1065E00023FD009A019B07F0A5FC32003B0004004C
:1065F0000D000020164907F065FFFAF715FD0200AF
:106600000B000098019907F095FC002206000F008E
:1066100000232000290007F08DFC02000B00300051
:10662000390006F02BFC039B1860596018009C6031
:10663000DD6007B0F0BC08BC02B0184700200021A4
:1066400004000D00EFE7C046182D4454FB2109401B
:106650000000E03F82B0F0B597B01C921D930D9002
:1066600000221E981F991C9C1D9D002305F02AFBEB
:10667000002824D0002200232000290005F032FB4E
:1066800000281CD020002900FAF744F822002B0033
:1066900005F018FB00281AD00022002300209049A2
:1066A00007F006F8002200230D9C206061602000A6
:1066B000A260E36017B0F0BC08BC02B0184700222B
:1066C00020002900874B05F003FB002856D020004E
:1066D000854A864B290007F02DFC834A06000F00EF
:1066E0001E981F99814B07F025FC32003B00019159
:1066F000009012A8FEF736FD129A139B149E159F68
:1067000008920993002022002B00754907F0DAFE59
:10671000002200230692079380221F9B1E9C1206D4
:106720009B18019302000B00009412A80694FFF737
:1067300091FF14981599129A139B04900591029257
:106740000393089A099B12A80096019705F008FB8D
:10675000129A139B14981599029203930024002314
:1067600004900591009301945F4A604B12A805F0D4
:10677000B9FD12981399149A159B95E720002900EA
:10678000574B002207F09EFE002400230A930B942F
:106790000123534C06900791089309940124544D0A
:1067A000E3002000EB181E685F681E9A1F9B04928E
:1067B000059308F01DFB069A079B06F05FFB00227D
:1067C0000023029003910092019312A832003B0033
:1067D00005F088FD129A139B08980999149E159F3D
:1067E00006F04CFB3200089009910A980B993B0087
:1067F00006F044FB01340A900B910B2CD0D1069883
:10680000079900223B4B06F039FB0022354B06F07E
:1068100035FB04000D0034483749FAF783FA0022AB
:1068200006000F00069807992E4B06F027FB1E9ACC
:106830001F9B049205931F9B0290039101931E9B43
:1068400022000693009312A82B00FFF765FE149A0E
:10685000159B129813990E920F9332003B0007F08C
:1068600069FB32003B00109011910E980F9907F0D0
:1068700061FB002200230E920F9380231F9A1B06B8
:10688000D318019380230F00060006981B062200F0
:106890000090EB1812A80E94FDF784FB149815993C
:1068A000129A139B0490059102920393109A119BE4
:1068B00012A80096019705F053FA149815990A9CAE
:1068C0000B9D129A139B04940595089C099D0090BA
:1068D00001910294039512A805F042FA49E7C046D7
:1068E0000000F03F0000E03F182D4454FB21094018
:1068F00010F4000000002240FB211940030070B595
:10690000840714D1032A12D90C040B0623430B432A
:106910000C0223430400861808C4351B032DFBD842
:106920000324131F9B089B00C318043322409A18AA
:10693000934200D170BD19700133F9E710B51622EA
:1069400000210348FFF7DAFFFBF798FE10BDC046B1
:106950008001001070B50D4B0D4C1B78002B13D12E
:106960000C4D2800FBF782FE00280DD02800FFF711
:1069700049FD2300A8330022186059600023B03479
:1069800022606360FFF7DAFF70BDC0460C0C001098
:10699000700B00108001001070B5FFF7DBFF074B94
:1069A000074A1E00146855689068D168E836F033CD
:1069B000346075601860596070BDC046700B00107F
:1069C000180C0010F0B587B0FFF7E6FF0D4C0E4D28
:1069D00020686168A668E76802000B0002A80197BA
:1069E0000096FEF74BF802980399049A059B2060E5
:1069F00061602900B0310A604B600123A4352B701F
:106A000007B0F0BD180C0010700B0010F0B587B087
:106A1000FFF7C2FF0D4C0E4D20686168A668E7685D
:106A200002000B0002A801970096FDF7BBFA02983E
:106A30000399049A059B206061602900B0310A60C7
:106A40004B600123A4352B7007B0F0BD180C00106B
:106A5000700B0010F0B58BB0FFF79EFF154C164B76
:106A6000164D986ED96E1E6F5F6F22686368029232
:106A70000393A268E36800962E0004920593F8360B
:106A800002000B0006A80197FFF746FD069807993C
:106A9000089A099B30607160206061602900B03104
:106AA000B260F3600A604B600123A4352B700BB019
:106AB000F0BDC046180C001000F40000700B001070
:106AC000F0B58FB0FFF768FF184C194B2600186817
:106AD00059689A68DB68A836089209930794346865
:106AE000756802940395099B089AB468F568019348
:106AF000049405950B00009202000AA8FFF70CFD14
:106B00000A9C0B9D0C9E0D9F079B3200F8331C6066
:106B10005D609E60DF6020003B002900F9F71EFBEE
:106B20000122079BA4331A700FB0F0BD700B001048
:106B3000280C0010F0B5244B8DB00793234B1B7825
:106B4000DB0605D52F22224B0799CA540DB0F0BDA4
:106B5000FFF722FF079B0022A8331E685F689C682E
:106B6000DD6830000023390005F0ACF800280CD0B7
:106B7000002200232000290005F0A4F8002804D0FA
:106B8000079B873301221A70E0E7079BB833186828
:106B9000596804940595029603979A68DB680092F9
:106BA000019302000B0008A805F09CFB089C099DBE
:106BB0000A9E0B9F20003B0029003200F9F7CEFA15
:106BC000079BA433DEE7C046700B00100C0C0010CE
:106BD00072070000F0B58DB0FFF7DEFE574C584B42
:106BE00025001B78A8355BB22E686F68012B40D159
:106BF000AB68EC683000390006930794FEF7E0F9C3
:106C000004000D0006980799FDF780F902000B00BB
:106C10002000290007F08EF904000D003000390033
:106C2000FEF720F906000F0006980799FDF726F9F0
:106C300002000B003000390007F07CF9002206004A
:106C40000F0000232000290007F074F902000B0058
:106C50003000390006F012F9384B3A4A10605160A2
:106C60001A00B032146055600122A4331A700DB0BE
:106C7000F0BD013339D1AB68EC683200069307945C
:106C800004930594029603970093019408A83B008F
:106C900005F066F8089809990A9C0B9D00222A4B7A
:106CA00006F0ECF8019502000B00009408A8FDF72F
:106CB000E5FE089809990A9C0B9D32003B0006F0FE
:106CC000DDF8069A079B06000F002000290006F059
:106CD000D5F8320000903B00019108A8FDF79EFD19
:106CE000089809990A9C0B9DB6E7F9F7E9F901287C
:106CF0001AD023007E331B78002B06D030003900D9
:106D0000FDF704F900240025A6E77F34237800224C
:106D1000002B07D00D4B3000390006F0C9FCFAF704
:106D200083F9EFE70A4BF6E7A968EA683B000192AE
:106D30000091320008A8FEF715FAD1E7700B001099
:106D4000F40B0010180C00100000F03F0000694028
:106D500000806640F0B595B0FFF71EFE7A4C7B4B85
:106D600025001B78A8355BB22E686F68012B40D1D7
:106D7000AB68EC683000390006930794FEF772F8B0
:106D800004000D0006980799FDF7C0F802000B00FB
:106D90002000290007F0CEF804000D003000390073
:106DA000FEF70EF906000F0006980799FDF766F842
:106DB00002000B003000390007F0BCF8002206008A
:106DC0000F0000232000290007F0B4F802000B0098
:106DD0003000390006F052F85B4B5D4A106051609C
:106DE0001A00B032146055600122A4331A7015B035
:106DF000F0BD013354D1AB68EC68002206930794D0
:106E000030003900534B06F039F8079D069C02000C
:106E10000B00019500940CA8FDF730FE0C9A0D9B19
:106E200030003900089209930E9A0F9B0A920B9337
:106E30000022484B07F046FB019502000B0000942E
:106E40000CA8FDF71BFE0C9A0D9B0E980F99029251
:106E500003930A9B0B9C0490059100930194089A5C
:106E6000099B0CA804F07CFF0C980D990E9C0F9DBB
:106E700032003B0006F002F8069A079B06000F005E
:106E80002000290005F0FAFF3200019100903B003C
:106E90000CA8FDF7C3FC0C980D990E9C0F9D9BE769
:106EA000F9F70EF9012820D023007E331B78002B40
:106EB00006D030003900FCF7E1FF002400258BE705
:106EC0007F3423780022002B0DD0234B3000390073
:106ED00006F0EEFB02000B000020204907F0F2FA5A
:106EE000FAF7A2F8E9E71E4BF0E7A868E96812ABE9
:106EF00010AAFEF7F5F830003900FDF707F8129AEE
:106F0000139B07F017F80690079130003900FCF743
:106F1000B5FF109A119B07F00DF8002204000D0038
:106F200006980799002307F005F802000B002000DF
:106F3000290007F0C7FA802212069446069B1C001F
:106F4000079B63441D0047E7700B0010F40B001013
:106F5000180C00100000F03F000069400000E03F06
:106F600000806640F0B5A1B0FFF716FD724E734B7E
:106F700037001B78A8375BB23C687D68012B42D193
:106F8000BA68FB68200006920793290022002B00B4
:106F900005F074FF06000F00FEF712F8069A079B33
:106FA000089009911000190005F068FF04000D0019
:106FB000FCF764FF02000B000898099905F05EFFDA
:106FC0000690079120002900FCF7A0FF069A079B76
:106FD00006F06EFB04000D0030003900FDF742FFA3
:106FE000069A079B06F064FB002206000F000023B0
:106FF0002000290006F09EFF02000B00300039003F
:1070000005F03CFF33E001333ED100224C4B18A881
:10701000049205930022002302920393BA68FB684E
:107020000092019322002B0004F09AFE1A9C1B9DF3
:1070300018981999009400240195424D02000B0004
:1070400018A8FDF713FC1A981B99189A199B049419
:107050000595802500242D0600900191029403954A
:1070600018A804F07DFE189819991A9C1B9D324BA4
:10707000354A106051601A00B03214605560012228
:10708000A4331A7021B0F0BDF9F71AF8012867D0BF
:1070900033007E331B78002B2CD02C4A6B005B080E
:1070A000934208D8012300220093002320002900E6
:1070B000FCF7AEFF08E0264A934208D922002B00D5
:1070C0002000290007F0FEF900240025CFE71CAEC0
:1070D000320020002900FCF7EFFC1E9E1F9F1C9C25
:1070E0001D9D022243001340013AD31A009332003F
:1070F0003B00DBE77F3633780022002B19D0154B9D
:107100002000290006F0D4FA04000D00F9F78CFFE6
:1071100022002B0006000F0000200F4907F0D2F9D3
:10712000F9F782FF02000B003000390006F0C0FAC8
:10713000CAE70A4BE4E7C046700B0010F40B0010DE
:107140000000F03F0000F0BF180C0010FB21E93FE9
:10715000FFFFEF7F000069400000E03F00806640D5
:107160002200BE68FF682B002000290005F086FE83
:1071700006900791FCF782FE32003B0004000D00F0
:107180003000390005F07AFE08900991FDF718FFEC
:1071900002000B002000290005F070FE06000F0021
:1071A000FCF786FC0022944B04F092FD002800D1ED
:1071B000F7E006980799FCF77BFC0A900B9108987A
:1071C0000999FCF775FC8D4A0C900D910A980B9962
:1071D0008B4B06F06DFA0022002304000D0004F032
:1071E00095FD0022874B002800D1EFE02000290008
:1071F00005F044FE07F0C0FD07F0FAFDA822804B21
:10720000D20506000F0006F095FE02000B000A985A
:107210000B9907F057F9802204000D003000390067
:10722000794B520506F086FE02000B002000290073
:1072300007F048F9754A04000D0030003900744B1E
:1072400006F078FE02000B002000290007F03AF952
:1072500002000B0006F06EFE0C9A0D9B0026002724
:10726000109011911000190006F064FE0022340005
:107270003D00684B129013910E920F930C920D9358
:107280000A920B93002220002900624B05F0F6FDC4
:107290000A9A0B9B04000D0006F04CFE00220A9097
:1072A0000B915C4B2000290005F0E8FD04000D0067
:1072B00002000B000A980B9906F03CFE0C9A0D9BFD
:1072C0000A900B911098119906F034FE0E9A0F9BBC
:1072D0000C900D911298139906F02CFE02000B00F1
:1072E0000E900F910C980D9905F0C8FD0A9A0B9B12
:1072F00006F0DEF932003B0005F0C0FD00221690DA
:107300001791444B2000290005F0B8FD04000D0042
:1073100002000B000A980B9906F00CFE00220600F2
:107320000F00200029003B4B05F0A8FD02000B00D8
:1073300004000D003000390006F0FCFD0C9A0D9B96
:107340000A900B911098119906F0F4FD0E9A0F9B7C
:107350000C900D911298139906F0ECFD0C9A0D9B70
:107360000E900F9107F0AEF80A9A0B9B06F0A0F969
:1073700002000B00149015911698179905F07EFDE8
:1073800002000B0006000F001498159906F090F902
:10739000FCF78EFB204A214B04F0AEFC002800D005
:1073A00070E7002200233000390004F08BFC002835
:1073B00011D000221A4B0020002106F0BBFD002254
:1073C000174B05F05BFD0024154D50E62000290009
:1073D00007F078F80EE708980999FDF743FD3200A9
:1073E0003B0006F065F904000D0006980799FCF7CC
:1073F0008DFD32003B00F5E50000D03F182D4454D0
:10740000FB2109400000E03F460B213E6EC04531A4
:1074100063626A3C0000F03F4F64A14091B49F3C1E
:107420000000F07FF0B5194B194C1B788DB0DB06CE
:1074300004D52A22174BE2540DB0F0BD25002600DA
:10744000B835A836FFF7A8FAB068F1682A686B6803
:10745000049005913068716802900391A868E9680A
:107460000090019108A804F07BFC0A9A0B9B089EEF
:10747000099F06920793069A079B30003900F8F798
:107480006DFE0123A4342370D6E7C0460C0C001017
:10749000700B001072070000F7B5144B144C1B78EA
:1074A000DB0603D52D22134BE254F7BD2500260041
:1074B000B835A836FFF770FA3268736828686968CB
:1074C00007F000F8B268F36800900191A868E968D5
:1074D00006F0F8FF06000F00009801993B0032000B
:1074E000F8F73CFE0123A4342370DEE70C0C0010F7
:1074F000700B001072070000F0B587B0F8F7E0FDE0
:107500003B4C0390002804D002238734237007B03B
:10751000F0BDFFF741FA3749002208684968364B49
:1075200005F0ACFC250002000B0004900591210041
:10753000F8352A636B633931304BFF311A685B6869
:10754000086849680092019305F098FC009A019B35
:107550002600286469641000190006F0EBFC493627
:10756000FF3602000B003068716805F087FC286563
:107570006965210023005931B833FF311E685F6807
:107580000868496832003B0005F078FC3200286644
:1075900069663B003000390006F0CCFC0B0018494E
:1075A00002000868496805F069FC28676967009867
:1075B0000199250032003B0006F0BCFC7935FF350F
:1075C00002000B002868696805F058FC094B286028
:1075D00069609868D968049A059B084D2A606B60B9
:1075E0002300B03318605960A434039B8EE7C04673
:1075F000700B0010980C00100000F03F180C0010E9
:10760000D80C0010F7B5144B144C1B78DB0603D5CF
:107610002B22134BE254F7BD25002600B835A836BF
:10762000FFF7BAF9326873682868696805F026FCC4
:10763000B268F36800900191A868E96805F01EFC43
:1076400006000F00009801993B003200F8F786FD14
:107650000123A4342370DEE70C0C0010700B001023
:1076600072070000F0B585B0F8F72AFD3E4C0128FE
:1076700004D102238734237005B0F0BDA834FFF78E
:107680008BF96568246820002900F9F7CFF802001B
:107690000B00009001912000290006F013FF00224A
:1076A000324B06F047FC0F00060007F065FB0400B4
:1076B00007F09EFB02000B003000390006F002FFCD
:1076C00000222A4B06F036FC0022294B06F032FC41
:1076D000FAF710F90022264B05F0EAFF0022234BAF
:1076E00006000F0004F012FB002808D0300039001B
:1076F00000221E4B06F0E6FE06000F0001343B2C74
:1077000008DD0098019900221A4B05F0B7FB0090A4
:1077100001913C3C6420184B6043039307F068FBE5
:10772000002204000D0000980199144B06F002FCA1
:1077300002000B002000290005F0A0FB32003B00F6
:1077400005F09CFB00220D4B05F0B2FF039B186077
:107750005960054B00201A000021B03210605160C2
:107760000122A4331A7087E7700B001000004E400E
:1077700080842E410000F03F180C00100088C340A8
:10778000F8B5F8F79DFC194C012803D10223873482
:107790002370F8BD2500A835FFF7FEF8A868E96852
:1077A0000022134B05F084FF02000B0005F066FB7E
:1077B000104A114B06F0BEFB002206000F0028689D
:1077C00069680B4B05F074FF02000B0005F056FBD7
:1077D000094B084A06F0AEFB2300B0331E605F6021
:1077E000286069600123A434D2E7C046700B001002
:1077F00000807640182D4454FB210940F0B587B035
:10780000FFF7CAF81A4D1B4CAE68EF6830002A68C3
:107810006B68390002920393F9F708F80090019120
:1078200002980399F9F702F8002204900591009854
:107830000199002306F07EFB049A059B05F01EFBD0
:1078400002000B000298039906F03CFE009A019B8F
:107850002860696025003000390006F033FE0123FE
:10786000B035A43428606960237007B0F0BDC0460D
:10787000180C0010700B0010F0B587B0FFF78CF8F3
:10788000F8F71EFC224B234C1E685F68012813D0BA
:10789000002230003900204B04F01AFA00280BD1E6
:1078A0003900300007F068FA07F0A2FA32003B0016
:1078B00004F008FA002821D100223000164B3900CC
:1078C00005F0DCFA2300A8339D68DE6802000B0097
:1078D00002A801960095FEF7BDFE02980399049A4E
:1078E000059B2500A835286069602100B0310A6039
:1078F0004B600123A434237007B0F0BD0022064B77
:1079000030003900F9F7D6FA00220023E9E7C04633
:10791000180C0010700B00100000F03FF0B591B093
:10792000FFF73AF8644B654A1E0011685268393314
:10793000FF335C681B680293039433005933FF33B1
:107940005C681B68049305943300793300910192BD
:1079500000980199FF331A685B6806F0EBFA049A05
:10796000059B04000D000298039906F0E3FA02005B
:107970000B002000290006F0A5FD33004933FF333A
:107980000A900B911A685B680098019906F0D2FA88
:10799000029A039B04000D001000190006F0CAFAB9
:1079A00002000B002000290006F08CFD3300693333
:1079B000FF33069007911A685B680098019906F0FA
:1079C000B9FA049A059B04000D001000190006F096
:1079D000B1FA370002000B002000290006F072FD0A
:1079E000A8373B687C6808930994BC68FD680C90D4
:1079F0000D910898099922002B00F8F79DFB304B58
:107A00009C6EDD6E1A6F5B6F0E920F930E9A0F9B3A
:107A100020002900F8F770FB0C9A0D9B0698079937
:107A200006F088FAF9F77EF9340002000B000A9894
:107A30000B9905F03DFEB8343300206061600022F0
:107A40000021C03319605A60089A099B0098019977
:107A500006F070FA029A039B06F034FD0A9A0B9B1B
:107A600006F068FA069A079B04000D000498059931
:107A700006F060FA02000B002000290005F0FEF974
:107A8000069A079B04000D000098019906F052FA2F
:107A900002000B002000290005F00AFE330000223E
:107AA000386079600021B03319605A6033000122D8
:107AB000A4331A7011B0F0BD700B0010980C0010B8
:107AC00080F20000D0B5F8F7FBFA134C002803D081
:107AD000022387342370D0BDFEF75EFF2300B83346
:107AE0001E685F682300A8331A685B68300039009D
:107AF00006F0E8FC0022094B05F0C0F902000B007B
:107B000030003900F9F7D6F900230022F8F726FBF8
:107B1000A4340123DEE7C046700B00100000F03FE4
:107B200030B58BB0FEF738FF0E4C0F4DA068E16802
:107B3000226863680490059100900191029203937A
:107B400006A804F00DF906980799089A099B206089
:107B500061602900B0310A604B600123A4352B70AD
:107B60000BB030BD180C0010700B0010F0B587B0D2
:107B7000FEF712FF0D4C0E4D20686168A668E7689D
:107B800002000B0002A801970096FCF747FE02983E
:107B90000399049A059B206061602900B0310A6056
:107BA0004B600123A4352B7007B0F0BD180C0010FA
:107BB000700B0010F0B58FB0FEF7EEFE204C214D9B
:107BC00020686168A668E76802000B0001970096CC
:107BD0000AA8FCF723FE0A9A0B9B0C9E0D9F0892A5
:107BE0000993194B986ED96E1A6F5B6F06920793C3
:107BF000079B069A019300920B0002000AA8FCF76B
:107C00000DFE0C980D990A9A0B9B04900591029217
:107C10000393089A099B0AA80096019704F062FB57
:107C20000A980B990C9A0D9B206061602900B03175
:107C30000A604B600123A4352B700FB0F0BDC04625
:107C4000180C0010700B001000F4000070B5F8F76D
:107C500037FA114C002803D002238734237070BDFB
:107C6000FEF79AFE25002100A835B8312A686B6816
:107C70000868496806F05EF9084B002205F018FD17
:107C800023002860696000200021B033186059602B
:107C9000A4340123E2E7C046700B001000005940F5
:107CA000F8B5F8F70DFA144C002803D002238734F6
:107CB0002370F8BDFEF770FE25002300A835B83309
:107CC0001E685F682868696832003B0006F0FAFBAE
:107CD00000220A4B06F02EF93B00320005F0E8FCCA
:107CE00023002860696000200021B03318605960CB
:107CF000A4340123DCE7C046700B0010000059409B
:107D000070B5FEF749FE0A4D0A4CAA68EB68286870
:107D10006968F9F76BFE2200286069600020002185
:107D20002300B032106051600122A4331A7070BD7C
:107D3000180C0010700B0010F0B589B0FEF72CFE87
:107D4000F8F7D6FA154D164C2F00A268E368029298
:107D50000393039B029A06002068616801930092D6
:107D60000B00020004A8FCF7D5FF04980599069AB9
:107D7000079BB03720606160002E06D13A607B60BF
:107D80000123A4352B7009B0F0BD002200233A6016
:107D90007B60F8F79DFC20606160F1E7700B0010DC
:107DA000180C0010F0B58BB0FEF7F6FDF8F7A0FA4E
:107DB000214D224BAE68EF680390029328686968F2
:107DC000019702000B00009606A8FCF7A3FF069A95
:107DD000079B089E099F1A481A4906F073FB002268
:107DE0000490059100233000390006F0A3F80B0041
:107DF00002000498059906F065FB029C039B28602D
:107E00006960B034002B0DD132003B00002000210E
:107E100006F058FB206061600123029EA436337097
:107E20000BB0F0BD0022002322606360F8F750FC25
:107E300028606960F0E7C046180C0010700B001055
:107E4000182D4454FB21F93FF0B589B0FEF7A4FD8D
:107E5000154C164B20686168A568E668020003931C
:107E600001960B00009504A8FCF700FD049E059FF9
:107E7000069A079B039D26606760B0352A606B6099
:107E8000F8F71EF9012809D030003900F8F720FC76
:107E900000220023206061602A606B600122039B46
:107EA000A4331A7009B0F0BD180C0010700B00104C
:107EB00010B5074B074C1B78002B04D18534227872
:107EC000002A01D0237010BDFEF766FD0123F9E7FB
:107ED000F60B0010700B0010F0B58DB0FEF75CFDD6
:107EE000454D464B2E00186859689A68DB68089221
:107EF000099302230A900B91A53634780F2207A923
:107F00000AA83370FDF77AFE0F2206A908A8FDF72C
:107F100075FEA6353470287806F098FF02000B0035
:107F200000203749FDF754F904F0A8FE032C03D1D3
:107F30000A22002303F0F4FE04F0BEFE0A9A0B9B13
:107F400004000D0005F0F6FFF9F7D4FC22002B0029
:107F500005F0AEFB089A099B06000F0020002900DF
:107F600005F0E8FFF9F7C6FC22002B0005F0A0FBA6
:107F700000900191079806F03BFF02000B000020E3
:107F80001F49FDF725F902000B003000390005F00C
:107F9000D1FF00220023029003910098019905F07F
:107FA000C9FF04900591069806F022FF02000B001D
:107FB00000201349FDF70CF906000F0002000B002A
:107FC0000498059905F0B6FF029A039B04F056FF4A
:107FD000094C0A4D3B002860696000980199250012
:107FE000320005F0A7FF0123B035A4342860696092
:107FF00023700DB0F0BDC046700B0010180C0010BF
:1080000000002440F0B587B0F8F75AF8364F012841
:1080100004D1022287373A7007B0F0BD3E00A8367F
:10802000FEF7BAFC3468756820002900F8F7FEFBFB
:1080300002000B00009001912000290006F042FA96
:1080400000222A4B05F076FF0022294B05F072FF33
:10805000F9F750FC0022264B05F02AFB3B000400F8
:108060000D0000200021B033186059602900200065
:1080700006F082FE06F0BCFE02000B0002900391A7
:108080002000290006F01EFA0022184B05F052FFCE
:10809000184A194B049005910298039905F04AFF7C
:1080A000F9F728FC154A164B04000D0004980599B1
:1080B00005F040FFF9F71EFC02000B00200029002C
:1080C00004F0DCFE00220F4B05F0F2FA00220E4B0A
:1080D00005F0EEFA009A019B04F0D0FE0123A437CC
:1080E000306071603B7097E7700B001000005940E2
:1080F00084D797415555555543DEA341E4388EE367
:108100005831454180842E410088C34070B5F7F74F
:10811000D7FF104C012803D102238734237070BD90
:108120002500A835FEF738FC2868696800220A4B4C
:1081300005F000FF094B0A4A05F0BAFA230028604F
:10814000696000200021B03318605960A434012315
:10815000E4E7C046700B001000807640FB21194018
:10816000182D4454F7B5FEF717FC134D134CA868AF
:10817000E968F8F75BFB2E686F68009001913000AA
:108180003900F8F753FB06000F0000980199002210
:10819000002305F0CFFE32003B0004F06FFE230009
:1081A000B033286069600099019A19605A60012310
:1081B000A4342370F7BDC046180C0010700B0010DB
:1081C000F0B587B0F7F77CFF3B4C0390002804D054
:1081D00002238734237007B0F0BDFEF7DDFB37497B
:1081E000002208684968364B06F06CF92500020049
:1081F0000B00049005912100F8352A636B63393137
:10820000304BFF311A685B68086849680092019337
:1082100006F058F9009A019B260028646964100052
:10822000190005F087FE4936FF3602000B00306862
:10823000716806F047F92865696521002300593106
:10824000B833FF311E685F680868496832003B0038
:1082500006F038F93200286669663B0030003900C4
:1082600005F068FE0B00184902000868496806F02E
:1082700029F92867696700980199250032003B00B9
:1082800005F058FE7935FF3502000B002868696853
:1082900006F018F9094B286069609868D968049A53
:1082A000059B084D2A606B602300B033186059604D
:1082B000A434039B8EE7C046700B0010980C00108E
:1082C0000000F03F180C0010D80C0010F0B585B07D
:1082D000F7F7F6FE294E002804D0022387363370C4
:1082E00005B0F0BDFEF758FB3300A836B833776809
:1082F00036681C685D6832003B002000290006F0EB
:10830000E1F802000B00009001913900300003F009
:10831000E9FC01004A1E9141030003910098019974
:10832000002B01D1300039000022154B04F0A6FDCE
:108330000B00020029002000F8F7BCFD039B04009D
:108340000D0000980199002B01D030003900002267
:108350000B4BF8F7AFFD02000B002000290005F0E1
:10836000A7F904000D000022002320002900F7F7E0
:10837000F5FE0122034B1A70B2E7C046700B0010E5
:108380000000F03F140C0010F0B5294A294C137876
:108390008DB0002B07D0012B03D10B3313700DB020
:1083A000F0BD013BFAE7FEF7D5FA2300A8331968C0
:1083B0005A68069107929E68DF680698079900221E
:1083C000002303F07FFC00280BD0002200233000A4
:1083D000390003F077FC002803D087340123237091
:1083E000DDE723000699079AE83319605A602300F5
:1083F000F0331E605F6013000A00250002920393B1
:108400000022002308A800920193049605970022F9
:10841000094BA83503F066FF089A099B0A980B9947
:108420002A606B602300B03318605960A434D5E72C
:10843000F30B0010700B00100000F03FF7B5FEF7D3
:1084400089FA1548154904008A68CB680500086850
:108450004968F834A260E3602B00B8331E685F6897
:10846000206061609A68DB6830002E000092019302
:10847000009A019B3900D836F7F770FE22686368CE
:10848000A068E168326073602B00E03318605960C7
:108490000123A4352B70F7BD700B0010180C0010D1
:1084A000F0B585B0FEF756FA174E184B370018682E
:1084B00059689C46DC689B6800930194009A019B74
:1084C0003400F834A260E3606346B837206061602E
:1084D000BC68FD68029403953C687D6838607960EB
:1084E0001C605D60029A039B34003100B034C031DF
:1084F00022606360009B019C0B604C600123A436EA
:10850000337005B0F0BDC046700B0010180C0010A1
:10851000F8B5FEF71FFA0D4F00223C687D68002376
:108520002900200005F006FD094E02000B00B86886
:10853000F96804F0A3FC32003300B03214605560D7
:108540000122A433386079601A70F8BD180C00104D
:10855000700B0010F0B587B0FEF7FCF9494B4A4AA2
:1085600002934A4B146855681E685F68029B039229
:108570007933FF331A685B682000290005F0DAFCC4
:10858000434B009001911A685B683000390005F098
:10859000D1FC02000B000098019905F093FF029BAB
:1085A000049005914933FF331A685B682000290065
:1085B00005F0C0FC320004000D003B003000390023
:1085C00005F0B8FC02000B002000290005F07AFF3E
:1085D000304B009001911C685D689E68DF68200048
:1085E000290032003B00F7F7A7FD2B4B9C6EDD6E98
:1085F0001E6F5F6F32003B0000260027200029001D
:10860000F7F77AFD009A019B0498059905F050F858
:10861000029B029CC0331E605F601D4BB8341A6819
:108620005B68206061600098019905F083FC174B3E
:1086300004001A685B680D000498059905F07AFC3F
:1086400002000B002000290005F03CFF039B040002
:108650001A685B680D000098019905F06BFC020038
:108660000B002000290005F023F80122094B1860B7
:108670005960029BB0331E605F60029BA4331A7086
:1086800007B0F0BD700B0010980C0010A80C001083
:10869000C80C0010180C001080F20000F7B5FEF7AF
:1086A00059F90E4D0E4CAA68EB68009201932E68A2
:1086B0006F68009A019B30003900F7F73DFD094AC9
:1086C000094B00202A606B6023000021B033186042
:1086D00059600123A4342370F7BDC046180C001064
:1086E000700B0010182D4454FB210940F8B5FEF71B
:1086F00031F9084B1C685D689E68DF68290032000C
:108700003B002000F7F718FD0122034BA4331A7039
:10871000F8BDC046480C0010700B0010F7B5FEF70E
:1087200019F90F4D0F4CAA68EB68009201932E685F
:108730006F68009A019B30003900F7F7FDFC2100BB
:10874000E8318A68CB680868496828606960210058
:10875000B0310A604B600123A4342370F7BDC046DA
:10876000180C0010700B0010F0B585B0FEF7F2F891
:10877000224B1C685D689E68DF682000290032007B
:1087800001933B00F7F7D8FC1D4B9C6EDD6E1E6F0E
:108790005F6F2000290032003B00F7F7ADFC194C59
:1087A00000262300210029335931FF33FF311A6895
:1087B0005B682500086849680292039304F078FF1B
:1087C000B835286069602100230000273931C033A3
:1087D000FF311E605F6008684968029A039B04F0DD
:1087E00067FF019B186059602300B0331E605F6013
:1087F0000123A434237005B0F0BDC046180C00104E
:1088000080F20000700B0010F0B58DB0FEF7A2F8FA
:10881000454B1C685D689E68DF68200029003200B7
:1088200003933B00F7F788FC404B9C6EDD6E1E6F98
:108830005F6F2000290032003B00F7F75DFC3C4CE5
:1088400023002933FF331A685B6800920193009874
:10885000019923003933FF331A685B68049205934A
:1088600023004933FF331A685B6808920993230099
:108870005933FF331E685F6800222E4B05F022FE3D
:10888000009A019B05F056FB23006933FF331A68F9
:108890005B68069007910098019905F04BFB320048
:1088A0000A900B913B003000390005F043FB0200B9
:1088B0000B000A980B9905F005FE069A079B04F039
:1088C000F7FEF8F72FFA2300B833186059600098C4
:1088D0000199230000260027C0331E605F60089ABC
:1088E000099B05F027FB049A059B0090019110005D
:1088F000190005F01FFB02000B000098019905F01C
:10890000E1FD069A079B04F0D3FEF8F70BFA039BF0
:10891000186059602300B0331E605F600123A434E7
:1089200023700DB0F0BDC046180C001080F200009E
:10893000700B00100000F03F012270B5164B174C71
:108940001A70230086331B780500002B0ED07C3470
:10895000FEF700F8124B22889B185878FAF77EFE33
:10896000040020000F49FAF72BFE10E023009C338F
:108970001B78002B0DD0FDF721FD85342378C0B284
:10898000002BEBD001002800F7F754FE064C200026
:1089900070BD054CE5E7C046140C0010700B0010CC
:1089A0009C030010680C0010FFFFFF7FF0B57920DA
:1089B00085B0FFF7C1FF039064281ADC0E4C0F4D01
:1089C000206861682A686B6804F058FAAA68EB6846
:1089D00006000F00A068E16804F050FA26606760A6
:1089E000A060E160320000903B0003980191FAF72B
:1089F0006DFF05B0F0BDC046680C0010180C0010EB
:108A0000F0B57A2085B0FFF797FF039064281ADC51
:108A10000E4C0F4D206861682A686B6805F052FDA6
:108A2000AA68EB6806000F00A068E16805F04AFD3F
:108A300026606760A060E160320000903B00039810
:108A40000191FAF743FF05B0F0BDC046680C001075
:108A5000180C0010F0B57B208BB0FFF76DFF050000
:108A6000642821DC114C124E22686368B068F168FA
:108A7000049005913068716802900391A068E168E4
:108A80000090019106A803F06BF906980799089EDB
:108A9000099F020020606160A660E7600B0028006B
:108AA00001970096FAF712FF0BB0F0BD680C0010AA
:108AB000180C0010F0B57C208BB0FFF73DFF0500CF
:108AC000642821DC114C124E22686368B068F1689A
:108AD000049005913068716802900391A068E16884
:108AE0000090019106A803F0FDFB06980799089EE7
:108AF000099F020020606160A660E7600B0028000B
:108B000001970096FAF7E2FE0BB0F0BD680C00107A
:108B1000180C001073B57D20FFF70EFF642818DCD9
:108B20000C4C0D4D2600A868E968F836B268F36869
:108B300004F0A4F9326873680090019128686968AC
:108B400004F09CF9009A019BB034286069602260AF
:108B5000636073BD700B0010180C001073B57E209D
:108B6000FFF7EAFE642818DC0C4C0D4D2600A868BF
:108B7000E968F836B268F36805F0A4FC32687368F7
:108B8000009001912868696805F09CFC009A019B9F
:108B9000B034286069602260636073BD700B0010A0
:108BA000180C001070B57F208AB0FFF7C5FE64284E
:108BB0001DDC104C104D26002A686B68F836B06832
:108BC000F168049005913068716802900391B034A7
:108BD000A868E9680090019106A803F0C1F8069A18
:108BE000079B089809992A606B60206061600AB051
:108BF00070BDC046700B0010180C001070B58020BE
:108C00008AB0FFF799FE64281DDC104C104D260039
:108C10002A686B68F836B068F1680490059130688E
:108C2000716802900391B034A868E96800900191DE
:108C300006A803F057FB069A079B089809992A6033
:108C40006B60206061600AB070BDC046700B0010A0
:108C5000180C001010B5FDF771FE00200021064B26
:108C6000064A106051601A00B03210605160002254
:108C7000A4331A7010BDC046700B0010180C001001
:108C80000F2270B50D4B0E4E0E4C30001A700021A5
:108C90000532FDF733FE230000259C331D700A4B7F
:108CA00030000A4A0A49E554FAF762FD230083348A
:108CB000A0331D602570FDF741FE70BDE80B00106C
:108CC000F80B0010700B001072070000000000107D
:108CD0000EEF000070B5164C164E2368164DB342C9
:108CE00011D1FDF76BFB061E00D10136F7F74AFCE8
:108CF0000400B04200DD34002000F7F7A5FB7C350E
:108D000024182C8070BDFFF7BBFFF7F73BFC06F083
:108D10006FF8F8F711F92B00013078331870074914
:108D20000748FAF725FD01239C3526602B70E9E7FB
:108D3000100C0010D58C0000700B001055EF0000D7
:108D4000F80B001070B5114D114E2B68114CB34249
:108D50000DD1FDF733FBC0B2F7F730FB002803D18C
:108D600004238734237001E07C34208070BDFFF73A
:108D700087FF230002227833074908481A709C3481
:108D8000FAF7F6FC09232E60ECE7C046100C001041
:108D9000458D0000700B001061EF0000F80B001013
:108DA00070B5FDF7D7FD234D234C2B78002B0AD04F
:108DB00085342378002B05D0FDF700FBC1B20720D6
:108DC000F7F738FC70BD230086331B78002B19D0D1
:108DD000230001222500A4331A707C35174B2A8802
:108DE0009B185878F7F7EAFA002807D123000422E5
:108DF00087331A700123A4342370E3E72880F7F740
:108E00007BFBF7E7230085331B78002B0FD0FFF7A0
:108E100037FF0C232B702300094AA0331A6002236A
:108E20007834084908482370FAF7A2FCCAE7FFF72C
:108E300089FFC7E70C0C0010700B00109C0300109A
:108E4000A18D00006CEF0000F80B001010B5224857
:108E5000FAF71CF8002802D1FDF770FD10BD1F4C79
:108E60002000F9F703FC00280BD00023201801385C
:108E700003702000F9F7FAFB0028EFD1184B1870A7
:108E8000ECE7184A184B1278002A02D0FFF7F8FED8
:108E9000E4E71A0085321278002A1AD07C331C8845
:108EA000002CDBD0114B185DF7F7A6FA002802D092
:108EB000A01C022107E02000F7F7C6FA01210300F9
:108EC000601C002BF5D14942F7F780FBF7F714FB44
:108ED000C4E7FFF7BFFEC1E7F0EE0000800100101D
:108EE000140C00100C0C0010700B00109C030010F0
:108EF000F7B5214D214C2B78002B0CD0FDF75EFAF5
:108F0000230085331B78C0B2002B11D001000D2047
:108F1000F7F790FBF7BD230086331B78002B19D0A1
:108F2000FDF718FD22007C32154B12889B185878EB
:108F3000FAF794FB2300A8331E685F689968DA6823
:108F40003B00019200913200FAF7C0FC0123A434E7
:108F50002370DFE7FDF7FEFCFFF792FE56232B7030
:108F60002300084AA0331A600223783406490748D0
:108F70002370FAF7FDFBCDE70C0C0010700B00100E
:108F80009C030010F18E000075EF0000F80B00103C
:108F9000F7B52D4D2D4C2B78002B23D0FDF70EFA75
:108FA000230085331B78C5B2002B04D02900112083
:108FB000F7F740FBF7BD264B9E6EDF6E1A6F5B6FB7
:108FC00000920193009A019B39003000F7F7B4F842
:108FD0002800FAF743FB1F49FAF7F2FA0123A434F9
:108FE0002370E7E7230086331B78002B1AD0FDF7A8
:108FF000B1FC22007C321288174B9B185878FAF784
:109000002DFB0500124B9E6EDF6E1A6F5B6F009298
:109010000193009A019B30003900F7F78DF8280082
:109020000C49D9E7FDF796FCFFF72AFE56232B7073
:1090300023000A4AA0331A600223783408490948F9
:109040002370FAF795FBB5E70C0C0010700B0010BD
:1090500080F20000180C00109C030010918F00009B
:1090600079EF0000F80B001070B51C4D1C4C2B78EC
:10907000002B0CD0FDF7A2F9230085331B78C0B27A
:10908000002B0FD001004420F7F7D4FA70BD230065
:1090900086331B78002B0ED022007C32114B1288B5
:1090A0009B185878FAF716FB2300A6331870012393
:1090B000A5342370EAE7FDF74DFCFFF7E1FD23003F
:1090C00002227833084909481A70FAF751FB084B15
:1090D000A034236005232B70D8E7C0460C0C001089
:1090E000700B00109C0300107DEF0000F80B0010C7
:1090F0006990000070B51C4D1C4C2B78002B0CD0D7
:10910000FDF75CF9230085331B78C0B2002B0FD02C
:1091100001004820F7F78EFA70BD230086331B78D4
:10912000002B0ED022007C32114B12889B185878ED
:10913000FAF7D0FA2300A63318700223A53423705F
:10914000EAE7FDF707FCFFF79BFD230002227833D7
:10915000084909481A70FAF70BFB084BA034236042
:1091600005232B70D8E7C0460C0C0010700B0010C4
:109170009C03001081EF0000F80B0010F590000038
:1091800070B51D4D1D4C2B78002B0CD0FDF716F93A
:10919000230085331B78C0B2002B0FD001004C2078
:1091A000F7F748FA70BD230086331B78002B11D0E7
:1091B00022007C32124B12889B185878FAF78AFAF0
:1091C000002800DC01202300A63318700323A534F7
:1091D0002370E7E7FDF7BEFBFFF752FD23000222F5
:1091E0007833084908481A70FAF7C2FA074BA034D6
:1091F000236005232B70D5E70C0C0010700B0010BA
:109200009C03001085EF0000F80B00108191000016
:1092100070B5FDF79FFB214D214C2B78002B1BD007
:10922000FDF7CCF8C6B23000FAF738FA23008533E0
:109230001B780500002B04D031005020F7F7FAF915
:1092400070BDFFF71DFD002D02D0E8B202F02CF832
:109250000123A4342370F3E7230086331B78002B0B
:109260000BD022007C320F4B12889B185878FAF7EB
:1092700015FA0028ECD0C0B2E8E7FFF701FD09239A
:109280002B702300084AA0331A6002237834074960
:1092900007482370FAF76CFAD2E7C0460C0C0010AE
:1092A000700B00109C0300101192000089EF000069
:1092B000F80B0010F0B52C4D2C4C2B7885B0002B02
:1092C0000DD0FDF77BF8230085331B78C0B2002B4F
:1092D00012D001004320F7F7ADF905B0F0BD23002F
:1092E00086331B78002B2DD0FDF734FB22007C3217
:1092F0001F4B12889B185878FAF7B0F92700250001
:109300000600F835A837B868F968A860E9603A68D7
:109310007B68390030002A606B60FAF751F9AA685F
:10932000EB682868696802920393039B029A019391
:1093300000920B0002003000FAF7C8FA0123A434AF
:109340002370CAE7FDF706FBFFF79AFC07232B7093
:109350002300084AA0331A600223783406490748DC
:109360002370FAF705FAB8E70C0C0010700B001028
:109370009C030010B592000094EF0000F80B001061
:10938000F0B5324D324C2B7889B0002B0BD08534A0
:10939000FDF714F82378002B03D0C1B24720F7F76C
:1093A00049F909B0F0BD230086331B78002B3AD071
:1093B000FDF7D0FA22007C321288264B9B18587891
:1093C000FAF74CF905002D0165192F00224E0937D7
:1093D0003100FAF7F5F83068716807AB009305AA19
:1093E00006ABF8F7CDFA0798059EFF37BA68FB6819
:1093F000361A0292039305F0FBFC02000B0038685A
:10940000796805F05FF8029A039BF835AA61EB6171
:10941000069B286169619E4201DCF7F729F8012368
:10942000A4342370BDE7FDF795FAFFF729FC072365
:109430002B702300094AA0331A60022378340849AC
:1094400008482370FAF794F9ABE7C0460C0C0010FB
:10945000700B00109C030010680C0010819300003A
:1094600099EF0000F80B0010F0B5324D324C2B781C
:1094700089B0002B0BD08534FCF7A0FF2378002B9C
:1094800003D0C1B24B20F7F7D5F809B0F0BD2300E7
:1094900086331B78002B3AD0FDF75CFA22007C3231
:1094A0001288264B9B185878FAF7D8F805002D013A
:1094B00065192F00224E09373100FAF781F830681C
:1094C000716807AB009305AA06ABF8F759FA07983D
:1094D000059EFF37BA68FB6886190292039305F070
:1094E00087FC02000B003868796803F0C7FC029A19
:1094F000039BF835AA61EB61069B286169619E4276
:1095000001DDF6F7B5FF0123A4342370BDE7FDF7B5
:1095100021FAFFF7B5FB07232B702300094AA0337C
:109520001A6002237834084908482370FAF720F9B2
:10953000ABE7C0460C0C0010700B00109C03001031
:10954000680C0010699400009DEF0000F80B0010FB
:1095500070B5FDF7FFF9204D204C2B78002B1BD068
:10956000FCF72CFFC6B23000FAF798F823008533D9
:109570001B780500002B04D031004F20F7F75AF874
:1095800070BDFFF77DFB002D02D0280001F05EFFCB
:109590000123A4342370F3E7230086331B78002BC8
:1095A0000AD022007C320E4B12889B185878FAF7AA
:1095B00075F80028ECD0E9E7FFF762FB09232B7070
:1095C0002300084AA0331A6002237834064907486A
:1095D0002370FAF7CDF8D3E70C0C0010700B0010D5
:1095E0009C03001051950000A1EF0000F80B001043
:1095F000F8B5FDF7AFF91B4D1B4C2B78002B21D094
:10960000FCF7DCFEC0B2F6F7C1FEFA22D2009042AF
:109610000CDA03000226154D93420BD102211B1ACE
:1096200001334942C91AC018F6F7D0FF00237C3431
:109630002380F8BDE95C5629F0D05F1CB143EDD022
:109640003B00E9E7FFF71CFB08232B702300084AC7
:10965000A0331A6002237834064907482370FAF7CA
:1096600087F8E6E70C0C0010700B00109C0300104C
:10967000F1950000B0EF0000F80B001070B5FDF799
:1096800069F9204D204C2B78002B17D0FCF796FE63
:10969000230085331B78C0B2002B04D001006B205F
:1096A000F6F7C8FF70BDFAF727F8ED232018DB00A6
:1096B000C0180123A43403702370F3E7230086331A
:1096C0001B78002B0DD022007C32104B12889B1887
:1096D0005878FAF711F8230087331B78002BE4D071
:1096E000E0E7FFF7CDFA05232B702300084AA033EB
:1096F0001A6001237834074907482370FAF738F8CD
:10970000D0E7C0460C0C0010700B00109C0300103A
:109710007D960000BDEF0000F80B001070B5FDF75E
:1097200019F9224D224C2B78002B17D0FCF746FE5E
:10973000230085331D78C0B2002D04D001006F20B6
:10974000F6F778FF70BDF9F7D7FFED232018DB009F
:10975000C01805700123A4342370F3E72300863377
:109760001B78002B12D022007C32124B12889B18DF
:109770005878F9F7C1FF230087331B78002BE1D11C
:10978000ED222018D20080180370E3E7FFF778FA83
:1097900005232B702300084AA0331A600123783474
:1097A000064907482370F9F7E3FFCBE70C0C0010DC
:1097B000700B00109C0300101D970000C7EF000005
:1097C000F80B001070B5FDF7C5F81E4D1E4C2B7838
:1097D000002B0AD08534FCF7F1FD2378002B03D051
:1097E000C1B27320F6F726FF70BD230086331B78C5
:1097F000002B16D022007C32144B12889B1858780C
:10980000F9F77AFF230087331B78002BECD1ED2387
:109810002018DB00C0180378002BE5D1F6F728FEEE
:10982000E2E7FFF72DFA05232B702300084AA03347
:109830001A6001237834074907482370F9F798FF25
:10984000D2E7C0460C0C0010700B00109C030010F7
:10985000C5970000D3EF0000F80B0010F7B56A4E73
:109860006A4C3578002D14D085342378002B0FD026
:10987000674C2000F8F7FAFE012805D12000FCF71C
:1098800063FD0130C5B2357029007620F6F7D2FEAF
:10989000F7BD230086331B78002B00D19AE0FDF73B
:1098A00059F822007C325B4B12889B185D78F6F7E2
:1098B00007FC002809D00C2D03D8574BEB40DB07E1
:1098C00003D4022387342370E2E72300A8331E6801
:1098D0005F682300681EB8331A685B6800920193C2
:1098E0000B2819D802F0EAF8061B262D343B4E5DF2
:1098F000606366692100A83100228868C968002376
:1099000002F0E0F9002812D00022002330003900D4
:1099100002F0D8F900280AD0F6F7AAFD07E00022E5
:1099200000233000390002F0E7F90028F4D00123C9
:10993000A434C8E7002200233000390002F0C8F93F
:10994000F3E7002200233000390002F0DFF9ECE7F2
:10995000002200233000390002F0C4F9E5E72100BD
:109960002300A831B8339A68DB688868C96802F0B8
:10997000A9F90028D0D0009A019B3000390002F0EC
:10998000A1F9D2E721002300A831B8339A68DB6837
:109990008868C96802F096F90028C8D0009A019B2F
:1099A000B4E7009A019BBCE7009A019BC4E7009AC8
:1099B000019BC8E7009A019BCCE72100A831002257
:1099C0008868C968002302F07DF90028A4D000222D
:1099D0000023D2E7230085331B78002B00D157E703
:1099E000FFF74EF9220020219C3211702200012342
:1099F0000A49A0321160783409490A48337023704B
:109A0000F9F7B6FE44E7C046F30B0010700B0010E8
:109A1000800100109C030010C21000005D9800003F
:109A2000DFEF0000F80B0010F7B53F4B3F4C1D78FF
:109A3000002D65D03E4B3F481B783F4D002B0FD18A
:109A40002300A0331B68AB4202D03C4A934216D19C
:109A50003B4BE35C002B12D13A492830F9F788FEE2
:109A60002300A0331B68AB422AD1354BE05C2A3877
:109A700005280ED802F022F81C090D180D2023002D
:109A800083331B78002BEBD1F7BD23002E4AA03384
:109A90001A602300A0331B68873498472378002B73
:109AA0002BD0FCF74BFFEFE72300284AA033EFE76A
:109AB0002300274AA033EBE72300264AA033E7E739
:109AC0001E4A9342E5D11E4BE05C2A380528E0D8B7
:109AD00001F0EAFF0B03DF07DF0F23001E4AA0336C
:109AE000D6E723001D4AA033D2E723001C4AA03347
:109AF000CEE723001B4AA033CAE7FFF7C1F8C3E74C
:109B0000FCF728FF2300A8331E685F689A68DB68AB
:109B100000920193009A019B30003900A434F6F7BB
:109B2000EBFA2570B0E7C0460C0C0010700B00106B
:109B30008001001058010010F18E0000918F00008C
:109B40007207000051EF0000AD890000018A00009B
:109B5000558A0000B58A0000158B00005D8B00005F
:109B6000A58B0000FD8B000070B5104B104C1B78CE
:109B70009B0709D50F48037E002B02D10E49F9F748
:109B8000F7FDFFF751FF70BDFCF706FF21008025B0
:109B90002000A8318A68C9682D064B19B0300260D0
:109BA00043600123A4342370EDE7C0460C0C001081
:109BB000700B001080010010F0EE0000F0B56E4B4D
:109BC0006E4C1B7891B05B070AD56D4B1B7E002B4A
:109BD00002D14920F8F792FDFFF726FF11B0F0BD42
:109BE000FCF7B8FEF6F76CFA012834D12500A83549
:109BF000AA68EB6806920793230080331B7800263F
:109C00000027B034002B21D02A686B680892099392
:109C100008980999069A079BF7F7E8FE089A099BA6
:109C20000A900B9106980799FAF752FD0A9A0B9B36
:109C3000266067602A606B60F6F74AFD32003B00E1
:109C4000F6F75AFA01224F4B1A70C7E72660676091
:109C500006980799F2E7022802D187342070BDE701
:109C60002300B83319685A68089109929A68DB682A
:109C7000069207932200230080321278A833002630
:109C8000186859680027002A50D023007E331B78BB
:109C9000002B0FD17F3423780022002B44D03A4B85
:109CA00003F006FD02000B0003F0E8F8374A384BDA
:109CB00004F040F9374B384C18605960374B0200BC
:109CC0001E605F600023029603970493059400963C
:109CD00001970B000CA802F043F80C980D990E9C0C
:109CE0000F9D02000B00019500940CA8FAF75AF999
:109CF0000C9A0D9B0E980F9902920393069B079C5A
:109D00000490059100930194089A099B0CA802F015
:109D100027F80C9C0D9D0E9E0F9F200029003200FD
:109D20003B00F6F71BFA8DE71D4BB9E700241A4DEF
:109D300002960397049405959A68DB680092019354
:109D400002000B000CA802F00BF8089A099B0C9873
:109D50000D990E9C0F9D03F091F8069A079B060043
:109D60000F002000290003F089F804000D003000E6
:109D7000390022002B00D4E70C0C0010700B0010EF
:109D800080010010140C001000007940182D44547C
:109D9000FB210940180C00100000F03F200C0010BF
:109DA00000807640F7B51E4B1E4D1B785B0609D52B
:109DB0001D48037E002B02D11C49F9F7D9FCFFF79F
:109DC00033FEF7BD2C00A834FCF7C4FDA268E3689D
:109DD0002668676800920193009A019B3000390061
:109DE000F6F7AAF901F060FD05F002F8104A114BF0
:109DF00003F05EFCEB23DB00EB1818605960EC23EA
:109E000020606160DB002900EE1800220023B031E1
:109E1000326073600A604B600123A4352B70D0E779
:109E20000C0C0010700B00108001001051EF0000AE
:109E30000000C0FFFFFFDF41F0B5404B89B01800C4
:109E40000093F8F713FC3E4C070028220021200065
:109E5000FCF754FD3B4D3C4BEE5C002E10D00098BF
:109E6000F8F704FC421EAB1888331B7819002A3916
:109E7000012903D902218B432D2B2BD12F4BD654F3
:109E8000324B304D1A78324E002A27D0314B920097
:109E90009B189A6B310002A8F9F76AFC2B009C33DF
:109EA0001B78DB0603D520002B4901F01DFD2000A7
:109EB00002A901F019FD2B009C331B78002B33D035
:109EC0002A00A032254B12680026254F9A4223D142
:109ED00009B0F0BD2D1888352E70D1E71223DB1B99
:109EE0001F4F0193BB7D019A934209DD1D4A20005B
:109EF0001D49F9F73DFCBA7D019BD21ABA18C9E792
:109F0000009A31002000F9F733FC3A00C2E7200044
:109F1000164901F0E9FC01362B0078331B78BA7D35
:109F20009B1AB342F3DCD3E70D4B9B7D0E2BCFD8AE
:109F300020000E4901F0D8FCCAE7C046F80B00101B
:109F4000980B0010700B001072070000F30B00104C
:109F50000EEF000000F3000082F000005D980000AA
:109F60008001001003000010E5EF0000E9EF0000A1
:109F7000002200231349144810B50A634B638A6317
:109F8000CB630A644B648A64CB640A654B658A655B
:109F9000CB650A664B668A66CB660A674B678A673B
:109FA000CB67010079308131FF30FF3102604360BF
:109FB0000A604B60FCF7C2FC402200210348FCF71A
:109FC0009DFC10BD680C0010700B0010180C0010E8
:109FD000CC2210B500210248D200FCF78FFC10BD46
:109FE000780C0010842210B5002102485200FCF7C2
:109FF00085FC10BD94020010F0B5C34F89B0282233
:10A0000000213800FCF77AFCC04D282200212800EE
:10A01000FCF774FCBE4C142200212000FCF76EFCFF
:10A0200014220021BB48FCF769FC3B003A00853351
:10A0300079321B781278134300D1D2E03B007C3395
:10A040001988002904D0002238000139F9F79CFB57
:10A050003E007C36012228003188F9F795FB3088D4
:10A06000F6F776FA0200692807DCAB49632801DDC0
:10A07000AA49233A2000F9F77BFB9C373B78002B59
:10A0800001D0FFF7D9FEA64B9F4C1B78002B32D096
:10A09000012B03D12000A349F9F76AFB2300873382
:10A0A0001B78022B03D120009F49F9F761FB2300A5
:10A0B00087331B78042B03D120009C49F9F758FB08
:10A0C000230087331B78052B03D120009849F9F72B
:10A0D0004FFB230087331B78032B03D120009549C6
:10A0E000F9F746FB230087331B78062B03D12000AA
:10A0F0009149F9F73DFB23007A331B78002B03D0FD
:10A1000020008E49F9F734FB230086331B78002B9F
:10A1100014D12300A5331B78042B0FD023008433E4
:10A120001B7887495BB2012B00D1E4E0013300D0FA
:10A13000D4E01D2283497748F9F71AFB23008533C1
:10A140001B78734D002B27D12300A5331B78042BDC
:10A1500022D023007E331B78002B03D028007A49BD
:10A1600001F0C2FB23007F331B78002B03D02800B3
:10A17000764901F0B9FB764BE35C002B03D07549BF
:10A18000644801F0B1FB230080331B78002B03D01F
:10A190002800714901F0A8FBFFF724FF20000021EF
:10A1A000F9F77AFB08215948F9F776FB0023832158
:10A1B0001A0028008334F8F7B7FF2378002B00D16A
:10A1C0009DE00123082268216448F8F7ADFF0123D0
:10A1D000082252216248F8F7A7FFF8F7D8FF09B024
:10A1E000F0BD3B0086331B78002B0FD03A007C3249
:10A1F0005C4B12889B5C2A2B08D038005A49F9F72F
:10A20000B7FA28005949F9F7B3FA3CE73B00A53300
:10A210001B785748042B4FD1F8F728FA16245549D4
:10A22000241A3800F9F7A4FA384B53491800079359
:10A23000F9F79EFA3800F8F719FA3D18B8373A6876
:10A240007B68BE68FF6804920593300000220023FB
:10A25000390001F037FD002832D12800049A059B0F
:10A26000029401970096FBF7CBFF0798F8F7FEF9E9
:10A27000079B1D18244B0793404B1E685F689A6824
:10A28000DB6804920593049805990022002301F0ED
:10A2900019FD00281BD1059B32000193049B280067
:10A2A000009302943B00FBF7ABFF079A344B9C32C0
:10A2B0001B7E12781343E2E6F8F7D8F91224AEE7D2
:10A2C0002800049A059B0094FBF7BEFDCDE7320001
:10A2D0003B0028000094FBF7B7FDE6E7230082333C
:10A2E0001B782849002B06D1230081331B78002BD3
:10A2F00000D123E72449074801F0F6FA1EE70822B7
:10A300008321044867E7C046700B0010980B0010CB
:10A31000C00B0010D40B0010F6EF0000EBEF0000B4
:10A32000F70B001015F0000021F000002EF00000E7
:10A3300037F0000044F000004FF0000061F0000032
:10A3400067F0000069F000006FF0000073F000009B
:10A350007307000076F0000079F000007CF0000048
:10A3600080F000009C03001001F0000009F00000E4
:10A37000000000100FF0000012F00000180C001098
:10A380008001001007F000006DF0000010B5054BD3
:10A390001B78002B05D0FFF72FFEFA208000F8F77E
:10A3A00007F810BDF60B0010FA23F0B5DB0085B0FE
:10A3B000984200DB99E0002856D0862301227C24B5
:10A3C0005C4F5D49FA544A685C4B02924A683853C4
:10A3D000FA500191FFF710FE3B5B1C1E009300D169
:10A3E00097E00025564E02E00135002C05D0013CD7
:10A3F000305DF6F701F80028F6D1ED0700D56EE0E4
:10A40000504C009BF35C002B30D02B2B00D172E022
:10A41000802B1CD89B001B59002B18D09847019B00
:10A42000029A5B689B1A632B00D96AE08623FB5C67
:10A43000002B00D16FE08723FB5C002B07D1F6F7E0
:10A4400017F8002803D17C23FB5A0093D9E7012495
:10A450009C238621FA5C00237B5438497B50002AD8
:10A4600027D0200005B0F0BD0130A6E79C33FB5C8F
:10A470000293009B012B55DD023B00250393F4184A
:10A4800004E0631E0135A64205D01C002078F5F7D4
:10A49000B3FF0028F5D1ED073FD500237C220399B7
:10A4A000B9520A32BB54254ABB50029B0024002BF0
:10A4B000D7D1019D28352800F8F7D8F80028D0D04A
:10A4C0002800FBF79FFF3B00A8330022186059606B
:10A4D0000023B0373A607B60FCF730FAC1E7F5F74C
:10A4E000C7FF7C23FB5A00938AE787220321114B85
:10A4F00001249954B5E7F5F7BBFF7C23FB5AF35CC5
:10A5000086E7F9F713FA0028A1D1019B5B68029353
:10A510008CE70B4E74E700249AE7009900237C2215
:10A520000139BDE7002BF8D11A008623FA54034BFA
:10A53000FA50BAE7700B00105801001074070000C1
:10A540009C030010A4F80000F8B504000D001000F2
:10A55000002600220027074B01321C605D609E60D0
:10A56000DF601033042AF7D1FFF71EFF014B186894
:10A570005968F8BD180C001010B5FCF7EBF9074A44
:10A58000074B1178002904D000231370F5F770FFF2
:10A5900010BD7C331888FFF707FFF9E7F60B0010B2
:10A5A000700B0010F7B5FCF7D5F9254D254C2F7829
:10A5B000002F0AD085342378002B05D0FBF7FEFE50
:10A5C000C1B20620F6F736F8F7BD26008636337896
:10A5D000002B1DD025007C351B4B2A889B185878F2
:10A5E000F9F75CF8002803D1042387342370EBE7E4
:10A5F0002B88019323000124A4331C70FFF7D4FEA1
:10A60000002801D03770DFE7019B34702B80DBE737
:10A61000230085331B78002B0FD0FEF731FB0C2372
:10A620002B702300094AA0331A60022378340849AA
:10A6300008482370F9F79CF8C6E7FEF74BFBC3E721
:10A640000C0C0010700B00109C030010A5A500005E
:10A6500084F00000F80B001070B5174B174D1B78F5
:10A660001A0708D5164B1B7E002B03D1F8F746F8C6
:10A67000FFF7DAF970BD002BFCD12B0085331B7876
:10A680002330C4B2002B04D021000720F5F7D2FFFD
:10A69000F0E7FCF75FF92B000122A43320001A70C9
:10A6A000F8F7FCFF002802D0FFF77EFEE2E7042364
:10A6B00087352B70DEE7C0460C0C0010700B0010C5
:10A6C0008001001010B54120FFF7C6FF10BD10B586
:10A6D0004220FFF7C1FF10BD10B54320FFF7BCFFBC
:10A6E00010BD10B54420FFF7B7FF10BD10B54520D1
:10A6F000FFF7B2FF10BD70B5234D244C2B78002B13
:10A7000024D0FBF75BFEC6B23000F8F7C7FF23008A
:10A7100085331B780500002B0AD0002803D00523C1
:10A720008734237003E031002B20F5F783FF70BDE1
:10A73000002808D0FEF7A4FA0123A43428002370CF
:10A74000FFF732FEF3E704238734EAE7230086337A
:10A750001B78002BEBD1FCF7FDF8FEF791FA0823EC
:10A760002B7023000A4AA0331A6023000222783398
:10A770001A708534237807480749002B00D1074910
:10A78000F8F7F6FFD3E7C0460C0C0010700B001072
:10A79000F7A60000F80B00108DF0000097F0000005
:10A7A00010B508210120F7F7EBFC02210020F7F794
:10A7B000E7FC00210220F7F7E3FC06210220F7F76F
:10A7C000DFFC03210800F7F7DBFC0321002208006F
:10A7D000F7F78CFC002206210220F7F787FC012204
:10A7E00006210220F7F782FCFFF7FCFBF8F7CFFC0D
:10A7F000A220F7F7BAFCA020F7F7B7FCC020F7F7C4
:10A80000B4FCF820F7F7B1FC0020F7F7AEFC0A2003
:10A81000F7F7CEFD4020F7F7A8FC2C20F7F7A5FCB2
:10A820003220F7F7C5FD2E20F7F79FFC3220F7F70F
:10A83000BFFD2F20F7F799FC0A20F7F7B9FD252077
:10A84000F7F793FC0A20F7F7B3FD8120F7F78DFCAB
:10A850000020F7F78AFCAF20F7F787FCA420F7F772
:10A8600084FC10BDF7B58022002107252A4B2B4C14
:10A87000920301912000DA679022FCF73FF8019BD8
:10A88000274EA360274B284F1A68AA431A6001225B
:10A89000196811431960254B1968A9431960196893
:10A8A00011431960802322495B01086803430B6050
:10A8B000204B1A60823232601F4A126819681F4B9F
:10A8C000D86F504301F036F8E1210009090201F088
:10A8D00031F810221A4B1B491A60030A0B6003233C
:10A8E000C0B2386060203360174B1D60174B1A6888
:10A8F00001921A680240602AFBD15F3A1868104240
:10A9000007D122708022124B92031A6005230B603C
:10A91000F7BD38680190F1E704E100E0040200109F
:10A920000C800040A440044000800040A840044047
:10A9300080800440988004407880044058010010D2
:10A9400028800040048000400880004014800040BF
:10A9500000E100E0FA2110B50C4C8900E06F01F035
:10A96000B7F880235B04984209D20023084A0138D3
:10A9700063601060074A13600722074B1A60FFF7F5
:10A9800071FFF8F731FCF8F7E7FD10BD5801001032
:10A9900014E000E018E000E010E000E010B500284E
:10A9A00038D080211D4A13688B43136001231C4952
:10A9B0000A681A42FCD003221A4B1A6001230021B4
:10A9C000194A13601160136011681942FCD0174ACC
:10A9D0001749136080230C685B0223430B60002837
:10A9E00004D180230D490C6823430B60114B9968F7
:10A9F00081420ED09860434258410F4B404218406C
:10AA00000E4B1168C01800F095FF0D4CE067FFF782
:10AA1000A1FF10BD034B1860D0E7C0463882044048
:10AA20000C800440708004407480044078800440AE
:10AA3000808004400000001000AFDAFD006CDC02F2
:10AA400058010010064A10B5936901339361054B14
:10AA50009868FFF7A3FFF8F70DFCC046C04610BD8D
:10AA6000D801001000000010F0B585B0070001917A
:10AA700072B68022784B1202DA676C220024774B80
:10AA800077491A60774B00201A680A401A601A68E2
:10AA90001A60754B1A680A401A601A6804211A6015
:10AAA0000122F7F701FB012204210020F7F71EFB2A
:10AAB000012205210020F7F7F7FA012205210020E5
:10AAC000F7F714FB694B6A4D1C606B782E78190000
:10AAD0000122300000930134F7F7E6FA002230003B
:10AAE0000099F7F703FB02350A2CEED10024002071
:10AAF000F7F77CFB5F4B21005F48DC60F7F762FBF8
:10AB000021005E48F7F75EFB21005D48F7F75AFB2E
:10AB100021005C48F7F756FB21005B48F7F752FB32
:10AB20005A4B5B4D1A685B4B5B4E1A607B427B4114
:10AB30005A4A9B019B185A4A13600423594A1168C8
:10AB40000B43594913602C600B68584A13400B6043
:10AB5000019B2A68012B00D179E0EC235B011343B0
:10AB60002B6080233360DB1833608023DB0033608D
:10AB700080235B01336080231B013360002F4FD0A3
:10AB800000244B4B4B4F1C604B4B38001C604B4B15
:10AB900021001C604A4B1C60F7F714FB22000921BE
:10ABA0002000F7F781FA220009212000F7F79EFA2A
:10ABB0008021444A444813680B43136007223B68D2
:10ABC00093433B603B68053A13433B603F4B404F28
:10ABD000186003203F4B1C603F4B18603F4B1868C8
:10ABE00038401860186801431960802380219B0059
:10ABF0002D484902336031600168194301602968BA
:10AC00000B432B60012336490B6036490A60364AF4
:10AC100013601460136011681942FCD0244A136059
:10AC20000122324B52421A60314B9A69039262B64A
:10AC300030BFC046039A9B699A4206D130BF2D4B64
:10AC40009868FFF7ABFEF8F715FB05B0F0BD802361
:10AC50001B0113432B608EE704E100E01800004065
:10AC6000F8FCFFFF304004403440044004800440BE
:10AC7000CAF200005801001008400440004004409F
:10AC8000AC400440144004401C400440388204405E
:10AC9000048204403482044000E100E0BF18000058
:10ACA0003082044010ED00E0008204407FE2FFFFAC
:10ACB00004C00040644004400400014004400140DE
:10ACC0000480014080800440841E000018C00040C1
:10ACD0000FF0FFFF08C0004014C000403CC000401F
:10ACE00078800440708004407480044008820440EE
:10ACF000D80100100000001010B50A20F7F758FB2B
:10AD0000F8F714FE0128F8D01C4C237A002B18D039
:10AD1000002323722373E371637A002B07D1C122CE
:10AD200002210E205200F8F703FC01236372A37A7C
:10AD3000227A5B00134301210C2208001A43F8F722
:10AD4000F7FBAC20F7F711FAAE20F7F70EFAA520C3
:10AD5000F7F70BFA00200121FFF786FE0020F7F736
:10AD600075FA002802D10121FFF77EFEFFF718FDDA
:10AD7000FFF738F9F8F70BFA10BDC046D8010010FC
:10AD8000F7B5F7F783F9CE4A012413681B0B1B03B1
:10AD90001360CC4A13681B0B1B031360CA4A136869
:10ADA0001B0B1B031360C94A13681B0B1B031360A7
:10ADB0000022C74B1A60C74B1C601A601C601A68DF
:10ADC0002242FCD02322C44B01201A60FFF7E6FD8B
:10ADD000F7F75CF940213F20C04B1A688A431A609C
:10ADE000BF4A1060BF4A14601A688A431A60FFF7AE
:10ADF000D7FCFFF7F7F8FFF7ADFDBB4B0093DB681F
:10AE0000002B01D1F7F704FA0021B848F7F7DAF977
:10AE10000021B748F7F7D6F9F7F7BEF9F8F79CFB2A
:10AE2000B4480921B44D00F059FD0020E872F7F74D
:10AE30000DFA00285AD1F8F723FB0026009B5E612B
:10AE4000FA239B00EB61FFF70DFDCC223100D2000D
:10AE5000AA48FBF753FD0222A94CAA4BFF321A80E5
:10AE60002300FD3AA6331A7023000B3278331A7090
:10AE70002300A54A7C33A549A5481E80F8F778FC35
:10AE8000FBF75CFDF7F7FAFBFFF7B6F8F8F74EFDB6
:10AE9000A04A0600A35C002800D159E1002B04D091
:10AEA0000023A35422007C3213800022009B9A616D
:10AEB000230087331F7897423DD01A70F7F7DEFBE7
:10AEC0009622009B92009B69934204D3FFF714FFE4
:10AED0000023009A9361FFF78FF88E4BE35C002B01
:10AEE000D4D103210A20FFF7BFFDCFE7F8F7FEFA20
:10AEF0000C2203001340104202D02A7913432B7115
:10AF00002B795B0711D5F8F7BBFAAB79002B03D08F
:10AF10002B7B012B02D801332B7302E0009B5B6972
:10AF2000EB610023009AEB71536100232B71EB7AE4
:10AF3000002B82D17FE7A02E4FDDA021300000F052
:10AF4000ADFE0D2917D1FDF79BFE7348F8F7ECFB1A
:10AF50000126724B7248995DF8F7E6FBFA23013639
:10AF6000DB009E42F5D16F4E3000F8F7DDFB30007C
:10AF7000F8F7DAFBA2E711290CD1FDF781FE2300D7
:10AF80007C331F800123634A6748A354F8F7CCFB46
:10AF90006448EDE7072907D1230086331B78002B8F
:10AFA0008CD1FDF7CFFE89E7062907D12300863330
:10AFB0001B78002B82D1FDF78DFE7FE7322900D070
:10AFC0007CE7FA223900D2005448FBF797FC2300B3
:10AFD0007C331F80FDF754FE70E723009C331B7801
:10AFE000002B3CD033003D3B012B28D928213000D9
:10AFF00000F054FE122903DC4C4BCB40DB071ED47F
:10B000003200143A142A15D801239340484A1342B7
:10B0100015D1112213420DD0230083331B78002B4E
:10B020000DD114290EDC434BCB40DB070AD5283168
:10B03000C8B205E033000422373B9343F1D1F0B2AC
:10B04000F8F7D6FA00982830F7F710FB230078338A
:10B050001B78984200D031E7FEF7E6FC2EE723008C
:10B0600085331B78F7B23800002B23D0F5F7C4F9ED
:10B0700000281ED13C2F63D82B2F13D8122F1CD998
:10B080002821380000F0DCFCFB230539194210D0E0
:10B090003B007F33DBB21E2B0BD900213800F5F7C4
:10B0A000C9FA0BE73A00244B2C3AD2B2D340DB0763
:10B0B000E6D53800F8F79CFA00E7204BF340F6E7B6
:10B0C000008000500080015000800250008003503A
:10B0D000408004404480044008800440388204409A
:10B0E00024800440D8800440580100109840044057
:10B0F0009C400440DC010010D8010010780C0010C6
:10B10000700B0010140C0010000000100EEF000077
:10B11000F80B001073070000AAF000009C03001059
:10B12000A0F00000B4F00000A4F000002200040031
:10B13000E6DD1F0010911900513101000A000400E2
:10B14000532F02D8512F9BD9B3E7612F98D1B0E785
:10B15000002B00D1B4E63A4A917B537B994200D14F
:10B1600094E6937BD318DE7B937B0133DBB293733E
:10B170005BB2002B01DA002393730D2E03D00A2E4D
:10B1800001D0202E28D12F0020373800FBF7DCF823
:10B190000A22002101903800FBF7B0FB294B310057
:10B1A0002948DF60F8F7C0FA019BFF2B00D96DE654
:10B1B00022007C321688002E39D1FA223100234831
:10B1C000D200FBF79BFB23000136B6B27C33019A19
:10B1D0001E801E4B9A5559E6082E01D07F2E18D19D
:10B1E000184FFB6801932B00019A20339A42B2D981
:10B1F000154E08213000F8F797FA20213000F8F7B3
:10B2000093FA08213000F8F78FFA019B013BFB60AD
:10B21000A1E73300303B092B9DD831000A48F8F7ED
:10B2200083FA084AD368591CD1601E7093E7084B13
:10B230009E42C8D100231380064AA35426E6C04686
:10B240000402001000000010F3EF00009C03001047
:10B25000CF0700007307000010B50A4A0A4B0B49DC
:10B260008B4206D300210A4B0A4A934206D3FFF7CA
:10B2700087FD1078013218700133F1E7197001333E
:10B28000F3E7C046F4FC0000000000105801001075
:10B2900058010010201400100023CA5CC25401336E
:10B2A000002AFAD17047C046F0B5604B89B01B68E0
:10B2B0005F4C05935F4B06901A685B6800920193A0
:10B2C000009801992300B8331E685F6832003B0084
:10B2D00000F012FD00280CD000220023F834266074
:10B2E0006760A260E360009A019B009601971600D8
:10B2F0001F0000980199069AFFF726F94E4B0400AB
:10B300001B780D00002B00D18AE009B0F0BD049B32
:10B31000069A0133300039000493FFF715F9220033
:10B320002B000290039103F0CDF804000D00F8F714
:10B33000BFFB424A424B00F0CBFC002843D13E4BBE
:10B3400007931B78002BE0D1009A019B3000390055
:10B3500003F0B8F8029A039B02F0ECFD22002B00E8
:10B3600002F0A6F90B0002003900300003F0AAF841
:10B37000049B04000D00652B07D1079A5F3B1370F7
:10B380000096019726002F001DE0284B059A009398
:10B390001B689B1A632B06D9F8F7C8FA0028EFD16F
:10B3A000009B1B6805930096019726002F00029CC6
:10B3B000039D02980399F8F77BFB204A204B00F08D
:10B3C0009BFC0028A3D1049803F012FD184C1D4DDE
:10B3D00000222860696021000023E0310A604B6090
:10B3E000029A039B2100C8310A604B6021000022B1
:10B3F0000023D0310A604B60009A019B2100B831D4
:10B400000A604B60210000220023C0310A604B60BB
:10B410002100B034A8310E604F602260636074E791
:10B4200000220493084B02920393C2E75C010010D0
:10B43000700B0010180C0010F70B00101656E79E4A
:10B44000AF03D23C480C00100000F03FF0B5B74B02
:10B45000DDB01B6816901793B54B1B78181C0F2B8B
:10B4600000D90F20C0B2404203F0C2FC02000B0022
:10B470000020B049F9F7ACFEAF4B1890199100933A
:10B48000AE4B1E685F68009B3000B8331C685D6877
:10B49000390022002B0000F02FFC00280DD00022E4
:10B4A00000230099F8318A60CB6032003B000C60C9
:10B4B0004D6026002F0014001D0022002B003000DC
:10B4C000390001F0DBFC00229D4B02F033FD0890B7
:10B4D00009918021002300220020C905F9F778FE98
:10B4E00008980999169AFFF72FF804900591954B43
:10B4F0001B78002B00D00FE13B0032002000290018
:10B5000002F0E0FF0022904B02F014FD00228F4B6E
:10B510000A900B9102F00EFD0B00020010901191A9
:10B520000498059902F006FD1CAB03933CAB029313
:10B5300001231F001C901D910693784203F058FCD4
:10B540000B001290139180210200C9050020F9F729
:10B550003FFE00227E4B02F0B5FF02000B0004000C
:10B560000D0002F0E7FC02000B000C900D91002092
:10B57000764902F0A7FF22002B0002F0DBFC0A9ABA
:10B580000B9B02F0D7FC089A099B01F077FC169AF6
:10B59000FEF7DAFF0E900F916A4B1E78002E00D056
:10B5A000BAE0069B00200133009369490C9A0D9B79
:10B5B00002F088FF0E9A0F9B02F0BCFC0C900D91DC
:10B5C0000E96009B069A981A03F012FC149015919F
:10B5D000380003F00DFC0B0080210200C90500209B
:10B5E000F9F7F6FD00225A4B02F06CFF02000B0047
:10B5F0001498159900F076FB002800D0AEE00C9A64
:10B600000D9B0498059901F039FC129A139B049044
:10B61000059180210020C905F9F7DAFD02000B0031
:10B620001098119902F086FC049A059B02F082FCA6
:10B63000029B01241D0018605960039E2A686B68F4
:10B6400006920793069807990CCE02F03BFF0C90E8
:10B650000D91200003F0CCFB02000B0000203D49BF
:10B66000F9F7B6FD00223A4B02F02CFF02000B0066
:10B670000C980D9902F01CF8069A079B01F0FEFB4E
:10B680000134A860E9600835BC42D7DD029BF900AF
:10B690005A181368546806930794039B591808397D
:10B6A000069A079B0868496802F00CFF069A079BF8
:10B6B0000C900D9101F0FCFFF8F7FAF902000B0075
:10B6C000012F00D1A3E01898199900F015FB00286C
:10B6D00000D19CE0184C009803F08AFB2300002660
:10B6E00000271D4DD033286069600C980D991E60AD
:10B6F0005F60F8F7DDF92300B833186059600699E8
:10B70000079A2300C0331E605F602300A833B03463
:10B7100019605A60266067605DB0F0BD029B039AB5
:10B720000393009B0292069307E7C0465C0100105A
:10B73000160C001000002440700B0010180C0010B4
:10B740000000E03FF70B00100000D03F0000084071
:10B750000000F03F00001040380C00100120009B5A
:10B76000C01B0133009303F043FB0B008021020058
:10B77000C9050020F9F72CFD02000B00200029006C
:10B7800001F07CFB02000B0004000D0002F0D2FB74
:10B7900002000B00149015910020374902F092FE30
:10B7A00022002B0002F0C6FB0A9A0B9B02F0C2FBA0
:10B7B000089A099B01F062FB169AFEF7C5FE1A90E3
:10B7C0001B912E4B1B78002BA6D12D4E179A336858
:10B7D0009B1A632B08D9F8F7A9F8431E98410E9BD2
:10B7E00003430E9333681793149A159B0020254941
:10B7F00002F068FE1A9A1B9B02F09CFB02000B00F1
:10B800000C980D9901F03AFB0C900D91D9E60E9B26
:10B81000002B00D05EE70137112F00D07EE7062213
:10B82000164B194C1A70009803F0E2FA2300002618
:10B8300000272500D0331E605F60029BC8359A6FD9
:10B84000DB6F00920193039B286069600098019967
:10B8500080331A685B6802F035FEF8F729F9230097
:10B86000B833186059600099019A2300C0331E60F4
:10B870005F602300A8334AE700000840F70B001080
:10B880005C0100100000F03F700B0010C317C018DF
:10B89000584070470022034B1B68983318605A6069
:10B8A0007047C04610000010094B10B51C68094ACB
:10B8B000983420686168084B00F0C8F80122002322
:10B8C00080185941206061604800400810BDC046A2
:10B8D000100000102D7F954C2DF4515810B50A0022
:10B8E0000021FBF70BF810BD70B50400830716D1DB
:10B8F00002680E4B0E4DD31893432B420FD1426872
:10B900000A4B0430D31893432B4208D14268074BAB
:10B910000430D31893432B42F1D000E00130037878
:10B92000002BFBD1FFF7B8FC200070BDFFFEFEFE30
:10B9300080808080002243088B4274D303098B42AD
:10B940005FD3030A8B4244D3030B8B4228D3030CEF
:10B950008B420DD3FF22090212BA030C8B4202D391
:10B960001212090265D0030B8B4219D300E0090AB9
:10B97000C30B8B4201D3CB03C01A5241830B8B42C2
:10B9800001D38B03C01A5241430B8B4201D34B03AB
:10B99000C01A5241030B8B4201D30B03C01A524110
:10B9A000C30A8B4201D3CB02C01A5241830A8B4295
:10B9B00001D38B02C01A5241430A8B4201D34B027E
:10B9C000C01A5241030A8B4201D30B02C01A5241E2
:10B9D000CDD2C3098B4201D3CB01C01A5241830996
:10B9E0008B4201D38B01C01A524143098B4201D3D0
:10B9F0004B01C01A524103098B4201D30B01C01AFB
:10BA00005241C3088B4201D3CB00C01A5241830874
:10BA10008B4201D38B00C01A524143088B4201D3A1
:10BA20004B00C01A5241411A00D201465241104601
:10BA30007047FFE701B5002000F006F802BDC046E0
:10BA40000029F7D076E770477047C046F0B5CE467C
:10BA50009946030C9C46130447461B0C1D000E0020
:10BA600061460404240C80B50700100C4B43654369
:10BA7000414360432C0CC01824188C46A34203D9C0
:10BA800080235B029846C444494679435643230CBD
:10BA90002D042D0C8919634424046019C918C0BCF5
:10BAA000B946B046F0BDC04602B4714649084900E7
:10BAB000095649008E4402BC7047C04602B4714624
:10BAC00049084900095C49008E4402BC7047C046E1
:10BAD00003460B437FD4002243088B4274D30309EF
:10BAE0008B425FD3030A8B4244D3030B8B4228D390
:10BAF000030C8B420DD3FF22090212BA030C8B42B6
:10BB000002D31212090265D0030B8B4219D300E055
:10BB1000090AC30B8B4201D3CB03C01A5241830BDA
:10BB20008B4201D38B03C01A5241430B8B4201D38A
:10BB30004B03C01A5241030B8B4201D30B03C01AB3
:10BB40005241C30A8B4201D3CB02C01A5241830A2D
:10BB50008B4201D38B02C01A5241430A8B4201D35C
:10BB60004B02C01A5241030A8B4201D30B02C01A86
:10BB70005241CDD2C3098B4201D3CB01C01A5241ED
:10BB800083098B4201D38B01C01A524143098B4276
:10BB900001D34B01C01A524103098B4201D30B015F
:10BBA000C01A5241C3088B4201D3CB00C01A524184
:10BBB00083088B4201D38B00C01A524143088B4249
:10BBC00001D34B00C01A5241411A00D201465241E2
:10BBD000104670475DE0CA0F00D04942031000D301
:10BBE0004042534000229C4603098B422DD3030A56
:10BBF0008B4212D3FC22890112BA030A8B420CD366
:10BC0000890192118B4208D3890192118B4204D38E
:10BC100089013AD0921100E08909C3098B4201D30E
:10BC2000CB01C01A524183098B4201D38B01C01A48
:10BC3000524143098B4201D34B01C01A52410309BF
:10BC40008B4201D30B01C01A5241C3088B4201D36E
:10BC5000CB00C01A524183088B4201D38B00C01A1B
:10BC60005241D9D243088B4201D34B00C01A5241F2
:10BC7000411A00D20146634652415B10104601D37F
:10BC80004042002B00D54942704763465B1000D309
:10BC9000404201B50020FFF7D7FE02BD0029F8D0D1
:10BCA00016E770478446100062468C4619006346CA
:10BCB00000E0C0461FB502F0CFF8002801D40021F3
:10BCC000C8421FBD10B502F011F84042013010BD4E
:10BCD00010B502F0C1F8002801DB002010BD0120E2
:10BCE00010BDC04610B502F0B7F8002801DD0020F5
:10BCF00010BD012010BDC04610B502F03DF800286F
:10BD000001DC002010BD012010BDC04610B502F0BE
:10BD100033F8002801DA002010BD012010BDC04614
:10BD2000002B11D1002A0FD1002900D1002802D008
:10BD30000021C943080007B4024802A1401802903C
:10BD400003BDC04605FDFFFF03B4684601B5029878
:10BD500000F0C8FF019B9E4602B00CBC7047C04675
:10BD6000F0B516001F0091B03900189A199B050014
:10BD700030000A960B9702F0DDF81A9A1B9B02908E
:10BD800003911698179902F0D5F81A9A1B9B049004
:10BD900005913000390002F0CDF8169A179B0690F5
:10BDA00007911898199902F0C5F8049A059B089014
:10BDB00009910298039902F085FB089A099B0600F5
:10BDC0000F000698079901F059F832000090019190
:10BDD0003B003000390002F0ADFF002808D1009B85
:10BDE000019C28002E606F60AB60EC6011B0F0BD6C
:10BDF0000098019902000B0002F09CFF0028EED091
:10BE00000A990B9A530001225B080D93169B0C9123
:10BE10000E93179B52425B005B080F930C980D9991
:10BE2000874B02F087FF002809D10C980D99012259
:10BE3000834B5242FFF756FF002800D104E10E98D1
:10BE40000F9901227E4B524202F074FF002809D163
:10BE50000E980F9901227A4B5242FFF743FF0028B8
:10BE600000D1F1E001221A9B52420C931B9B5B0014
:10BE70005B080D93189B0E93199B5B005B080F9357
:10BE80000E980F996E4B02F055FF002809D10E98BD
:10BE90000F9901226A4B5242FFF724FF002800D17C
:10BEA000B0E10C980D990122654B524202F042FF1D
:10BEB000002809D10C980D990122614B5242FFF7DD
:10BEC00011FF002800D14CE10299039A530001228E
:10BED0005B08039302915A4B52420298039902F075
:10BEE00029FF002808D1029803990122544B52429D
:10BEF000FFF7F8FE002849D00499059A5300012263
:10BF00005B08039302914E4B52420298039902F050
:10BF100011FF002808D1029803990122484B524290
:10BF2000FFF7E0FE002831D00699079A530001225E
:10BF30005B0803930291424B52420298039902F02C
:10BF4000F9FE002808D10298039901223C4B524285
:10BF5000FFF7C8FE002819D00899099A530001225A
:10BF60005B0803930291364B52420298039902F008
:10BF7000E1FE002800D032E7029803990122304BFD
:10BF80005242FFF7AFFE002800D028E70A980B992D
:10BF900002000B0002F0CEFE002800D091E1169ABC
:10BFA000179B1000190002F0C5FE002800D07DE1AB
:10BFB000189A199B1000190002F0BCFE002800D04E
:10BFC00069E11A9A1B9B1000190002F0B3FE0028C9
:10BFD00000D055E1189A199B0A980B9901F0AAFF15
:10BFE0001A9A1B9B06000F001698179901F0A2FFE2
:10BFF00002000B003000390002F064FA0022114BFD
:10C0000001F098FF1A9A1B9B06000F000A980B99E3
:10C0100001F090FF189A199B0090019116981799BA
:10C0200001F088FF02000B000098019900F026FF44
:10C030000022044B01F07EFF00900191CFE6C04644
:10C04000FFFFEF7F0000F07F01220C980D99A24BBB
:10C050005242012602F06EFE00280AD10C980D997A
:10C0600001229D4B5242FFF73DFE431E9841404244
:10C07000064001235E40F0B202F0BAFE0E9E0F9F12
:10C080000B9B4A00DB0FDB0752081A431100012209
:10C090000A900B91904B300039005242012402F07B
:10C0A00049FE00280AD101228B4B30003900524250
:10C0B000FFF718FE431E98414042044001235C40B4
:10C0C000E0B202F095FE179B4A00DB0FDB07520837
:10C0D0001A431100189A199B169017911000190015
:10C0E00002F028FE002800D0BFE0189B1E00199B1C
:10C0F0005B005F081A9A1B9B1000190002F01AFEE1
:10C10000002800D08CE001221A9B30000C931B9B6E
:10C1100039005B005B080D9352426F4B02F00AFE40
:10C12000002808D10122300039006B4B5242FFF742
:10C13000D9FD002866D00C9E0D9F012230003900E9
:10C14000654B524202F0F6FD002800D042E7012282
:10C1500030003900604B5242FFF7C4FD002800D088
:10C1600038E70023002600275C4C0C930D941999A6
:10C170007800C90FC9074008084332000C9E0D9F84
:10C18000030018921993012230003900524B524299
:10C19000012402F0CFFD00280AD101224E4B3000CD
:10C1A00039005242FFF79EFD431E98414042044031
:10C1B00001235C40E0B202F01BFE1B9B4A00DB0F38
:10C1C000DB0752081A4311001A901B910A980B9929
:10C1D00002000B0002F0AEFD002816D1169A179B44
:10C1E0001000190002F0A6FD002800D1F2E6179910
:10C1F00000220023002902DA802300221B06169267
:10C200001793E7E60026364FB1E70B99002200238B
:10C21000002902DA802300221B060A920B93DDE735
:10C220001B9900220023002902DA802300221B062A
:10C230001A921B93012230003900274B524202F020
:10C2400079FD002800D0C5E6012230003900224BDC
:10C250005242FFF747FD002800D0BBE60023002430
:10C2600000260C930D941E4F81E71999002200239C
:10C27000002902DA802300221B061892199334E762
:10C280001B9900220023002902DA802300221B06CA
:10C290001A921B939EE6199900220023002902DAC4
:10C2A000802300221B06189219938AE61799002210
:10C2B0000023002902DA802300221B06169217931E
:10C2C00076E60B9900220023002902DA802300225F
:10C2D0001B060A920B9362E6FFFFEF7F0000F07FE0
:10C2E0000000F03FF0B54746CE4680B589B01D004E
:10C2F000129B80461E00139B14005B005F08149B7A
:10C3000030000093159B39005B005B080193009A95
:10C31000019BFFF7DDFC0122C64B5242002800D1F1
:10C320008CE000980199FFF7F1FC002825D000224D
:10C3300020002900C04B01F0FDFD0022BE4B04008F
:10C340000D001098119901F0F5FD00221090119147
:10C3500012981399B84B01F0EDFDB74B1290139161
:10C3600014981599002201F0E5FD14901591149B85
:10C370000093159B5B005B080193002200980199D4
:10C38000AE4BFFF7A5FC002800D12BE100222000D6
:10C390002900AB4B01F0CEFD0022A94B04000D009B
:10C3A0001098119901F0C6FD002210901191129879
:10C3B0001399A34B01F0BEFD002212901391149823
:10C3C00015999F4B01F0B6FD14901591149A159B89
:10C3D0001298139901F06CF902000B0006000F008F
:10C3E0001298139901F0A6FD149A159B00F046FDD2
:10C3F0007B000290039159088023300000225B03E8
:10C40000FFF77AFC002800D11EE132003B0020003B
:10C41000290001F08FFD109A119B00F02FFD029A68
:10C42000039B01F045F932003B0000900191109808
:10C43000119901F07FFD22002B008CE030003900C3
:10C44000FFF764FC002824D00022200029007A4B4A
:10C4500001F070FD0022784B04000D001098119936
:10C4600001F068FD00221090119112981399724BFF
:10C4700001F060FD704B12901391149815990022F1
:10C4800001F058FD129B149015911E00139B5B0048
:10C490005F08002230003900684BFFF719FC0028C4
:10C4A00000D176E0002220002900654B01F042FD1A
:10C4B0000022634B04000D001098119901F03AFD21
:10C4C000002210901191129813995D4B01F032FDEA
:10C4D00000221290139114981599594B01F02AFDDE
:10C4E00014901591129A139B1498159901F0E0F885
:10C4F00002000B0006000F001498159901F01AFDB8
:10C50000129A139B00F0BAFC7B0002900391590829
:10C510008023300000225B03FFF7EEFB002800D1F0
:10C52000BDE01098119932003B0001F003FD22009C
:10C530002B0000F0A3FC029A039B01F0B9F8320033
:10C54000009001913B002000290001F0F3FC020063
:10C550000B001098119901F0B5FF029A039B01F0AE
:10C56000A7F806000F000098019902000B0002F0E6
:10C57000E1FB002800D0E1E0009B019C42464046E0
:10C58000136054609660D76009B0C0BCB946B0462D
:10C59000F0BD6B005B080193109B00940293119B0C
:10C5A0000022009801995B005B08039380235B03E2
:10C5B000FFF78EFB002800D1ABE00298039901221F
:10C5C000204B5242FFF784FB002800D18AE701226A
:10C5D000300039001B4B5242FFF77AFB002800D194
:10C5E00080E75FE76B005F08109B00220293119BBE
:10C5F00020005B005B080393802339005B03FFF797
:10C6000067FB002800D16FE00298039901220D4BCF
:10C610005242FFF75DFB002800D1D7E60098019950
:10C620000122084B5242FFF753FB002800D1CDE610
:10C63000ACE6C046FFFFDF7F0000E03F0000B03CFB
:10C6400000003043FFFF9F7C149A159B20002900B7
:10C6500001F02EF8129A139B01F06CFC109A119BBA
:10C6600000F00CFC029E039F32003B0001F020F81A
:10C67000149A159B009001911098119901F018F8E7
:10C68000129A139B01F056FC22002B0001F01AFFB6
:10C6900032003B0001F00CF806000F0063E7129A2D
:10C6A000139B1098119901F003F8149A159B01F04F
:10C6B00041FC22002B0000F0E1FB029E039F3200B0
:10C6C0003B0000F0F5FF129A139B009001912000AF
:10C6D000290000F0EDFF149A159B01F02BFC0200DD
:10C6E0000B0010981199D1E780230298039900223A
:10C6F0005B03FFF7EDFA002800D167E60122200076
:10C7000039009A4B5242FFF7E3FA002800D15DE668
:10C7100084E780230298039900225B03FFF7D8FA8D
:10C72000002800D1DEE60098019901228F4B524289
:10C73000FFF7CEFA002800D1D4E648E732003B00EC
:10C740003000390002F0F6FA002800D114E7129800
:10C75000139900220023FFF7B5FA002800D109E160
:10C760001498159900220023FFF7ACFA002800D096
:10C770000FE201226B005B08039302947C4B524250
:10C780000298039902F0D6FA002809D10298039979
:10C790000122774B5242FFF7A5FA002800D11BE196
:10C7A0000122109B52420693119B5B0099465B0845
:10C7B0000793069807996E4B02F0BCFA002809D13E
:10C7C0000698079901226A4B5242FFF78BFA00281C
:10C7D00000D1FEE100220021149B0693159B5B0013
:10C7E0005B08079313000A000492059306980799C3
:10C7F00001225F4B524202F09DFA002800D0BBE6B6
:10C800000698079901225A4B5242FFF76BFA00280B
:10C8100000D0B1E6029803990122554B524202F032
:10C8200089FA002800D0A7E6029803990122504B0C
:10C830005242FFF761FA002800D09DE6109B0122CA
:10C8400002934B465B0803935242494B029803996B
:10C8500002F070FA002800D08EE6029803990122B7
:10C86000434B5242FFF748FA002800D084E6049870
:10C87000059901223E4B5242012602F05BFA002844
:10C8800009D1049805990122394B5242FFF72AFA3F
:10C89000002800D1061C01207040C0B202F0A8FAA6
:10C8A000139B4A00DB0FDB0752081A43149B0392C9
:10C8B0001E00159B01225B005F0801230290994630
:10C8C000300039002A4B524202F034FA002809D1D4
:10C8D000012230003900264B5242FFF703FA0028AC
:10C8E00000D1814601204B464340D8B202F080FA85
:10C8F000159B4A00DB0FDB0752081A43060017009E
:10C90000029A039B2000290001F014FB32003B0037
:10C91000009001911098119901F00CFB02000B009E
:10C920000098019900F0AAFA0022002301F002FB0E
:10C93000029A039B009001911098119901F0FAFA64
:10C9400032003B00029003912000290001F0F2FA2E
:10C9500002000B000298039901F0B4FD00220023AD
:10C9600001F0E8FA06000F0006E6C046FFFF9F7CD4
:10C97000FFFFEF7F01226B005B080393129B029481
:10C980000493139B52425B005B0805930298039942
:10C99000A84B02F0CFF9002800D0B8E00298039924
:10C9A0000122A44B5242FFF79DF9002800D0AEE0CF
:10C9B0000498059901229F4B524202F0BBF90028CE
:10C9C00000D0D9E50498059901229A4B5242FFF70D
:10C9D00093F9002800D0CFE50122149B5242029324
:10C9E000159B5B005B08039302980399914B02F03F
:10C9F000A1F9002800D0BFE50298039901228D4BD0
:10CA00005242FFF779F9002800D0B5E500228A4BA1
:10CA100002920393119B5B009946029803990122AD
:10CA2000844B5242012602F085F9002809D1029870
:10CA3000039901227F4B5242FFF754F9002800D19D
:10CA4000061C01207040C0B202F0D2F9EB0F4A0080
:10CA5000DB0752081A43109B03921C004B4601222D
:10CA60005D08029029002000724B5242012602F01C
:10CA700061F9002809D10122200029006D4B5242A2
:10CA8000FFF730F9002800D1061C01207040C0B229
:10CA900002F0AEF9119B4A00DB0FDB0752081A4384
:10CAA0000400129813991500029A039B01F042FAB0
:10CAB000220006000F00149815992B0001F03AFA95
:10CAC00002000B003000390000F0D8F900225A4B68
:10CAD00001F030FA22002B00009001911298139976
:10CAE00001F028FA029A039B04000D00149815998E
:10CAF00001F020FA02000B002000290001F0E2FC06
:10CB000000224D4B01F016FA06000F0034E5012219
:10CB1000109B52420693119B5B0099465B0807935A
:10CB200006980799434B02F005F900281AD1069898
:10CB3000079901223F4B5242FFF7D4F8002811D148
:10CB40000498059901223B4B524202F0F3F8002869
:10CB500008D1049805990122364B5242FFF7CCF8D0
:10CB6000002836D0049805990122324B524202F037
:10CB7000E1F8002856D10498059901222D4B524224
:10CB8000FFF7B0F800284DD100222B4B04920593FB
:10CB900040E622002B002000290002F0CBF80028FC
:10CBA00037D1139B0026244F002B01DA0026234F98
:10CBB00022002B003000390001F0BCF9109A119BC3
:10CBC000009001913000390001F0B4F906000F0027
:10CBD000D2E40122149B52420693159B5B005B0832
:10CBE000079306980799134B02F0A4F8002809D17F
:10CBF0000698079901220F4B5242FFF77DF8002853
:10CC000000D10AE7129B0493139B5B005B0805931A
:10CC1000ECE5109A119B1000190002F08BF8002827
:10CC2000BFD0A9E4149B0693159B5B005B08079398
:10CC3000DCE5C046FFFFEF7F0000F07F0000F0FF63
:10CC400070B500220C4B04000D00FFF75FF80028C0
:10CC500004D12000290002F08FF870BD064B00229D
:10CC60002000290001F02EFC02F086F880231B062C
:10CC70009C466044F1E7C0460000E04170B50022E8
:10CC80000B4B0D00040001F055F9FFF7D9FF06002A
:10CC900002F0DCF80022074B01F04CF902000B0017
:10CCA0002000290001F00EFCFFF7CAFF310070BD23
:10CCB0000000F03D0000F04170B50600080002F0F1
:10CCC000C5F80022064B01F035F90D0004003000D4
:10CCD00002F0BCF82B00220000F0D0F870BDC04676
:10CCE0000000F041F0B557464E464546DE46E0B5F9
:10CCF00004000D009246994683B08B4230D82DD067
:10CD00004946504602F0E4F829000600200002F0EF
:10CD1000DFF8331A9846203B34D49B4653465A4694
:10CD2000934042461F00534693401E00AF423BD8FB
:10CD3000AF4200D179E05B46A41BBD41002B00DA75
:10CD400076E0002200230092019301235A4693408B
:10CD50000193012342469340009329E08242CFD9B8
:10CD600000220023009201930C9B002B01D01C6039
:10CD70005D600098019903B0F0BCBB46B246A9467D
:10CD8000A046F0BD42469B4620239B1A5246DA40FD
:10CD9000414613004A468A40170042461F43534605
:10CDA00093401E00AF42C3D900220023009201939A
:10CDB0004346002BD8D0FB0772081A4346467B082F
:10CDC0000EE0AB4201D1A2420CD8A41A9D41012031
:10CDD00024196D410021013E24184D41002E06D03A
:10CDE000AB42EED9013E24196D41002EF8D10098D6
:10CDF00001995B4600196941002B24DB2B005A4640
:10CE00004646D3402A001C00F2405B461500002B2A
:10CE10002ADB26009E40330026004746BE403200F3
:10CE2000801A9941009001919EE7A342BCD882E705
:10CE30004246202300219B1A0022009101920122E8
:10CE4000DA40019285E7424620239B1A2A00464693
:10CE50009A402300F340464613432A001C00F24048
:10CE60005B461500002BD4DA202342462F009B1B83
:10CE700097402600DE403B003343CDE7F0B54F46F8
:10CE80004646D646C0B50D0382B0009201934E00CF
:10CE9000C300CC0F690A450F9C46009A019B0D43C5
:10CEA0005F001903D80F009B490A5B0F1943009BD1
:10CEB000760D7F0DDA00F31B844258D0002B13DD72
:10CEC000002F00D088E00800104300D159E1581E1F
:10CED000012B00D1C2E2B14FBB4200D141E1382861
:10CEE00000DD6AE2030064E1002B00D1B1E0BB1B6E
:10CEF000002E00D0E1E164462C4300D176E25C1EB6
:10CF0000012B00D1E8E2A54EB34200D1B7E2382CA4
:10CF100000DC6BE3541EA242924152428D1AA0469D
:10CF20001E0004002A0268D443461F1D47459B414A
:10CF30005B42ED182B0200D49DE3984A01369642DD
:10CF400000D1EBE0964A73052A405B0D5107FF08BC
:10CF500052020F43120B1B051343E407234338000F
:10CF6000190002B0E0BCBA46B146A846F0BD002B9D
:10CF700000DCD7E0002F00D09AE00800104300D179
:10CF8000FFE0581E012B00D148E2844FBB4200D184
:10CF9000E7E0382800DCB8E280221204154200D114
:10CFA00049E31E000023150098467C4B01369E4243
:10CFB00000D1B3E07A4B01211D4043465A08194085
:10CFC000EF070A4317436D087B07B3D00F233B409D
:10CFD000042BAFD0B846A7E77048864200D1C0E026
:10CFE000382B00DCE2E001235B4263449C45804136
:10CFF00040422D1A98462B0296D501235B42984653
:10D00000684D280001F046FF0300083B2021404600
:10D01000CA1AD040020040469D4098402A438046AC
:10D02000B34200DA72E1981B43460130091A4546C3
:10D030008B40C5405E1EB34117008F402B431F43FA
:10D04000C2403B00150000261343BDD1002700223B
:10D0500081E7554F731C3B4200D01BE163460F0034
:10D060002B431743002E00D0C4E1002B00D145E232
:10D07000002F00D107E163469B1A9846C445B6418C
:10D080006B1A76429B1B80263604334200D1CBE2DA
:10D090006346D31A9A4292411F00491B52428A1A90
:10D0A0009C46174300D0EDE204000023002252E723
:10D0B0003A48864255D0382B00DD48E180200004F4
:10D0C00001431F2B00DDE3E12027F81A8246080008
:10D0D0005746B840814610004F46D84007433800B5
:10D0E0005746BA40D940571EBA416D1810436044A4
:10D0F0008046E045804140422D182B0200D554E780
:10D1000043465B0700D1B9E20F2342461340042B8C
:10D1100000D009E733004246D20834E03300002251
:10D12000002718E7002B00D18FE0BB1B002E00D09A
:10D1300033E16046284300D140E2581E012B00D164
:10D140000AE2164EB34200D185E2382800DC87E2BD
:10D1500080252D04294200D19CE21E000023984620
:10D1600023E763466E07D8080643ED0837002F43D0
:10D1700011D0802212032A4312033700074B120BEF
:10D18000E9E66246D2086E071643044AED08934268
:10D19000ECD03700D6E0014B0022DCE6FF070000B0
:10D1A000FFFF7FFFFFFF7F00FE07000080200004DD
:10D1B00001431F2B00DDB1E02027F81A824608004A
:10D1C0005746B840814610004F46D84007433800C4
:10D1D0005746BA40D940571EBA416D1A10436346AC
:10D1E0001B1A9C458041984640422D1A2B0287D538
:10D1F0006D026D0A002D00D003E7404601F04AFEA3
:10D20000030018331F2B00DC00E742460838824039
:10D210009E4200DD91E09B1B581C1F2800DCF8E1BA
:10D2200017001F3BDF40202805D040231B1A9A40DF
:10D23000531E9A411743002F3CD000267B0700D095
:10D24000C4E63500B846330065E7CB48731C03429B
:10D2500000D085E063462B43002E00D092E10F0002
:10D260001743002B00D1D8E1002F0CD06244624557
:10D2700080416D1840422D182B0200D5F2E11700B5
:10D2800094462F4316D063466F07D8080743002300
:10D29000ED0857E063469B1A9846C445BF416B1A98
:10D2A0007F42DB1B1F0200D5AEE047461D001F4337
:10D2B000A0D10024002300224DE6B04CA74200D1AB
:10D2C000DDE0382B00DD85E08024240425431F2B7E
:10D2D00000DDECE02026F41AA1462C004E46B440B6
:10D2E0006646DE403443A04666464C46A640DD40D6
:10D2F000741EA6414446491B3443131B9A42924173
:10D300005242984604003E008D1A6FE7F61A030059
:10D310009B4D15405B0700D0F6E6FBE618000F00BA
:10D320002038C740202B03D04020C31A99400A431D
:10D33000531E9A411000384351E79149F31A0A40AD
:10D340005707D5082A035B05120B5B0D03E6802304
:10D350001B041D4200D1BBE01D000023984624E6BB
:10D360008648834200D1DAE662446245804169180A
:10D3700040420918C8075208104380464D0852071A
:10D3800005D00F221E000240042A00D0CCE5424600
:10D390006F07D20817430D09D4E77848874200D1B8
:10D3A000D5E0382B00DCB2E080252D04294200D1E5
:10D3B0004CE100233E009846F7E5012252426244C8
:10D3C0009445804140422D1A90461E002A0200D505
:10D3D00013E6A9E5531E9A42924152428D1A98468D
:10D3E00004003E002B0200D507E69DE504000D0079
:10D3F000D208C8E6002B00D0E3E0002F3FD1802206
:10D4000000245E4B1203A6E56346D31A9A4292416A
:10D410004D1B524298460400AD1AEBE662441600DA
:10D42000664580416A1840421218130200D49DE0FC
:10D43000534973080A40D107194357085B0700D1C5
:10D44000FEE00F230B40042B00D1F9E00B1D9846A2
:10D450008845AD416D420223ED195CE663469B1A97
:10D460009C4580416D1A40422D1A98462B020DD4DE
:10D4700043466F07DB081F43ED08012362E74E07B1
:10D48000D20804001643CD0870E604000126AFE67A
:10D4900018000F002038C740202B03D04020C31AAB
:10D4A00099400A43531E9A41100038431FE61C005E
:10D4B0002E00203CE640202B05D04024E31A9D405E
:10D4C00063462B439C466446631E9C41344314E7E9
:10D4D00001236344984627E56346D31A9A42924152
:10D4E0004D1B5242AD1A98462B02CED443466F07CD
:10D4F000DB081F4304000123ED0823E7002F00D1C0
:10D50000D7E604000D009446BDE60300D9E580206F
:10D51000000405431F2B6BDC2020C01A8046280026
:10D520004646B0406646DE400643B1466046464643
:10D53000B040DD40461EB0414E464919304380465A
:10D5400090449045924152423E005518D5E54E0711
:10D55000D2081643CD0809E663469E1896429241CA
:10D56000691852428A18130200D561E75707F60876
:10D5700001233743D508E5E6FE070000FF0700005A
:10D58000FFFF7FFF002BE2D06346DE086B071E43E0
:10D590000B00ED08134300D1E8E580231B031D4277
:10D5A00006D0C808184203D10500D60849070E4323
:10D5B000730FF600F6085B071E43D7E50D00D2088F
:10D5C000E1E56346DE086B071E43ED08002F00D13E
:10D5D000CCE580231B031D42EAD0CF081F42E7D1D0
:10D5E000D608490704003D000E43E1E723006EE63C
:10D5F00018002E002038C640202B05D04020C31A2A
:10D600009D4063462B439C466046431E98413043F1
:10D6100095E720210023091A0EE50023002F00D1F1
:10D62000BAE50D00904676E547461F4300D140E637
:10D630001D00C44627E60122624490461E0073E4A2
:10D64000C9087F0702230F4315097BE6531C984640
:10D650000D003E0068E4D6084B071E43CD0885E563
:10D66000030057E7114BD2082B405F0717435A02BC
:10D67000120B01236FE43300B8464CE54346DA0849
:10D68000330080E532420AD0084B04001A40674656
:10D6900001235BE4013290460D001E0044E4DB08E8
:10D6A00057071F4304000023D5084BE6FFFF7FFF09
:10D6B000F0B5DE46454657464E46E0B587B0009287
:10D6C00001930B031B0B9B46CA0F4B0004008046C3
:10D6D0005B0D029200D1BFE08F4A934238D0594689
:10D6E000420FC9000A43802109041143C200904639
:10D6F0008A4A894692469A44002300240393009E56
:10D70000019F3B031B0B7A0030009B46520DFD0F1F
:10D71000002A00D17FE0804B9A426ED05946730FA9
:10D72000C9000B438021090419438B467B49F30050
:10D730008C46514662448A1A92460021029E6E40EF
:10D74000F6B20F2C00D9F9E0754AA4001259974699
:10D750005A460243914600D0B6E09A4602239046CC
:10D7600008240393CBE72E000021002300228846E3
:10D770001B051343F60733434046190007B0F0BCBE
:10D78000BB46B246A946A046F0BDCB464346029DE5
:10D790000399022900D1FAE1032900D1A1E001296E
:10D7A000E1D0604A524490464446002C00DC00E23E
:10D7B0005A0704D00F221A40042A00D07FE22E001C
:10D7C000DA085B46DB0106D55946574B80241940E1
:10D7D0008B46E4005444554B9C4209DC5B465B0796
:10D7E000134398465B4664055A02120B630DBFE76C
:10D7F000002100228846484BBAE75B46009A134353
:10D800004B4A9446E244002B59D102221443002291
:10D810000221934692E75B46009A134349D05B4648
:10D82000002B00D1A4E1584601F034FB03000200B4
:10D830000B3B1D27009EFB1A11005846DE4008399D
:10D840008840330003439B46009B8B403949524438
:10D850008A460021924471E75B460343994621D0F2
:10D860005B46002B00D171E1584601F013FB0B23FE
:10D870005B429C460200844466461D239B1B260097
:10D8800011005846DE40083988403300034399466A
:10D8900023008B409846284B00249B1A9A4600236D
:10D8A00003932CE7002398469A46013304240393FC
:10D8B00025E7012214430022012193463EE703237A
:10D8C00003211C43330039E79A460323D9460C242D
:10D8D000039314E700238022984600260E4B120380
:10D8E00046E78022594612030A43120398462E0047
:10D8F000094B120B3CE7802249461203114202D029
:10D9000059461142F0D080224B4612031A431203AB
:10D91000029E014B120B2BE7FF07000001FCFFFFEB
:10D92000ACFC0000FF030000FFFFFFFEFE0700004D
:10D9300001F8FFFFF30300000DFCFFFFCB4500D211
:10D94000FAE000D1F5E0012252429446002244461A
:10D9500048469046E2445A461F0E12021B020293AA
:10D96000130C994617433B041B0C49460093FEF7E2
:10D9700067F8009A0B044243210C050019438A42C0
:10D9800007D9C919013D8F4203D88A4201D9851EA2
:10D99000C919881A4946FEF753F8009A24044243ED
:10D9A0000904240C03000C43A24204D9E419013BEE
:10D9B000A74200D8F7E00299A01A2D040C0C090424
:10D9C0001D43090C2A0C2B04AB460D001B0C5D43B8
:10D9D000059163435143049462435B182C0CE31894
:10D9E000994203D9802149028C466244190C2D04C6
:10D9F0001B042D0C8A185D19904200D287E000D1DB
:10DA000082E043465D1BA8459B41801A5B42C01AD9
:10DA1000B14B534498461C00874200D10CE1494663
:10DA2000FEF70EF80200009B03905A430B04290CEA
:10DA300019438A420AD90300C919013B03938F4253
:10DA400004D88A4202D9831E0393C919881A494609
:10DA5000FDF7F6FF0A00120494462A046546009971
:10DA6000120C414303002A43914207D9D2190138CD
:10DA7000974203D8914201D9981ED219039B521A9A
:10DA80001B0403430598190C05008C461904090C66
:10DA90004D438946614600956546484304994D4388
:10DAA000AC464D464D432918009D2D0CA9464944CE
:10DAB000884203D9802040028146CC44009D080C56
:10DAC0002D0409042D0C60444D1982420FD30BD054
:10DAD00001221343814A92456CDB1A1D9A429B41F5
:10DAE0005B42D2089B446CE6002D00D193E0591EA6
:10DAF000BA188C46BA4200D285E0824200D2C7E012
:10DB000000D1D5E00B00E3E7A84500D379E75B46F9
:10DB1000591E029B9C46E0441C0098459B415B4279
:10DB2000DB19C018874238D2824278D875D08B462C
:10DB300067E7434500D906E74A46D40750084246FE
:10DB4000520814434246D207904604E701F0A2F976
:10DB500015239C4684440200634620321C2B00DCC3
:10DB60008AE623000838834099460023984692E6C7
:10DB700001F090F903000200153320321C2B00DC69
:10DB800057E600990838814000238B465EE6002165
:10DB90002E0000228846524BEAE58742C7D1444511
:10DBA000C2D98B462DE7A24200D804E7831EE419B0
:10DBB00001E72E0001224146521A382A00DDD3E542
:10DBC0001F2A3FDC47481C0050445946834081408F
:10DBD000D440581E834121430B435946D1400A008B
:10DBE000590709D00F211940042905D0191D994260
:10DBF0009B415B42D2180B00110268D50021012322
:10DC000000228846B4E50B00824200D060E7029A09
:10DC1000954200D05CE73500C6E5454587D902232B
:10DC20005B429C46029BE3449C46E04498459B41F2
:10DC30005B42DB19C018E4E6002B36DD012300222D
:10DC40009B44BEE51F2140464942091A5846C84038
:10DC50000100202A04D05846234A524490400343EE
:10DC60005A1E934107200B4301000022194018421D
:10DC700009D00F21194004291FD0181D984289414D
:10DC8000030049424907DB080B43984600236FE530
:10DC90000299023B49008C4602998C4589414942D0
:10DCA000C919521861460291AEE701235B4281E730
:10DCB0000299A942ECD36346A9E70021E3E71A1DC4
:10DCC0009A429B415B422E00D2089B4479E5510762
:10DCD0005202120BD7E7C046FF03000002FCFFFF11
:10DCE000FF0700001E0400003E040000F0B5574688
:10DCF000DE464E464546E0B50D000400E80F83467B
:10DD00000903D80F090B82461A488C461F03690085
:10DD10005E00490D3F0B760D81421AD0864211D02C
:10DD20000120B1420FD1BC450DD1A2420BD1D34548
:10DD30001ED0002907D1614611430A00531E9A41A3
:10DD4000100000E00120F0BCBB46B246A946A04648
:10DD5000F0BD01208E42F6D1614639430F001743D2
:10DD60002743F0D15B465246981A431E9841EAE792
:10DD70000020E8E7FF070000F0B557464E4645464D
:10DD8000DE46E0B50D000E034900490D8A46DF0F5F
:10DD9000E90FBC4683B02F4F040080460191580024
:10DDA00019039146360B090B400DBA451DD0B842F8
:10DDB0000DD05746002F2AD13443002824D10A43DE
:10DDC00036D0002C41D163465800013815E011438C
:10DDD00038D15346002B01D12643F4D0019B634533
:10DDE00007D1019B5800013807E026432AD150454E
:10DDF00021D00120019B5F42384303B0F0BCBB46F9
:10DE0000B246A946A046F0BD002CDCD0E6E70028CB
:10DE1000EFD0019B6345ECD18245EADCE1DB8E4229
:10DE2000E7D8DED1C845E4D80020C845E5D2D8E718
:10DE3000002CE2D0DDE7114304D1019B6345D8D12A
:10DE40000020DAE702204042D7E7019B6345E6D095
:10DE5000CFE7C046FF070000F0B557464E4645469F
:10DE6000DE46E0B50D000E034900490D8A46DF0F7E
:10DE7000E90FBC4683B02E4F040080460191580044
:10DE800019039146360B090B400DBA451ED0B84216
:10DE90000DD05746002F27D13443002833D10A43F1
:10DEA00034D0002C40D163465800013815E01143AE
:10DEB00012D15346002B01D12643F4D0019B634578
:10DEC0001DD00120019B5F42384306E0264303D169
:10DED0005045F6D111431CD0022003B0F0BCBB4624
:10DEE000B246A946A046F0BD0028EAD0019B634592
:10DEF000E7D18245E5DC02DB8E42E2D80ED0019B01
:10DF000058000138E9E7002CCDD0D7E7002CE4D049
:10DF1000D7E7019B00206345DFD0D2E7C845D0D8C2
:10DF20000020C845D9D2EAE7019B6345E4D0C8E7A1
:10DF3000FF070000F0B557464E464546DE46E0B5C1
:10DF40001F000B031B0B16009846CA0F4B00040062
:10DF5000924685B05B0D00D1C2E1CC4A934200D11C
:10DF600028E14146420FC9000A43802109041143B8
:10DF7000C2009146C64A884693469B44002300252A
:10DF800001933C037A00FB0F3000240B520D0093E9
:10DF900000D185E1BD4B9A4200D160E1BC4B9C466B
:10DFA000624493440A2D00DD14E1730FE4001C4326
:10DFB00080231B042343F0005246009900264A4068
:10DFC0009246022D11DD0122AA40A6211400C900AB
:10DFD0000C400A4200D0FDE0902189000A4200D0A6
:10DFE000D4E18821114200D0EFE049464A460904B5
:10DFF000140C090C020C0F0015000004000C654302
:10E0000047430195B9462F000D0006005543AC4625
:10E010004D4666432D0CB4446544AE4205D93E00DE
:10E0200080277F02BC46664401964F463F043F0C62
:10E030002E0C2D04ED1902951D0C1B041B0C0095D4
:10E040001D001F0065434F43AC46009D69436C4370
:10E050003D0CA946614449448C4503D980256D0295
:10E06000AC4664443F040D0C3F0C0904C919AC468E
:10E070007518039545462E04360C2F0C3500454384
:10E080007843804638006444AC462D0CA946504382
:10E09000724342444A44904503D980256D02A84604
:10E0A0004044150CA84665462D042D0CAC463500A1
:10E0B0005D4312046244AC467B43009D4044984655
:10E0C0002B006E4365467B4346442D0CAD191F0063
:10E0D0000093A84504D980235B02984647440097E3
:10E0E000039B019E98462B044644984663468E4205
:10E0F00089411B041B0C4344B61849421B195F1885
:10E1000096429241BC465242804691468C45894196
:10E11000A3429B41E044C14449425B429145924144
:10E120000B43804589412D0C494252420A435B19F9
:10E130009B18009A029994464A4663445B02D20DAA
:10E140001A43904672020A43511E8A41F60D164345
:10E150004A4652021643B146DB0154D44D4A5A4452
:10E16000002A00DC18E133005B0715D00F215B4665
:10E170003140042910D04946081D4845894181464F
:10E18000494288444146C90106D54146424A1140A8
:10E1900080228846D2009A18404B9A4200DD2BE13B
:10E1A00041464B464C07DB081C4352054B021B0BF8
:10E1B000520D1AE042460243914600D0E0E09B46F1
:10E1C0000223904608250193DBE6009A9846924682
:10E1D00081460196019B022B00D10DE1032B35D026
:10E1E000012B1BD100220023002412051A435346A1
:10E1F000DB071A432000110005B0F0BCBB46B24655
:10E20000A946A046F0BD012273083240134342469E
:10E21000D2071343994643465B08984680225B46E3
:10E22000D2005A440133002A00DCB6E049464907CF
:10E23000A8D00F214846014004299CD1A2E70F2D08
:10E2400000D1FDE0009BA0469A46B146802342469D
:10E250001B0313431B034C460C4A1B0BC5E70B491E
:10E2600033008C462343E344002B77D1022129431A
:10E270000A29AFDC5046009C60408246002D00D148
:10E280000EE10D00002002269DE6C046FF070000BB
:10E2900001FCFFFFFF030000FFFFFFFEFE07000081
:10E2A000230033434BD0002C00D1BBE0200000F012
:10E2B000F1FD030002000B3B1D20C31A3000D840C3
:10E2C00011000300300008398C4088402343594630
:10E2D0008A1A78498B4693440A2D00DC6CE679E76C
:10E2E00043460343994623D04346002B00D187E0A1
:10E2F000404600F0CFFD0B235B429C460200844465
:10E3000011004046083988401D23804660461B1A8C
:10E310002000D840030040460343984623008B402A
:10E320009946644B00259B1A9B460023019328E6DF
:10E33000002398469B4601330425019321E60122E0
:10E3400015430A2D00DD45E7524600994A409246A2
:10E35000022D00DC46E70020012634E603231D439E
:10E360000A2D00DD6BE75346009A882153400122B5
:10E37000AA409A4603262300114200D135E624E73D
:10E380009B46032381460C250193FAE500239A4618
:10E390008023494A1B0328E75B460121891A382953
:10E3A00000DD1FE71F295ADD1F204042821A404628
:10E3B000D040202908D0414A9446424663449A40BE
:10E3C00013004A461A4391464A460721531E9A4172
:10E3D0000C00024300231440114209D008311140BF
:10E3E000042960D0111D9142A4410A0064426407CF
:10E3F000D20814430022F8E6002300242E4AF4E653
:10E4000000F048FD15239C468444020063462032F8
:10E410001C2B00DC74E70023994623000838834056
:10E4200098467EE700F036FD0300020015332032E7
:10E430001C2B00DC40E7330008388340002046E70F
:10E44000802342461B031A4200D1FFE61C4200D043
:10E45000FCE6009A234392463400174AC5E6184A60
:10E46000404694464A4663449840CA4010434A4650
:10E470009A40531E9A4143460243CB40510709D06C
:10E480000F211140042905D0111D914292415242A1
:10E490009B180A00190208D5012200230024A4E6D3
:10E4A00000230024A1E60024A2E75C075B021B0B0B
:10E4B0009EE7C0460DFCFFFFFF0700003E04000082
:10E4C0001E040000F0B54E464546DE465746E0B510
:10E4D00083B0009001910D034E000199760DCC0F91
:10E4E000690A009D6D0F0D43009900920193C800C9
:10E4F0001903019BCB4A5B005B0D9946019B834648
:10E50000DB0F98464B0A0099490F1943009BDB002B
:10E510009C469A46914500D173E0012347465F40EF
:10E520004B46B846F31ABC4216D0002B00DC9AE2E8
:10E530004F46002F00D082E067460F4300D13AE1FA
:10E540005F1E012B00D1A4E2934200D12EE1382FAF
:10E5500000DD43E23B003EE1002B00DCD7E24F460A
:10E56000002F00D0F8E067460F4300D123E15F1E83
:10E57000012B00D157E2934200D117E1382F00DC84
:10E5800004E380221204154200D1AAE31E00150004
:10E590000027A44B01369E4200D103E10122A24B89
:10E5A0003A401D4079081143EA070A436D085307B2
:10E5B00009D00F231340042B05D017003A1DBA428F
:10E5C000BF417F42ED192B0200D477E39549013614
:10E5D0008E4200D1E6E0944973050D405B0D69075A
:10E5E000D2086D020A432D0B1B052B43E40723437E
:10E5F0001000190003B0F0BCBB46B246A946A046C5
:10E60000F0BD8A4BF21863460B434CD0444550D0C2
:10E61000002A6CD0002E00D17DE1634644464F07AE
:10E62000DA081743C8083A00024300D1CDE080253C
:10E630002D0305432D033A007A4B2D0BD4E7964268
:10E6400000D1B3E0382B00DCC2E0471EB842804165
:10E6500040422D1A2B02B1D50127754D7F4228006B
:10E6600000F018FC0838202339001A1A8540D140E0
:10E6700087402943B04200DA45E1801B01301B1A74
:10E680003D009F40C5407A1E97410A009A402F43A3
:10E690003A43C14013000D0000260B4300D086E72B
:10E6A00000220025A0E7474601235F40B8464445C5
:10E6B000AED1002A00D1EFE0002E00D088E14B4619
:10E6C0002A00024300D1A0E25A1E012B00D1B7E27A
:10E6D000544EB34200D17BE1382A00DC12E380259E
:10E6E0002D04294200D112E31E00002751E7514AB0
:10E6F000731C134200D0F4E062462B000A4303432C
:10E70000002E00D074E1002B00D123E2002A00D1BA
:10E71000E0E06346C71AB842924180266B1A524223
:10E720009B1A3604334200D1C1E26346181A84456D
:10E7300092414D1B5242AD1A0124020043462A4326
:10E740001C40002A00D1DBE0354200D1E9E2364B23
:10E7500002001D40012342E7964227D0382B00DDFE
:10E7600011E18022120411431F2B00DDA1E12022C0
:10E770000F00D21A914697406246DA401743B846D6
:10E7800062464F46BA40D940571EBA4147466D18B7
:10E7900017433F188742804140422D182B0200D575
:10E7A000F7E634E03300002500221DE7C0086F07BC
:10E7B0000743E80837E7C7086A071743194AE80814
:10E7C000934200D12FE73A00D8E0164B00250BE723
:10E7D0008022120411431F2B00DDB7E020220F001E
:10E7E000D21A914697406246DA401743B8466246CD
:10E7F0004F46BA40D940571EBA4147466D1A174393
:10E80000C71BB842804140422D1A2B0216D47B0709
:10E8100000D179E20F233B40042B00D0CEE6330039
:10E82000FF08C9E7FF070000FFFF7FFF01F8FFFFB8
:10E83000FFFF7F00FE070000444601266D026D0ABF
:10E84000002D00D00BE7380000F024FB0300183047
:10E850001F2800DC07E73900083B9940864200DDAD
:10E8600087E0831B581C1F2800DC14E20A001F3BB2
:10E87000DA40202805D040231B1A99404B1E9941AD
:10E880000A43002A3CD00026530700D091E6170027
:10E8900035003300FF088FE7CA4A731C13427AD150
:10E8A0002B000343002E00D092E162460A43002B66
:10E8B00000D1F4E1002A0DD06346C7188742804199
:10E8C0006D1840422D182B0200D512E23A00BB46CB
:10E8D0002A4315D05B466A07DF083A430023E8085D
:10E8E0004CE06346C71AB84292416B1A52429B1AD7
:10E8F0001A0200D587E03A001D001A43A0D1002477
:10E900000023002570E6B04D361A0D407B0700D07D
:10E9100080E7330084E74B462A0002437ED05A1E2C
:10E92000012B00D11FE1A94CA34200D198E1382A64
:10E9300000DC9CE16246571EBC45924152428D1A52
:10E9400044461E002A0200D586E637E61A000F006C
:10E95000203AD740B846202B05D04022D31A994000
:10E9600063460B439A4657467B1E9F4143461F43CF
:10E9700046E7954A331A11404A07C80805035B0564
:10E980002D0B5B0D30E680231B041D4200D1FBE004
:10E990001D000027FDE58D4A934200D103E7624642
:10E9A000821882428041691840420818C7075208FD
:10E9B00017434508520700D4AEE10F221E003A402B
:10E9C000042A00D0FAE5FF086A073A430009D5E7B0
:10E9D00063464F07DA081743C80824E6471EB842C3
:10E9E000804140422D1A1E002A0200D534E6E5E59A
:10E9F000002B00D00DE1002A00D069E18025002421
:10EA0000724B2D03F0E563461F1ABC459241012469
:10EA100043464D1B5242AD1A1C4011E76246444624
:10EA20000D00D708C8E66346C618864280416918BB
:10EA3000404209180B0200D40CE1634B70081940E6
:10EA4000CB0703434A08400700D43BE10F2018409E
:10EA5000042800D136E11F1D9F42AD416D420223C3
:10EA6000AD18FF08A8E6002B00D140E64B469B1BE3
:10EA7000002E00D150E7382B2EDD63465F1EBC45CB
:10EA8000924152428D1A44464E462B0200D5E3E590
:10EA900094E56346C71AB84280416D1A40422D1A68
:10EAA0002B0200D5C9E66A07FF0801233A43E808AC
:10EAB00064E71A000F00203AD740B846202B05D053
:10EAC0004022D31A994063460B439A4657467B1E11
:10EAD0009F4143461F435CE680223C0012041543DD
:10EAE0001F2B26DC20222F00D21A060090409740D0
:10EAF000DE40421E9041DD4037430743491B6346D9
:10EB0000DF1BBC45924152424E468D1A7DE6002BDA
:10EB100000D1C1E64B469B1B002E00D1D0E5382B1F
:10EB200036DD80252D04294200D1DDE04E46002748
:10EB30002FE51A002E00203AD640202B05D0402287
:10EB4000D31A9D402F000743BB465F467B1E9F4163
:10EB50003743D4E7002A00D1D1E6012443460D0013
:10EB6000E3461C40B6E663461F1ABC4592414D1B66
:10EB70005242AD1A2B0200D55EE66A07FF084446F2
:10EB800001233A43E808F9E6471C17E53B00EBE5AB
:10EB90008022120415431F2B6CDC20222F00D21A76
:10EBA000060090409740DE40421E9041DD403743D2
:10EBB0000743491967446745924152424E465518EA
:10EBC000ECE5C046FE070000FFFF7FFFFF070000E7
:10EBD000002B00D1FCE6C7086B071F436346E8081B
:10EBE0000B4300D11FE580231B03184207D0CA083E
:10EBF0001A4204D163461000DF0849070F437B0F18
:10EC0000FF00FF085B071F430DE562460D00D708B4
:10EC1000D2E5C7086B071F43E808002A00D102E5C8
:10EC200080231B031842EAD0CA081A42E7D1634680
:10EC30000124DF084346490710000F431C40DEE76C
:10EC400060446045924169185242891806000B02DF
:10EC500000D5F2E64A07F60801233243C8088DE6DC
:10EC60006346DF084B0744461F43C808DBE44446BD
:10EC7000130035E71A002E00203AD640202B05D08D
:10EC80004022D31A9D402F000743BB465F467B1EA0
:10EC90009F4137438EE7202300271B1AF5E400230A
:10ECA000002A00D192E567460D00FF0884E53A008E
:10ECB0001A4300D123E61D00BB460BE617003300C4
:10ECC000FF0879E5DB0852071A430809022355E6D5
:10ECD00063460124DA0843464F071743C8081C401F
:10ECE000A1E41E00471C69E467460D004E4601374B
:10ECF00064E40F4BFF081D406A076D0201233A438D
:10ED00002D0B71E4130046E73300FF0854E5674616
:10ED10000D001E00013751E46A07FF083A4300095D
:10ED20002CE6C0086A0702430023E80826E6C0462E
:10ED3000FFFF7FFFF0B5C6461E03360BB0460D4EF3
:10ED40000C034D005F0000B5240B6D0D7F0DB54227
:10ED50000BD0084900208F4204D1464616433000AC
:10ED6000431E984180BCB846F0BD04430120002CEE
:10ED7000F8D1EEE7FF0700000B00020070B5164D5A
:10ED80000C0382B04900002000920193240B490D2E
:10ED9000DE0FA94204DD1148814203DD104BF0185B
:10EDA00002B070BD8020400320430E4C641A1F2C1B
:10EDB00008DD0D4B5B1AD84003005842002EEFD1FE
:10EDC0001800EDE7094B009A9C46030061448B4014
:10EDD000E2401343F1E7C046FE0300001D040000BB
:10EDE000FFFFFF7F3304000013040000EDFBFFFF73
:10EDF00070B5002816D0C317C5185D40C40F280091
:10EE000000F048F8104B1B1A5B055B0D0A2814DC58
:10EE100002002E00153296400B22121AD5402D0307
:10EE20002D0B03E000240023002500261B052B43A7
:10EE3000E40723433000190070BD0B3885402D03D3
:10EE400000262D0BF2E7C0461E04000010B5041E7C
:10EE500010D000F01FF80E4B1B1A5B055B0D0A2843
:10EE60000FDC0B222100121AD14015300A03844016
:10EE7000120B01E0002300221B05134320001900A0
:10EE800010BD22000B38824012030024120BF3E75E
:10EE90001E0400001C2101231B04984201D3000C16
:10EEA00010391B0A984201D3000A08391B099842FD
:10EEB00001D30009043902A2105C40187047C04613
:10EEC0000403020201010101000000000000000033
:10EED00010B5002903D1FFF7DDFF203002E0080064
:10EEE000FFF7D8FF10BDC0462564257320257300A9
:10EEF0002869290052414E202300257500256425EC
:10EF0000732025733F002564257320257320257306
:10EF1000004E414E002D494E46002E2525302564D9
:10EF20006C6C7500256C6C7500204525640025739C
:10EF30002563257300257320202563257300257321
:10EF4000202B25732025630025732025732025633E
:10EF500000524E4400476F20546F204C696E653A52
:10EF600000476F20546F204C424C3A0047544F20CA
:10EF70004C424C3A0053544F0052434C00464958BF
:10EF80000053434900454E4700534F4C5645204CD3
:10EF9000424C3A0058201920004453450049534739
:10EFA00000494E54454752415445204C424C3A008A
:10EFB00044656C657465205072676D3A00536574E2
:10EFC00020466C61673A00436C65617220466C6153
:10EFD000673A00436865636B20466C61673A00548A
:10EFE0004553543A00257320005F0050726F6772DA
:10EFF000616D2025630050726F6772616D2025641A
:10F000000052756E6E696E67002E202E202E0059FC
:10F010003A00583A00446976696465206279203084
:10F0200000496E76616C69642074797065004E6F7A
:10F03000206C6162656C004C6162656C206578696A
:10F04000737473004F7574206F66204D656D004DAD
:10F0500061782049746572732052656163686564E4
:10F060000041626F72740068006825630066007278
:10F07000616400677200201000205000201C2000F6
:10F0800020102000475342204C424C3A0050696304
:10F090006B204C424C3A0052756E204C424C3A0068
:10F0A000256420005061737465207072674D656D32
:10F0B0006F72793A0D0A0058201120300058203E16
:10F0C00020300058203C20300058201220300058BA
:10F0D000201320300058203D20590058201120597D
:10F0E0000058203E20590058203C2059005820123A
:10F0F00020590058201320590058203D2030004549
:10F100006D70747900522F5300535152540047537D
:10F11000420047544F00655E5800521B0053494E51
:10F120000031305E5800582019205900434F5300D9
:10F13000595E580054414E00312F5800454E5445F9
:10F140005200454558004348530031003400370011
:10F1500035003800182B0033003600390050534575
:10F16000004C424C004100434C454152201800489D
:10F1700059500044494D004652414300434C4541DB
:10F18000522052454700436F6D7020636F6E6A00D6
:10F1900072756E54696D650059202B2069582019CD
:10F1A00000524553554C54004D4154524958007833
:10F1B00021001C5200792C72001C482E4D53004C2B
:10F1C0002E522E001C5241440050792C780052657A
:10F1D000201920496D001600534F4C564500585ECB
:10F1E000320052544E00485950201D004C4E0052DF
:10F1F0001A0053494E201D004C4F4700494E540001
:10F20000434F53201D00434C20580054414E201DB5
:10F21000001725004C41535420580014004142531C
:10F22000004D45414E001C50005346005354444588
:10F2300056001C4800434600182D001C444547005A
:10F24000463F00475241440043792C7800544553CF
:10F25000540053544F2B0053544F2D0053544F2AF6
:10F260000053544F2F0052434C2B0052434C2D005F
:10F2700052434C2A0052434C2F0000000000000073
:10F2800000000000000000000000000000000080FE
:10F290000000E0FE422EE63F0000E0FE422EE6BF08
:10F2A000763C7935EF39EA3D763C7935EF39EABD80
:10F2B000000000000000E03F000000000000E0BF90
:10F2C0002024282C383C4044484C02070208020104
:10F2D00000030109030402040205030500060007F8
:10F2E0000008000A0100000000000000000000000B
:10F2F000000000000000000000000040FB21F93F7A
:10F30000000000002D44743E000000809846F83C48
:10F310000000006051CC783B00000080831BF03976
:10F320000000004020257A38000000802282E33669
:10F33000000000001DF3693500000000B7F0000078
:10F34000BDF00000C3F00000C9F00000CFF00000E5
:10F35000D5F00000DBF00000E1F00000E7F0000075
:10F36000EDF00000F3F00000F9F0000000000000F4
:10F370004FBB610567ACDD3F182D4454FB21E93FCD
:10F380009BF681D20B73EF3F182D4454FB21F93FBC
:10F39000E2652F227F2B7A3C075C143326A6813C42
:10F3A000BDCBF07A8807703C075C143326A6913CED
:10F3B000182D4454FB21E9BFD221337F7CD9024070
:10F3C000D221337F7CD902C0000000000000008001
:10F3D000182D4454FB210940182D4454FB2109C029
:10F3E000000000000000F03F000000000000F83FB7
:10F3F000000000000000000006D0CF43EBFD4C3EB3
:10F4000000000000000000000000004003B8E23FE0
:10F41000010000000000F03F8A1EBD726654B64035
:10F420004E543EF2A6EFCCC078844D13BFE9CB40DA
:10F430004FFA050429CCB8C06C5C8AE26E56944041
:10F44000CC5CF6234F0B5BC0563BD76877D80440A3
:10F45000AC5913DC0D687EBFA38C9F98E6E76C3E29
:10F460005610B1E5EB4731BE00000000000024401B
:10F470000000000000000000060610387C1010108C
:10F48000050554341C1615060611514A2A24100687
:10F490000610242A4A5111080804423E02023E4244
:10F4A000200505007F3E1C080303403E010707605E
:10F4B00058464146586004046355494102022552AA
:10F4C0000505080C7E0C08050510307E3010060678
:10F4D0001010107C381004040404000E0505605060
:10F4E00068444005056000600060000201015F03A0
:10F4F000030600060505147F147F140505042A7F02
:10F500002A10050523130864620505364951225067
:10F5100001010602023E410202413E050544281057
:10F520002844050510107C1010020240300505101B
:10F530001010101002026060030360180605053EFB
:10F540005149453E050500427F400005056251498D
:10F5500049460505224149493605051814127F1010
:10F560000505274545453905053C4A494930050506
:10F57000017109050305053649494936050506495E
:10F5800049291E0202420002024022050508141405
:10F59000222205051414141414050522221414083B
:10F5A0000505020151090608083C023945453D415F
:10F5B0007E05057E0909097E05057F49494936050D
:10F5C000053E4141412205057F4141221C05057F41
:10F5D0004949494105057F0909090105053E4141A0
:10F5E000513205057F0808087F0303417F41050567
:10F5F000304040403F05057F0814224105057F400B
:10F6000040404005057F020C027F05057F0408107D
:10F610007F05053E4141413E05057F090909060573
:10F62000053E4151215E05057F091929460505263C
:10F6300049494932050501017F010105053F404067
:10F64000403F0505071860180705057F2018207F33
:10F650000505631408146305050304780403050510
:10F66000615149454302027F4103030618600202CB
:10F67000417F05050804020408050540404040405C
:10F680000202020404042054547804047F444438E1
:10F6900004043844444404043844447F0404385483
:10F6A00054580303087C0A040418A4A47C04047FAF
:10F6B0000404780303447D400202847D04047C102A
:10F6C000284401017F05057C0438047C04047C0483
:10F6D00004780404384444380404FC4444380404E2
:10F6E000384444FC04047C080404050508545454BC
:10F6F000200303047E4404043C40407C05050C3098
:10F7000040300C05053C403C403C05054464384C09
:10F710004404041CA0A07C030364544C83F9A2009D
:10F72000444E6E00FC291500D1572700DD34F5004A
:10F7300062DBC0003C999500419043006351FE009C
:10F74000BBDEAB00B761C5003A6E2400D24D42006B
:10F750004906E00009EA2E001C92D100EB1DFE00D4
:10F7600029B11C00E83EA700F535820044BB2E00FD
:10F770009CE98400B4267000417E5F00D691390078
:10F78000538339009CF439008B5F840028F9BD0055
:10F79000F81F3B00DEFF97000F980500112FEF00C8
:10F7A0000A5A8B006D1F6D00CF7E360009CB2700F3
:10F7B000464FB7009E663F002DEA5F00BA277500EE
:10F7C000E5EBC7003D7BF100F739070092528A0054
:10F7D000FB6BEA001FB15F00085D8D00300356002F
:10F7E0007BFC4600F0AB6B0020BCCF0036F49A00E7
:10F7F000E3A91D005E619100081BE6008599650084
:10F80000A0145F008D40680080D8FF0027734D0072
:10F8100006063100CA561500C9A873007BE26000D5
:10F820006B8CC000FB21F93FFB2109407CD91240C1
:10F83000FB2119407A6A1F407CD92240BBFD25403C
:10F84000FB2129403A462C407A6A2F405C473140E0
:10F850007CD932409C6B3440BBFD3540DB8F374058
:10F86000FB2139401BB43A403A463C405AD83D400F
:10F870007A6A3F404C7E40405C4741406C104240B9
:10F880007CD942408CA243409C6B4440AC34454000
:10F89000BBFD4540CBC64640DB8F4740EB58484058
:10F8A000FB21494000000000F9AC000079A50000F0
:10F8B00009360000C5690000C9010000A5A50000C7
:10F8C000A18D00000D6A0000E50100003D840000EC
:10F8D000D56B0000556A0000F18E0000A184000085
:10F8E000556D0000C16A0000918F00004D8E000030
:10F8F000656F000089830000299A0000299A0000A2
:10F9000005280000B53300007D2700008727000090
:10F91000A5270000C3270000E12700009127000071
:10F92000AF270000CD270000F97400009B270000DE
:10F93000B9270000D7270000057600009974000061
:10F9400025740000356B0000F9AC00008DA30000A9
:10F95000F7A60000C5A6000000000000719F00008F
:10F9600003020000CFA6000000000000F195000097
:10F9700019020000D9A60000FD770000D19F000009
:10F98000699B0000E3A60000B10200003102000004
:10F99000BD9B0000EDA60000A59D0000A59D0000F8
:10F9A000250200000102000079780000A502000095
:10F9B000B5920000699000001D7900006576000096
:10F9C00081930000F59000005585000081770000CC
:10F9D0006994000081910000C57A00001185000043
:10F9E0005195000011920000F9AC0000B17E0000BA
:10F9F000B1050000217B000000000000350300007D
:10FA0000DD0200006D7B000000000000ED860000BC
:10FA1000397D0000B57B000065810000D97E0000C3
:10FA2000A57D00004D7C000061030000558C0000A6
:10FA3000497E0000A17C00001D8700001D8700009A
:10FA40009D860000017D00006987000055030000CD
:10FA50007D960000B30200000988000005800000C8
:10FA60001D970000C1020000C18100000D8100004F
:10FA7000C5970000CD020000CD8200005D98000017
:10FA8000AD06000089060000AD890000018A000073
:10FA9000558A0000B58A0000158B00005D8B0000C0
:10FAA000A58B0000FD8B0000FFF0000000000000AF
:10FAB00005F100000000000009F100000000000056
:10FAC0000EF1000012F1000016F10000000000002D
:10FAD0001AF100001DF1000021F1000075EF000097
:10FAE00026F100002CF1000030F1000079EF000059
:10FAF0000000000034F1000038F100003CF100008B
:10FB00003CF1000042F1000046F10000BBF00000B3
:10FB10004AF100004CF100004EF100000DF0000031
:10FB2000E0F1000050F1000052F1000054F100003B
:10FB300057F1000059F100005BF1000055F10000A1
:10FB400039F2000073F2000078F2000000000000BB
:10FB50005DF1000061F1000065F1000000000000AF
:10FB600067F100006FF1000010F1000000000000DC
:10FB70000000000073F100007AF1000077F100004E
:10FB80007CF1000086F10000C7F1000000000000D9
:10FB900090F1000098F100009BEF0000F4EE0000EF
:10FBA000F4EE0000A1F10000A8F10000AFF10000A8
:10FBB000B2F100009DF100007DEF0000B5F1000002
:10FBC000B9F1000099EF000081EF0000BFF10000E3
:10FBD000C4F100009DEF000085EF0000C9F10000B6
:10FBE000CEF10000D6F10000D8F1000000000000C6
:10FBF0000000000000000000DEF100000000000036
:10FC0000E2F10000E6F10000ECF10000000000006D
:10FC1000EFF10000F2F10000F8F10000FCF100004B
:10FC200051EF000000F2000012F20000000000009E
:10FC300006F200000BF2000011F2000014F20000C6
:10FC400014F200001BF200001DF2000021F200007F
:10FC500026F2000029F200003CF200002CF2000025
:10FC600032F2000035F20000C5F1000038F2000069
:10FC70003BF2000040F2000043F2000048F20000B6
:10FC80004DF20000000000000000000052F20000F1
:10FC900057F200005CF2000061F2000066F2000022
:10FCA0006BF2000070F2000075F200003CD9000019
:10FCB000F0D7000068D7000092D7000068D7000096
:10FCC000D4D8000068D7000092D70000F0D7000019
:10FCD000F0D70000D4D8000092D700008AD70000E7
:0CFCE0008AD700008AD70000F6D8000088
:08FCEC00F8CFFF7F01000000CA
:10FCF400583A001F2C0000004D000000F8010010CD
:10FD0400180000100000000000000000E8120010BD
:10FD140050130010B8130010000000000000000091
:10FD240000000000000000000000000000000000CF
:10FD340000000000000000000000000000000000BF
:10FD440000000000000000000000000000000000AF
:10FD5400000000000000000000000000000000009F
:10FD6400000000000000000000000000000000008F
:10FD7400000000000000000000000000000000007F
:10FD8400000000000000000000000000000000006F
:10FD9400000000000000000000000000000000005F
:10FDA40001000000000000000E33CDAB34126DE6FC
:10FDB400ECDE05000B000000000000000000000065
:10FDC400000000000000000000000000000000002F
:10FDD400000000000000000000000000000000001F
:10FDE400000000000000000000000000000000000F
:10FDF40000000000000000000000000000000000FF
:10FE040000000000000000000000000000000000EE
:10FE140000000000000000000000000000000000DE
:10FE240000000000000000000000000000000000CE
:10FE340000000000000000000000000000000000BE
:08FE44000000000000000000B6
:040000030000B259EE
:00000001FF
